:100000000C94D00F0C94F80F0C94F80F0C94F80F7C
:100010000C94F80F0C94F80F0C94F80F0C94F80F44
:100020000C94F80F0C94F80F0C94D0150C941B6CD6
:100030000C94996E0C944A6C0C94F80F0C942F1637
:100040000C94BE150C94F80F0C9410750C94E0737E
:100050000C94F80F0C94F80F0C94F80F0C94F80F04
:100060000C940B6F0C9479160C94B46C0C944B6F2D
:100070000C94F80F0C94F80F0C94F80F0C94F80FE4
:100080000C94F80F0C94F80F0C94F80F2018251806
:10009000EB17F117F717F717F71716181B18201893
:1000A00025182A182F1835184D440D441844274494
:1000B0002D44314436441E4C344C424C574C654C14
:1000C000744C864CAC4CD54CE34C094D274D354D0A
:1000D000434D514DA4698E698869926997699D69FC
:1000E0008B69A169A669AD70B370C070C970DF700B
:1000F000F8700B711A712E7143714C7169716F71C7
:1001000077717C718171E971F371897190719A7164
:10011000A471AA71AE71B571D071D571DA71E27145
:10012000B970B971C071C871204F6C642056657286
:1001300073696F6E20454550524F4D202020434833
:1001400045434B2053455454494E47532F43414C4C
:10015000494200416C61726D732044697361626C45
:10016000656400506C656173652052657365742029
:100170005377697463686573005468726F74746C44
:1001800065206E6F742069646C65005265736574D8
:10019000207468726F74746C6500454550524F4D01
:1001A000206C6F77206D656D004C4F4144494E4780
:1001B000006D537461636B206F666C6F77006D53D5
:1001C0007461636B2075666C6F77004D45535341C6
:1001D000474500414C45525400707265737320616D
:1001E0006E79204B657900507265737320616E796A
:1001F000206B657920746F20736B697000414C45EA
:10020000525400034F4646414253525573525525AE
:10021000454C73454C25544873544825414C734113
:100220004C2550312050312550322050322550334A
:100230002050332500544852525544454C454944BA
:100240003049443149443241494C47454154524E6A
:1002500053573153573253573353573453573553FA
:1002600057365357375357385357395357415357C6
:1002700042535743002D2D2D004348002D2D2D2096
:10028000000450312020503220205033202048419B
:100290004C4646554C4C43594331435943324359DC
:1002A000433350504D3150504D3250504D335050DB
:1002B0004D3450504D3550504D3650504D375050B4
:1002C0004D38434831204348322043483320434887
:1002D000342043483520434836204348372043489C
:1002E000382043483920434831304348313143486E
:1002F0003132434831334348313443483135434840
:10030000313633504F5347563120475632204756E7
:100310003320475634204756352047563620475617
:100320003720002D2D2D2D0000006428100703011B
:1003300052554420454C45205448522041494C20B8
:100340000001020304010302040402030104030286
:10035000014F4E20004F4646001B1E272D36394BBD
:100360004E636C7278878D939CB1B4C6C9D2D8E1C4
:10037000E453706C6173680080400000000000006E
:10038000000000000000000000000000000000006D
:10039000000000000000000000000000000000005D
:1003A000000000000000000000000000000000004D
:1003B000000000000000000000000000000000003D
:1003C000000000000080C0E0E0F0F8F8FCFCFCF861
:1003D000F8F8F0400000000000808080000000007D
:1003E000000000000000000000000000000000808D
:1003F000C0C0E0E0E0F0F0F0E0C00000000000C0AD
:10040000F8FFFF9F8783838383838383838383832F
:10041000838383838383838383838303838083832F
:10042000838383838383838383838383838383839C
:100430008383838383C3E3733F1F0000000080E056
:10044000F0F8FCFEFFFFFFFF7F3F1F1F0F0783C376
:10045000E1E1E0E0C0000E1F3F7F7FFFF3E0E080BE
:100460000000000000000000000080F0FCFEFFFF24
:10047000FFFF7F3F0F0301010100000080F0FEFF3E
:10048000FFC7C1C1C1C1C1C1C1C1C1C1C1C1C1C118
:10049000C1C1C1C1C1C1C1C101C1F0FEFF3F0F0750
:1004A0000F0D0D0D1D19191919313131317161619E
:1004B00061E1C1C1C18100000080E0F8FCFFFFFFE5
:1004C000FF2F170F038180C0E0F0F8FCFEFFFFFF55
:1004D000FFFFFF7F01000000000000000101030793
:1004E000070E1E1C3870E0F0F8FEFFFF7F1F0F03A1
:1004F00000010000000000000000000000000000FB
:1005000000000000000000000000000000000000EB
:1005100000000000000000000000000000000000DB
:1005200000000000000000000000000000000000CB
:1005300000000000000000007EFFFFFFFFFFFFFB48
:10054000F8FCFCFEFF7F3F1F0F07C3FFFFFFFFFF0D
:10055000FF7F070000000000000000000000000016
:1005600000C0E0F8FEFFFF7F1F0F1F3D7CF8F8F092
:10057000E08000000000000000000000000000001B
:10058000000000000000000000000000000000006B
:10059000000000000000000000000000000000005B
:1005A000000000000000000000000000000000004B
:1005B0000000000000000000000001010101010333
:1005C0000707070301000000E0FCFFFFFFFFFF1F1C
:1005D000030000000000000000000000C0F078DE12
:1005E0002713090E070300000000000000000103AC
:1005F0000F7FFFFC7878F80000000000000000008A
:1006000000008080808080808080800080800080EA
:10061000800000000000000080808080808080805A
:1006200080808080808080808080000000000000CA
:1006300000000000000000000000000000000000BA
:10064000000000000080F0FEFFFFFFFF3F0F0100F1
:1006500000000000000000C0E0381E0F0300010091
:10066000000000000000000000000000000000008A
:100670000000000000030301000000000000000073
:1006800000000E0E02020202020303000F0F000F11
:100690000F080808080808080F0F08080808080FBE
:1006A0000F000000000F0F0000000000000000001D
:1006B000000000000000000000000000000000003A
:1006C000000000C0F8BFFFFFFF1F7F010000000017
:1006D00000000000F0FCFF7F783000000000000008
:1006E000000000000000000000000000000000000A
:1006F00000000000000000000000000000000000FA
:1007000000000000000000000000000000000000E9
:1007100000000000000000000000000000000000D9
:1007200000000000000000000000000000000000C9
:1007300000000000000000000000000000000000B9
:1007400000301C070E0F0701000000000000000031
:100750000000000000000000000000000000000099
:100760000000000000000000000000000000000089
:100770000000000000000000000000204D4F443A3F
:10078000204652534B59204E485420202020002010
:1007900053564E3A20657239782D723739310054EC
:1007A000494D453A2032313A31333A3134004441EF
:1007B00054453A2031312E30352E32303133005607
:1007C0004552533A2056312E3635372D4D696B65DB
:1007D0000056343D0756353D0E56363D0056313DE8
:1007E0000756323D0E56333D00096D706800537058
:1007F000643D096B7473204D61783D00416C743D1C
:10080000096D2020204D61783D004C6F6E3D004CFD
:1008100061743D0041323D0041313D0052504D0078
:100820004675656C0022047C5E54546D0003457867
:1008300070457846466E654D656443727300115489
:100840004F54000153544B115354250001544D454E
:1008500011545357005354415400035B4D454E55BA
:100860005D20746F207265667265736800746D61D7
:10087000696E0F6D7300746D7231204A697474650E
:10088000720F757300746D72314C6174206D696EF6
:100890000F757300746D72314C6174206D61780F47
:1008A0007573005354415432004D6F646500496EB6
:1008B000742E204672736B7920616C61726D0043F7
:1008C000726F73735472696D00456E61626C65205E
:1008D00050504D53494D0042616E64476170005362
:1008E0007469636B5363726F6C6C00506F74536305
:1008F000726F6C6C00416C61726D205761726E6931
:100900006E67004D656D6F7279205761726E696E0A
:10091000670044656661756C742053770054687293
:100920006F74746C65205761726E696E67005370E6
:100930006C617368204E616D650053706C61736803
:100940002073637265656E004C69676874206F6E12
:100950002053746B204D76004C69676874206F6675
:1009600066206166746572004261636B6C696768DA
:100970007420696E76657274004C696768742073C0
:10098000776974636800466C617368206F6E2062DB
:10099000656570004265657020636F756E74646F85
:1009A000776E004D696E75746520626565700054E0
:1009B00068726F74746C6520726576657273650019
:1009C000496E616374697669747920616C61726DD6
:1009D000136D0042617474657279207761726E697B
:1009E0006E6700436F6E74726173740020486170AB
:1009F00074696320537472656E6774680020537065
:100A000065616B657220506974636800566F6C7520
:100A10006D65000A4265657065722020202050696E
:100A200053706B72202020204265657072566F698A
:100A30006365506953706B566F69636500536F75DA
:100A40006E64204D6F646500065175696574204EB3
:100A50006F4B6579207853686F727453686F727446
:100A6000204E6F726D20204C6F6E672020784C6F87
:100A70006E672000426565706572004F776E657223
:100A8000204E616D6500524144494F2053455455F5
:100A90005000036D6F64650A252073726320207314
:100AA000770043616C004D756C7469706C69657298
:100AB000000363683163683263683363683400033A
:100AC0006F6666202B3D203A3D0007536C617665CA
:100AD00000000303030300545241494E455200569F
:100AE000455253494F4E005472696D2D202B00051D
:100AF000204D656E75204578697420446F776E20AF
:100B0000202055705269676874204C6566740044F3
:100B100049414700424700414E4100034D4F564571
:100B200020535449434B532F504F545300055345C2
:100B300054204D4944504F494E5400035B4D454E9F
:100B4000555D20544F2053544152540043414C4969
:100B500042524154494F4E000966726565004D4F3F
:100B600044454C53454C00464D00464D300F5245D0
:100B70005441004D4F444553005472696D73005306
:100B80007769746368000003464C204D4F4445006C
:100B900001524554410044454C455445204D4F4475
:100BA000454C0F5B4D454E555D00543254685472B0
:100BB000696700547261696E657200452E204C6948
:100BC0006D6974730003504F534E45470053686975
:100BD00066742053656C0050504D2031737420436F
:100BE00068616E004C50342F4C5035202044534DDA
:100BF000326F6E6C792044534D322F44534D580060
:100C000044534D20547970650053656E64205278CA
:100C1000204E756D626572205B4D454E555D0050EE
:100C2000504D2046724C656E0D6D536563000B523E
:100C3000784E756D000434434820364348203843CD
:100C4000482031304348313243483134434831360B
:100C50004348001375530011755365630050504DA0
:100C600020202050585820202044534D322020501E
:100C7000504D31362050504D53494D0050726F74D5
:100C80006F00524554413132330042656570204354
:100C90006E74005472696D20537700064578702099
:100CA0002020457846696E6546696E6520204D6551
:100CB0006469756D436F61727365005472696D206C
:100CC000496E6300542D4578706F00542D5472693D
:100CD0006D000A436F756E7420446F776E436F75B5
:100CE0006E742055702020005472696767657242E7
:100CF000005472696767657200566F6963652049C1
:100D00006E646578114D454E55004E616D6500006D
:100D100009000100000000000000060200534554D5
:100D20005550004475706C69636174696E67206D1D
:100D30006F64656C0044454C455445204D4F444517
:100D40004C004455504C4943415445204D4F444577
:100D50004C00657870202025202073773120737730
:100D6000320000034558504F2F445200445220484F
:100D7000696768004452204C6F77004452204D69E7
:100D800064004472537732004472537731005765E0
:100D900069676874004578706F00004558504F2FA0
:100DA000445200012B2A52004D495845520003205D
:100DB00044454C455445200003204D4F56452020C6
:100DC00020000320434F5059202020000320494E8B
:100DD000534552542000032045444954202020000C
:100DE00044454C455445204D49583F00035B4D4513
:100DF0004E555D0B5B455849545D00035945530BF7
:100E00004E4F005072657373205B455849545D2006
:100E1000746F2061626F7274004D6178206D697823
:100E20006572732072656163683A20333200025341
:100E30006C6F77202055700002536C6F7720204430
:100E40006F776E000244656C617920557000024432
:100E5000656C617920446F776E00084164642020DE
:100E60002020204D756C7469706C795265706C61CE
:100E700063652000024D756C7470780002576172D2
:100E80006E696E6700025377697463680043757218
:100E90007665000D4469666600025472696D000251
:100EA000466C4D6F64657472696D00024669782006
:100EB0004F6666736574004F666673657400466DB1
:100EC0005472696D56616C000257656967687400F9
:100ED00002536F757263650045444954204D49586B
:100EE0002000494E53455254204D49582000032DAF
:100EF0002D2D783E30783C307C787C663E30663CE8
:100F0000307C667C6331206332206333206334207D
:100F100063352063362063372063382063392063CC
:100F200031306331316331326331336331346331B2
:100F300035633136000E4F6E00072D2D2D2D2020EC
:100F400020763E6F66732020763C6F667320207C8F
:100F5000767C3E6F66737C767C3C6F6673414E4454
:100F6000202020204F522020202020584F52202087
:100F7000202076313D3D7632207631213D7632207B
:100F800076313E7632202076313C76322020763122
:100F90003E3D76322076313C3D76322054696D6597
:100FA0004F6666005357000003435553544F4D207E
:100FB000535749544348455300064F4E20202020A4
:100FC0004F4646202020424F54482020313553655B
:100FD000637333305365637336305365637356619F
:100FE0007269626C005653000720382053656373A2
:100FF0003132205365637331362053656373004E7D
:10100000756D62657220566F6963652053770000C5
:1010100000025341464554592053574954434845CB
:101020005300032D2D2D52746D45746D54746D4114
:10103000746D52454E525544454C455448524149B1
:101040004C50312050322050332063312063322005
:101050006333206334206335206336206337206395
:101060003820633920633130633131633132633189
:101070003363313463313563313600475600000144
:10108000474C4F42414C20564152530043757374B4
:101090006F6D20446973706C617900477073416CA7
:1010A000744D61696E00566F6C742054687265737C
:1010B0003D00034F464631323234303000416C74CB
:1010C000416C61726D004E756D20426C6164657398
:1010D000006D416820416C61726D00547852535329
:1010E00049616C726D00000101010054454C454D91
:1010F000455452593200013C3E00616C726D000152
:10110000762D5641004120206368616E6E656C004B
:10111000034D6574496D70000546724875625753FA
:101120004868690055737250726F746F0000010156
:101130000202010254454C454D4554525900434F5B
:101140005059205452494D205B4D454E555D00008D
:10115000034C494D4954530043560043555256459C
:10116000530050524553455400454449542D3E00C8
:101170000900435552564500032D2D2D494E56006A
:101180004756005B4D454E555D205748454E20441F
:101190004F4E4500F94FCB290027852605267C2B8D
:1011A0002037D956D335D733334E415B6D4D555526
:1011B0009F5C2E27A02C282912081200081C080862
:1011C000081C080000082200490022080000000056
:1011D00000227F22000000082200490022080000AF
:1011E00008220049002208000000227F220000009F
:1011F0000000082200490022080000081C08080816
:101200001C080001010100000002020202020202A9
:1012100002020200020202020202020200000000B8
:1012200000000002065761726E31205761726E3203
:101230002043686561702052696E6720205363699E
:10124000466920526F626F7420436869727020543F
:101250006164612020437269636B74536972656EC7
:1012600020416C6D436C6B526174617461546963AD
:101270006B20204861707463314861707463324838
:1012800061707463330054696D65720041203D00E4
:10129000032D2D2D59656C4F7267526564005452B1
:1012A0004530313241470052783D0054783D0020AE
:1012B0004142434445464748494A4B4C4D4E4F50A6
:1012C0005152535455565758595A61626364656672
:1012D0006768696A6B6C6D6E6F7071727374757626
:1012E0007778797A303132333435363738395F2D83
:1012F0002E0000010203FEFF0406080A0B0C0D0E6F
:101300000F23FD202425261D1E1F27F6F7F8F9FAC6
:10131000FBFCF5042D2D2D2D41313D2041323D208A
:10132000525353495453534954696D3154696D3282
:10133000416C742047616C744773706454313D2074
:1013400054323D2052504D204655454C4D61683138
:101350004D61683243766C7442617474416D707390
:101360004D61682043746F744661735641636358DE
:10137000416363594163635A5673706447767231AF
:1013800047767232477672334776723447767235D3
:1013900047767236477672374677617400537769BD
:1013A000746368205761726E696E670067656E7757
:1013B00072697465206572726F7200454550524FB4
:1013C0004D20466F726D617474696E67004261648E
:1013D00020454570726F6D2044617461004D4F442B
:1013E000454C2020202020004D452020202020207A
:1013F000202000454550524F4D206F766572666C37
:101400006F7700A060800000000000000000000076
:1014100000000000FFFF0000000000001F3F000070
:101420003F1F00003030FFFF3030FFFF303030789A
:10143000CCCCFFFFCCCC8C0C060F0F86C0E07038F4
:101440001C0C3CFEC7E3F33B1E0C00000000333BCA
:101450001F0F000000000000F0F81C0E0703000042
:10146000000003070E1CF8F000003030E0C0FCFC68
:10147000C0E03030C0C0C0C0FCFCC0C0C0C0000074
:101480000000000000000000C0C0C0C0C0C0C0C05C
:10149000C0C000000000000000000000000000804C
:1014A000C0E070381C0C00000000000000000000CC
:1014B00000000000383800000000000000000000BC
:1014C0000000000003033F3F03033F3F03030C0CF6
:1014D0000C0C3F3F0C0C07030C0E07030100183CDB
:1014E0003C180F1F383133331E1E33330000000009
:1014F000000000000000000003070E1C3830000050
:10150000000030381C0E07030000030301000F0F1A
:1015100000010303000000000F0F000000000000A6
:10152000333B1F0F0000000000000000000000001F
:1015300000000000183C3C18000000000C0E0703DF
:101540000100000000000000FCFE87C3E377FEFC02
:1015500000000C0EFFFF0000000000000C0E0783CF
:10156000C3E77E3C00000303C3C3C3E7FE3C0000A7
:10157000C0E070381C0EFFFF00003F3F3333337371
:10158000E3C30000FCFEC7C3C3C78E0C0000030307
:10159000C3E3733B1F0F00003CFEE7C3C3E7FE3C01
:1015A00000003C7EE7C3C3E7FEFC0000183C3C188B
:1015B000000000000000183C3C1800000000000083
:1015C000C0E0F0381C0E070330303030303030309F
:1015D000303003070E1C38F0E0C000000C0E07038B
:1015E0000383C3E77E3C00000F1F3B3130381F0FE1
:1015F000000030303F3F3030000000003C3E3733C9
:101600003130303000003030303030391F0F0000C2
:101610000303030303033F3F00000C1C3830303842
:101620001F0F00000F1F383030391F0F000000005F
:101630003F3F0000000000000F1F393030391F0FFE
:101640000000000030381C0E07030000060F0F06D4
:10165000000000000000333B1F0F000000000000EE
:10166000000103070E1C38300303030303030303C5
:10167000030330381C0E07030100000000000000C7
:1016800033330100000000003C7EE7C3C3E77E3C2B
:10169000F0F8DCCEC7C7CEDCF8F0FFFFC3C3C3C38E
:1016A000C3E7FE3CFCFE0703030303070E0CFFFF2A
:1016B000030303070E1CF8F0FFFFC3C3C3C3C3C378
:1016C0000303FFFFC3C3C3C3C3C30303FCFE07037A
:1016D000C3C3C3C7CECCFFFFC0C0C0C0C0C0FFFFE4
:1016E00000000303FFFF03030000000000000303EA
:1016F000FFFF0303FFFFC0E0F0381C0E0703FFFFEE
:101700000000000000000000FFFF0E1CF8F81C0E97
:10171000FFFFFFFF3870E0C08000FFFFFCFE070303
:1017200003030307FEFC00000000000000000000AF
:101730003F3F0000000000003F3F3F3F303030306F
:1017400030391F0F0F1F3830303030381C0C3F3FFE
:10175000303030381C0E07033F3F303030303030EF
:1017600030303F3F00000000000000000F1F383005
:10177000303030303F3F3F3F0000000000003F3F2F
:10178000000030303F3F303000000C1C3830303823
:101790001F0F00003F3F000103070E1C38303F3F82
:1017A00030303030303030303F3F0000000000003B
:1017B0003F3F3F3F0000000103033F3F0F1F383012
:1017C000303030381F0FFFFFC3C3C3C3C3E77E3CB5
:1017D000FCFE070303030307FEFCFFFFC3C3C3C3F1
:1017E000C3E77E3C3C7EE7C3C3C3C3C78E0C030381
:1017F0000303FFFF03030303FFFF000000000000DB
:10180000FFFFFFFF000000000000FFFFFFFF0000E0
:1018100000000000FFFF0F1F38F0E0E0F0381F0F5E
:101820003F7FE0C08080C0E07F3F03030383C3E3CA
:10183000733B1F0F0000FFFF0303030300000C1C9A
:101840003870E0C080000000000003030303FFFFC6
:10185000000030381C0E07070E1C38300000000056
:101860000000000000003F3F0000000000000000FA
:101870000F1F383033371E1C3F333F3F0000030734
:101880000E1C38300C1C3830303030391F0F00003F
:1018900000003F3F000000000F1F3830303030386C
:1018A0001F0F03070E1C38381C0E07030F1F383894
:1018B0001F1F38381F0F3C3E0703010103073E3C42
:1018C000000000013F3F010000003C3E3733313053
:1018D0003030303000003F3F30303030000000000A
:1018E0000000000103070E0C0000303030303F3F95
:1018F0000000000000000000000000003030303028
:10190000303030303030000003070E1C383000001B
:101910000000303030303070E0C0FFFFC0E0703089
:101920003070E0C0C0E07030303030300000C0E0D7
:1019300070303070E0C0FFFFC0E070303030307089
:10194000E0C0C0C0FCFEC7C303070E0CF0F89C0C3F
:101950000C0C0C0CFCFCFFFFC0E070303070E0C0E1
:1019600000003030F3F300000000000000003030D1
:10197000F3F30000FFFF0080C0E0703000000000C3
:101980000303FFFF00000000F0F03070E0E0707033
:10199000E0C0F0F0C0E070303070E0C0C0E0703007
:1019A00030303070E0C00000000000000000000097
:1019B0000C1E3F33333333333F3F3F3F3030303003
:1019C00030381F0F0F1F3830303030381C0C0F1FCD
:1019D0003830303030303F3F0F1F3B3333333333F9
:1019E000030300003F3F000000000000000133330C
:1019F0003333333B1F0F3F3F0000000000003F3FE9
:101A0000000030303F3F303000000C1C38303038A0
:101A10001F0F00003F3F03070F1C3830000000007D
:101A200030303F3F303000003F3F000003030000F4
:101A30003F3F3F3F0000000000003F3F0F1F383096
:101A4000303030381F0FF0F03030303030F0E0C040
:101A5000C0E0F0303030E0C0F0F0F0F0C0E07030C6
:101A60003070E0C0C0E0F030303030300000303056
:101A7000FFFF303000000000F0F000000000000028
:101A8000F0F0F0F0000000000000F0F0F0F00000D6
:101A900000000000F0F03070E0C08080C0E07030E6
:101AA000F0F0800000000000F0F03030303030B056
:101AB000F0F070300000C0E03C3E07030000000082
:101AC0000000FFFF00000000000003073E3CE0C0F4
:101AD0000000C0C0C0C00C1CF8F0E0C0C0E0F0F8CE
:101AE0001C0CC0C0C0C03F3F03030303030301003D
:101AF00000010303030303033F3F3F3F00000000D7
:101B000000000000303133333333333F1E0C00000C
:101B10000F1F383030381C0C0F1F383030381C0C79
:101B20003F3F03070E1C38381C0E07030F1F3838C1
:101B30001C1C38381F0F30381C0F07070F1C38309B
:101B4000000133333333333B1F0F30383C3E3733E0
:101B500031303030000000010F1F3830000000002D
:101B600000003F3F00000000000030381F0F010060
:101B70000000000000000C0E070301000001030735
:101B80000E0C000000005008500000000000000093
:101B9000006F000007000700147F147F14242A7FC1
:101BA0002A122313086462364955225000050300A7
:101BB00000001C2241000041221C0014083E0814B1
:101BC00008083E080800503000000808080808000F
:101BD000606000002010080402003E49453E0000FD
:101BE000427F40006251494600414949360018147D
:101BF000127F0027454539003E49493200017905E9
:101C0000030036494936000649291E0000363600D1
:101C10000000563600000814224114141414144114
:101C200022140800020151090600060909067E096E
:101C300009097E7F494949363E414141227F414160
:101C4000221C7F494949417F090909013E4149490F
:101C50007A7F0808087F00417F41002040413F0112
:101C60007F081422417F404040407F020C027F7F6A
:101C70000408107F3E4141413E7F090909063E416B
:101C800051215E7F09192946264949493201017FC0
:101C900001013F4040403F1F2040201F3F40304057
:101CA0003F631408146307087008076151494543EE
:101CB000007F41410002040810200041417F0004E0
:101CC0000201020440404040400001020400205450
:101CD0005454787F48444438384444442038444479
:101CE000487F3854545418087E0901020C5252524D
:101CF0003E7F0804047800447D40002040443D00BD
:101D00007F1028440000417F40007C041804787C48
:101D10000804047838444444387C14141408081423
:101D200014187C7C080404084854545420043F448C
:101D300040203C4040207C1C2040201C3C40204057
:101D40003C44281028440C5050503C4464544C44AB
:101D5000000836410000007F0000004136080008FE
:101D600008221C08081C22080840800804201002D1
:101D7000010000891112239B322446AD573665BFFE
:101D800074488CC19D5AAFD3BE6CCAE5DB7EE9F7BF
:101D9000F88110080193331A22A5562C47B7753ED7
:101DA00064C99C408DDBBF52AEEDDA64CBFFF9769F
:101DB000E802218B30100299132667AF763444BDB8
:101DC000554AADC3BC588ED19F6EEBE7FA7CC8F57F
:101DD000D983310A2091121803A7772E66B5543C97
:101DE00045CBBD42ACD99E508FEFFB66EAFDD8745F
:101DF000C904428D5316619F702004A9153227BB78
:101E0000364CCEC5DF5EEDD7FC6888E1997AABF33E
:101E1000BA85520C4397711E60A1142805B3373A56
:101E200026CDDE44CFDFFD56ECE9986089FBBB721E
:101E3000AA06638F7214409D512225AB343006B937
:101E4000174EEFC7FE5CCCD5DD6AA9E3B8788AF1FE
:101E50009B87730E6295501C41A3352A24B1163816
:101E600007CFFF46EEDDDC54CDEBB962A8F99A70DE
:101E70008B088481951AA793B62CC2A5D33EE1B7EF
:101E8000F04008C919522BDB3A644EED5F766DFFC6
:101E90007C899400859BB712A6ADD224C3BFF136CE
:101EA000E0C1184809D33B5A2AE55E6C4FF77D7EA6
:101EB0006C0AA583B4188691972EE3A7F23CC0B5AF
:101EC000D14229CB38500AD91B666FEF7E744CFD86
:101ED0005D8BB502A499961087AFF326E2BDD0348E
:101EE000C1C3394A28D11A580BE77F6E6EF55C7C66
:101EF0004D0CC685D71EE597F42880A1913AA3B36F
:101F0000B2444ACD5B5669DF78600CE91D722FFB45
:101F10003E8DD604C79FF516E4A9902081BBB3324D
:101F2000A2C55A4C4BD7795E68E11C680DF33F7A25
:101F30002E0EE787F61CC495D52AA1A3B03882B12E
:101F400093466BCF7A5448DD59622DEB3C700EF905
:101F50001F8FF706E69DD414C5ABB122A0B992300D
:101F600083C77B4E6AD5585C49E33D6A2CF11E78E5
:101F70000F28860A0C0D0B10072828282828282847
:101F8000288488979A111314151609181B122828EB
:101F9000282805191C1D1E1F2720A1222828F0789B
:101FA00011241FBECFEFD0E1DEBFCDBF11E0A0E016
:101FB000B1E0EEECF3EF02C005900D92A832B1074C
:101FC000D9F71EE0A8E2B1E001C01D92AC31B10723
:101FD000E1F71FE1C0EADFE104C02297FE010E94A1
:101FE000A079CE39D107C9F70E941D770C94E57905
:101FF0000C940000E1E2F5E040E0842F806487B9B2
:10200000369A3699FECF24B135B1369A3699FECF3D
:1020100084B195B1820F931F819391934F5F4830A4
:1020200061F70895853050F0883020F08E3020F42C
:1020300082E0089581E0089583E0089580E00895A6
:102040002AE0829FC00111248D519E4F089525E002
:10205000829FC00111248D5D9C4F08958F929F92A5
:10206000AF92BF92DF92EF92FF920F931F93CF93A5
:10207000DF93C82FD62F5A01122FF02E822F847093
:10208000D82E57FF10C0882311F08CE101C08FE0DB
:10209000212F4DE26D2F9C2F981B892F0E94C86421
:1020A000B194A194B108212F2F214AE36D2F8C2FD9
:1020B0000E94C8646CE370E0C5010E9449794B013D
:1020C0005C01012F00619B0140E050E062E0E62EE0
:1020D0006D2F8C2F0E94BA66DD2011F08AE101C0BD
:1020E0008FE00F2D0061950140E050E092E0E92E75
:1020F0006D2F8C0F0E94BA66DF91CF911F910F91C7
:10210000FF90EF90DF90BF90AF909F908F900895D9
:10211000CF93DF93D62FC22F206250E00E94CA6770
:10212000C7FD09C02C2F46E76D2F8091400CDF9131
:10213000CF910C94C864DF91CF910895242F4091E2
:1021400002010C9488100F93022F24FF03C00F7E0E
:102150009CE201C094E2411104C024E043E253E058
:1021600015C04530B0F4E091FA0494E0E99FF00125
:1021700011243197E40FF11DEF5BFC4FE49194E0E3
:10218000E99FA0011124445D5C4F24E00E947D651D
:102190000DC0941728F02BEF240F41E852E004C043
:1021A0002CED240F43E153E10E949F650F910895A8
:1021B0000F93CF93DF93C82FD62F022F411104C066
:1021C00024E04CE752E00EC04A3010F086E101C036
:1021D00081E18C0F50E0202F6D2F0E94CA6722E012
:1021E00049E752E06D2F8C2F0E947D65DF91CF91E2
:1021F0000F9108950F931F93CF93DF93D62FC42F82
:10220000022F16E0180F442341F0463151F04A3EA8
:1022100061F423E045E553E016C023E045E752E0D2
:1022200012C023E041E553E00EC047FF04C041E285
:102230000E94C864C195C1504C2F440F4C0F50E010
:102240004B5C5D4F23E06D2F812F0E947D65DF91F8
:10225000CF911F910F91089585E392E00895DF9249
:10226000EF92FF920F931F93CF93DF93F82ED62F09
:10227000142FE22EC091D40181E08217E0F14FE0EB
:102280004C0F4F31D0F42C2F332727FD309537FFDB
:1022900003C0319521953109012F43E052E06D2FA4
:1022A0008F2D0E949F65CF3FC4F5212F41E26D2FF6
:1022B0008AEF8F0D0E94C86430C074E2D72EDC0E06
:1022C0000AEF0F0D88E48D1520F01C1674F441EF11
:1022D00009C0212F4DE682E18F0D0E94C8641C16B3
:1022E0001CF44CED4C0F01C04D2D212F6D2F802F74
:1022F0000E94FA1012C082E0281313C0212F4091CF
:1023000044046D2F8AEF8F0DDF91CF911F910F91B4
:10231000FF90EF90DF900C94FA10E11002C0C130F2
:1023200069F3DF91CF911F910F91FF90EF90DF90B4
:102330000895EF92FF920F931F93CF93DF9379014C
:1023400024E0629F800111240A591B4FD801EC91AF
:10235000F0E0442311F0EE0FFF1F9F01DC010E940B
:10236000FC78E8012B81207C203C59F424E630E005
:1023700040E050E00E945D79F701808180628083B7
:1023800018C0E436F10578F4660F771F881F991F8F
:1023900023E330E040E050E00E945D79D7018C916A
:1023A00080638C9306C02FEF30E040E050E00E9445
:1023B0005D79C901DF91CF911F910F91FF90EF904F
:1023C0000895DF92EF92FF920F931F93CF93DF93C5
:1023D0001F92CDB7DEB7D82EF62E842FA22F0983F9
:1023E00094E0299F800111240A591B4F50E060E0BE
:1023F00070E0F8019381907C903821F4EE2081F018
:1024000041E003C0EE2089F040E09E012F5F3F4F86
:102410006A2F90E00E949911AC0160E070E018C052
:10242000440F551F661F771F13C0903C89F4282F57
:1024300030E0AFEFB0E00E94FC7824E630E040E00E
:1024400050E00E945D79BA01A90189818062898387
:10245000F801838186FD14C009810062B5E0EB2E8E
:102460009A01AB016F2D8D2D0E94BA66298127FD3F
:102470001BC046E76F2D8091400C0E94C86414C0B9
:1024800029816F2D8D2D0E94CA67F8018381807C80
:10249000803C61F4298127FD0BC041E46F2D8091C0
:1024A000400C0E94C86404C086E703C080E201C0FB
:1024B00081E40F90DF91CF911F910F91FF90EF90EA
:1024C000DF9008958C3038F4E82FF0E0EE0FFF1F16
:1024D000E857F84F22C08431C0F4482F50E0DA01A9
:1024E000AA0FBB1FAE5EBE4F2D913C91803148F4C8
:1024F000FA01EE0FFF1FE053FB4F80819181281BF3
:10250000390BC901880F991F0895843248F4E82FC8
:10251000F0E0EE0FFF1FE05CF84F8081918108959D
:10252000853418F484520C94AC1F80E090E0089538
:102530000E9419778111FCCF1092710C08950F93AE
:102540001F93CF93DF938C01EB010E94786424E00A
:102550004DEF51E060E082E20E94B365B80180E295
:102560000E94D365BE0188E20E94D36567EE71E0E8
:1025700080E30E94D3650E948E680E948A68DF9182
:10258000CF911F910F910C9498120F93462F50E00A
:102590004B5C5D4F00E023E060E10E947D650F91A0
:1025A00008950F931F93CF93DF93082FC9ECD1E0C9
:1025B0001AE0499124E0602F812F0E94C864155FC2
:1025C0001837B9F7DF91CF911F910F9108951F939D
:1025D000CF93DF93EC01162F0E947864BE0188E14F
:1025E0000E94D365111109C049ED51E068E38CE107
:1025F0000E94D96543ED51E002C04BEC51E024E06C
:1026000060E082E20E94B365DF91CF911F910C944C
:102610008E6861E00E94E7120C948A6870E088235B
:1026200099F090E0019725E0289FF001299FF00D97
:102630001124E60FF71FEE0FFF1FE257FB4F8081BB
:1026400091818B509E4F0895FB01EE0FFF1FED5FB0
:10265000FE4F0190F081E02D8081992787FD9095B4
:1026600008951F93CF93DF93D82F162FC4E0DD2357
:1026700099F0612F8D2F0E940E139C01253F81E060
:10268000380764F08BE0820F8D1710F08CE0820F1A
:10269000C15029F0D82FEBCFC0E001C0CD2F8C2F37
:1026A000DF91CF911F910895CF93C62F0E943113D0
:1026B0006C2FCF910C940E130F931F93CF93DF9336
:1026C000EA01062F10E08823B9F00E943113882315
:1026D00099F090E0019725E0289FF001299FF00DE7
:1026E0001124E00FF11FEE0FFF1FE257FB4FC55FF4
:1026F000D140D183C08317C0CE0183589F4F8B3FF9
:10270000910540F01C161D061CF4CDE7D0E002C078
:10271000C3E8DFEFF801EE0FFF1FED5FFE4F019002
:10272000F081E02DC08386E0DF91CF911F910F9162
:102730000C9410609F92AF92BF92CF92DF92EF9273
:10274000FF920F931F93CF93DF938C017B016A015C
:10275000922EB090AB019B2D9F7D943439F08091E7
:102760006607882309F487C0933439F4E801219679
:1027700083E10E940E7285E00BC0953419F092340B
:1027800009F07CC0E801219784E10E940E7284E088
:102790000E946C69811164C0E114F104E1F481E0EC
:1027A000C816D104C1F480E6B81619F08EE2B8124A
:1027B00012C010926607C1E00115110509F0C0E0D2
:1027C000D0E08B2D0E94BD698EE2B81206C081E078
:1027D0008093960702C0A12C02C0AA24A394409122
:1027E000400150914101C41BD50B80919607833065
:1027F00031F48091B401C80FD11D87FDDA95CC1654
:10280000DD0644F48B2D0E94BD6983E10E940E72A7
:10281000E6010AC0CE15DF053CF48B2D0E94BD6990
:1028200084E10E940E72E701C017D107B1F0209732
:1028300061F4A11003C08B2D0E94AD6917FF02C087
:1028400083E101C084E10E940E72892D83700E9491
:10285000106081E08093480113C01092480110C0BD
:10286000CC27DD27C01BD10B85E00E94BD6984E029
:102870000E94BD6991CF953409F484CFE8018CCFD3
:10288000CE01DF91CF911F910F91FF90EF90DF90DC
:10289000CF90BF90AF909F900895552747FD5095DA
:1028A000772767FD7095992787FD90950E949A1369
:1028B000089522E00C944D14462F22E060E00C9421
:1028C0004D1421E00C944D14462F21E060E00C944F
:1028D0004D14E0914901F0E0EE0FFF1FE45BFE4F65
:1028E000808191810895FC01A0914901B0E0AA0F77
:1028F000BB1FA65BBE4FED93FC938FEB099587E161
:102900000C940E72E7E9F7E0108E168A158A178A82
:102910000895E0E1FDE037A1303180F420A541E0E9
:10292000420F40A7DF01A20FB11DA20FB11D8D9371
:102930009C93403108F010A63F5F37A3089590E0C4
:102940008C5F9E4F0C94891490E00C9489148091B4
:102950001205992787FD909509970C948914FC011D
:102960009091050580A191FF74C091A1882311F079
:10297000946001C09B7F91A386A1813059F5C79ACD
:1029800037A121A1332321F181A541E0480F41A7BF
:10299000DF01A80FB11DA80FB11D8D919C9195A3CA
:1029A00084A3403108F011A6315037A397FD02C02F
:1029B00031E101C038E233A32C7F97FD226021A3CF
:1029C00081A18BBBC7988FE182A382E086A3089583
:1029D0002BBB48C081110CC0C79A81A1836081A321
:1029E0008BBB8091410C8D3308F43CC086E02FC036
:1029F000823009F438C081A18BBBC79ABF9800C050
:102A0000000000C086B38078BF9A96A1933049F445
:102A1000882329F083A1815083A3811123C084E0FE
:102A200016C0943021F48823E9F083E00EC095307D
:102A300039F483A1815083A3811114C081E007C0C0
:102A4000963081F4882371F084E183A385E086A326
:102A500009C09091020596FB992790F9891711F00A
:102A6000C79A0895C79808951BBA8FE18ABB00C022
:102A700099B38FEF8ABBECEAF1E08781882311F0EC
:102A800080E202C0892F807E8483292F207C808170
:102A9000281759F08074880F90783181891711F0C8
:102AA000315001C03F5F3183208382819381891738
:102AB00011F08383818308959091FA0490FD02C000
:102AC00093E08927E82FF0E0EE0FFF1FE857F84F5B
:102AD0008081918197FF02C081589F4F880F892F75
:102AE000881F990BE82F181624F0882321F0E19510
:102AF00002C080E801C080E0E8300CF0E7E0F0E0E0
:102B0000E85DFC4FE491EE2319F099E090935401B5
:102B10008E2B0895833021F0811103C083E001C022
:102B200080E0E82FF0E0EE0FFF1FEF5DFA4F8081AD
:102B300091810895FF920F931F93CF93DF93F12C10
:102B4000C0E0D0E08F2D0E948A15092F10E0C00F41
:102B5000D11FF39484E0F812F5CFCE01DF91CF912D
:102B60001F910F91FF9008950E948A152091FC04F7
:102B700020FF03C0919581959109089578941F9243
:102B80000F920FB60F9211248F93809128018F5FBF
:102B9000809328018F910F900FBE0F901F90189572
:102BA00078941F920F920FB60F9211242F938F9348
:102BB0009F93EF93FF93F89487B78F7B87BF7894A9
:102BC000209175018091770190910505882359F036
:102BD00090FF07C08091190E820F8093190E87FF16
:102BE00002C01B9A01C01B9891FF2AC080913F0828
:102BF000811126C0E0E1FDE086A1823009F583A1C4
:102C0000882311F081501BC021A1C79A82A180FDA9
:102C100009C02D7F84A195A196FD2260880F991F80
:102C200095A384A381E082278BBB81A3C79882A14F
:102C3000815082A3811104C083E086A385E083A331
:102C4000F89487B7806487BF7894FF91EF919F9144
:102C50008F912F910F900FBE0F901F901895789421
:102C60001F920F920FB60F9211242F933F934F9301
:102C70005F936F937F938F939F93AF93BF93EF93E4
:102C8000FF9381B7845681BF83E791E00E94BF6FB5
:102C90000E94CC690E94207680917D0C8260809396
:102CA0007D0CEBE0F1E08081815011F0808307C062
:102CB00084E6808381818F5F818381E08283838149
:102CC000815011F0838304C08AE0838381E0848390
:102CD000FF91EF91BF91AF919F918F917F916F91F4
:102CE0005F914F913F912F910F900FBE0F901F90CA
:102CF000189578941F920F920FB60F9211242F936C
:102D00003F934F935F936F937F938F939F93AF9373
:102D1000BF93EF93FF932091800030918100F8944E
:102D200080917D008F7D80937D00789480911A053D
:102D300090911B05A901481B590BCA0196958795CF
:102D400030931B0520931A059C01215A3F402F3DCB
:102D50003E4220F481E0809329012FC0E0912901B7
:102D60002FEF2E0F283048F59C0121523340273792
:102D7000354008F521E02E0F20932901F0E0EE0FF9
:102D8000FF1FE85DFE4FAC014C5D554020910005F2
:102D9000332727FD3095265F3F4F429FC001439F59
:102DA000900D529F900D11246AE070E00E944979C5
:102DB0007183608302C010922901F89480917D0094
:102DC000806280937D007894FF91EF91BF91AF91E5
:102DD0009F918F917F916F915F914F913F912F9133
:102DE0000F900FBE0F901F9018959C0155E03595E0
:102DF00027955A95E1F7280F391FAC01440F452F4D
:102E0000441F550B241B350B892F990F990B859562
:102E1000820F931F08959DE7980F9B3FA0F08E5758
:102E2000282F30E0220F331FF901E058FB4F80813B
:102E3000861714F46083862F48172CF4F901E058A4
:102E4000FB4F4083842F089544E66CE90C940B17E4
:102E50002091FA04217092E0921B21E0981320E067
:102E6000822F08959091DA0194FF08C00E942817DC
:102E700091E0811101C090E0892F089580E00895CC
:102E800049E28402900111243595279535952795BF
:102E900087FD815C86FB880F880B80F9A901481BA0
:102EA000510987FD5395CA0108955F926F927F92F1
:102EB0008F929F92AF92BF92CF92DF92EF92FF924A
:102EC0000F931F93CF93DF93982E742E25E0241732
:102ED00008F4F3C0882309F4EEC036E1831721F02B
:102EE0008AEE981203C0E9C081E0E8C096E1991526
:102EF0000CF4E3C0892D992787FD909597FF03C0B7
:102F00009195819591098A3040F4825F0E946C69A5
:102F100019140CF4D3C091E01BC08A50C82ED12CD8
:102F2000E601CC0FDD1FCC0DDD1DC15EDB4F8A81BC
:102F30008F7009F4C2C0F601E65AFE4F5F01F5E05A
:102F40007F1208C0F501908119140CF4B2C081E021
:102F50008927B4C0688059800E941210811119C05D
:102F60008FEF860D0E9462127C01888185326CF0A1
:102F7000ABED8A2E880E6981882D0E94511F8C012D
:102F8000882D0E943B1F882E19C089810E944017FE
:102F90000BC0823069F48FEF860D0E9462127C01B3
:102FA000898181500E9462128C018824839406C01A
:102FB0008824839400E010E0E12CF12C8A818F704A
:102FC00090E0FC013197EE30F10508F06EC0EA5B4D
:102FD000FF4F0C949E79F7FE33C0F194E194F10811
:102FE0002FC0F7FE32C0F194E194F1082EC001E049
:102FF000070D402F60E0862D0E945517182F402F97
:1030000060E0852D0E945517982F2A812F7025305A
:1030100031F4112309F449C0811145C046C026305E
:1030200019F4111140C029C0912727C091E0E01682
:10303000F106C9F422C091E0E016F106F1F413C0E4
:1030400091E00E151F05CCF00EC091E0E016F106E0
:10305000A4F009C091E0E016F1067CF404C091E010
:103060000E151F0554F490E008C0F601EA59FE4F12
:1030700090819095991F9927991F8820B1F09923E5
:10308000A9F08A81982F907F61F082958F708930A6
:103090000CF08F5F41E0470D60E00E945517982FBC
:1030A00005C091E003C08110ECCF90E0F501908362
:1030B0004BCF892F03C0862F01C080E0DF91CF91D5
:1030C0001F910F91FF90EF90DF90CF90BF90AF9046
:1030D0009F908F907F906F905F90089540E060E0A8
:1030E0008091E7040E945517811114C080913B0123
:1030F00090913C01892B71F41092300D8091410C1C
:1031000090912005981751F08093200580E19DE073
:103110000C94AF1481E08093300DF0CF089520918E
:103120003B0130913C012115310511F0215031094D
:10313000882319F08091FE0401C080E090913A014B
:10314000992329F090910605891708F4892F4AEFF1
:10315000849FC0011124880F991F8217930708F4D8
:10316000C90190933C0180933B010C946E18CF925F
:10317000DF92EF92FF920F931F93CF93DF93F89418
:103180008091420C9091430C789441E020911E056F
:1031900030911F058217930709F440E040933D01E9
:1031A00090931F0580931E0560E081E497E00E94E4
:1031B0006C3D80913D01882309F4BFC28091560186
:1031C00090915701A0915801B0915901AC01BD01F6
:1031D0004F5F5F4F6F4F7F4F4093560150935701A2
:1031E000609358017093590144365105610571058A
:1031F00098F083569109A109B109809356019093E3
:103200005701A0935801B09359018091540188232C
:1032100019F0815080935401E7E9F7E0878980FF36
:103220000DC0808D91E0980F908F943638F08356C2
:10323000808F858996890196968B858B80E00E9488
:1032400022600E9478640E940069182F082F0F7076
:103250000650C091DB01C43021F0C33019F4C4E042
:1032600001C0C8E0083008F09FC0F02EF6948091AD
:10327000160580FF03C083E08F19F82E6F2D809113
:1032800031050E943113E82E6F2D0E9454139C01CA
:10329000C1110DC0AC0197FF04C044275527481B3E
:1032A000590B5595479555954795C1E0C40F8091A9
:1032B000FA0480FBCC24C0F8D12C42E050E04C1939
:1032C0005D098F2D90E04817590761F48091DA016C
:1032D00080FF31C281E0C4E09091FC0490FF03C004
:1032E000C19501C080E0DD27C7FDD09500FF03C078
:1032F000C20FD31F04C0A9014C1B5D0BEA0120972C
:1033000021F09D2F932797FF11C081110FC0232B10
:1033100069F040E050E06F2D8E2D0E945C13812FEC
:103320000E94BD6986E10E940E723DC0CE018458A4
:103330009F4F893F910580F4AE016F2D8E2D0E9425
:103340005C13D7FF03C0D195C195D109D595C79519
:10335000D595C7954C2F21C01C161D061CF44DE7B2
:1033600050E002C043E85FEF6F2D8E2D0E945C138A
:10337000CE0183589F4F8B3F9105A8F4D7FF03C020
:10338000D195C195D109D7FD2396AE0155954795A5
:1033900055954795519541955109445C65E183E701
:1033A00091E00E94907010E0EEE3F1E080919407CC
:1033B0009091950720813181281B390B37FF02C07E
:1033C000215E3F4FB5E035952795BA95E1F7211578
:1033D000310561F024813581281B390B37FF02C08C
:1033E0002F5F3F4F35952795918380839583848305
:1033F0008091FC0485FF02C020E030E0338322830B
:10340000CCEAD1E02D818981821B8F3F09F480E0D5
:1034100087FD8F5F85958887982F990F920F9D83E1
:10342000812B0E948F18E0914901F0E0EE0FFF1F01
:10343000E65BFE4F808191818B539644B9F4888579
:103440008823A1F02E81992787FD9095820F911DE9
:1034500027FD9A958E37910514F08DE705C08338C6
:10346000EFEF9E070CF483E88E83188680910205A7
:1034700087FF3BC0809155018823B9F180915401A9
:103480008823A9F180911D0587FD03C08F5F80937C
:103490001D0582E00E945C15982F9F7789F020918E
:1034A0001D05921720F510921D05111120C0182F2F
:1034B0001095111F1127111F83E6811B182F17C0AC
:1034C00083E00E945C15982F9F7789F020911D055D
:1034D000921768F410921D05111109C0182F10954C
:1034E000111F1127111F1C5902C01092540181E0B5
:1034F0008093550151E8E52E54E0F52EC0E8D4E064
:103500006AE0C62ED12CF7018081882309F462C0BD
:10351000853068F40E947F6AE82FF0E0EE0FFF1F0D
:10352000EF5FFE4F0190F081E02D808104C0853077
:1035300021F48091B20188834DC08A30B8F485505F
:103540000E947F6AE82FF0E0EE0FFF1FEA57F84F66
:103550008081918197FD079623E0959587952A951F
:10356000E1F78338FFEF9F07DCF015C08D30D0F412
:10357000E82FF0E0EE0FFF1FE458F84F80819181B3
:1035800097FD079603E0959587950A95E1F78338AF
:103590002FEF92072CF08D3791056CF28DE7CBCF92
:1035A00083E8C9CF8D31B0F4E82FF0E0EE0FFF1FB4
:1035B000E25BF84F80819181B6010E9449796338BE
:1035C0004FEF74072CF06D3771051CF06DE701C0EB
:1035D00063E8688352E0E50EF11C22968FE8E81656
:1035E00084E0F80609F08FCF8091C7019091C8015F
:1035F000009761F060E00E94E7120E94197788232B
:1036000099F01092C8011092C7010EC01093AB013F
:10361000E0914901F0E0EE0FFF1FE65BFE4F0190E5
:10362000F081E02D812F09950E948E68C091650080
:1036300083E791E00E94AB6F882311F084E105C01D
:1036400080911B0E882321F0815080931B0E06C0B1
:10365000809163008695817080931A0E80911A0E76
:103660008093C501882309F464C08091020585FD1B
:1036700060C0CF7EC09365008091410C8F71823015
:1036800009F054C080912F0590913005AC01F4E011
:10369000440F551FFA95E1F797FD0796BC01E3E04B
:1036A00075956795EA95E1F72091E604332727FDA4
:1036B00030952A5F3F4F629FC001639F900D729FBC
:1036C000900D1124840F951F2091FC0426FD05C048
:1036D000609100017091010102C060EF70E00E94F2
:1036E000357980910201680F711D6F5F7F4F75956D
:1036F00067956093020180911C05805F80931C0593
:10370000811114C08091E504681780F4623370F071
:103710006EE281E10E9414728091FC0483FF06C076
:1037200082E390E090933C0180933B0110923A0138
:1037300004C0C0619FCF80E0CFCDDF91CF911F91BA
:103740000F91FF90EF90DF90CF900895CF93DF938C
:10375000C62F2091C601222329F09093C80180939F
:10376000C70133C060E00E94E712C11103C080911D
:10377000E40401C089E10E947B6867E182E10E9464
:1037800014720E949812D1E00E94197781111DC015
:1037900080917D0C833019F4A89510927D0C40E047
:1037A00060E08091E7040E945517811106C0809166
:1037B000FE04811102C0CC2329F0D093300D0E9469
:1037C0006E18E2CF1092300DFACFDF91CF910895AD
:1037D00090914901911103C0811106C017C0811158
:1037E00003C08FEF890F01C080E08093490187E11A
:1037F0000E940E72E0914901F0E0EE0FFF1FE65BC0
:10380000FE4F0190F081E02D8EEB099460E08EEB8D
:1038100091E00C94A61BCF93DF93EC0180914901BA
:10382000843038F060E081EB91E0DF91CF910C942F
:10383000A61B87E10E940E72A0914901AF5FA09381
:103840004901B0E0AA0FBB1FA65BBE4FCD93DC932E
:103850008FEBFE01DF91CF9109941F93CF93DF93FC
:10386000C6E9D4E090E0888111E0190F882341F087
:1038700040E060E00E945517882311F0812F05C0B9
:10388000912F2A96143079F780E0DF91CF911F9124
:103890000895CF92DF92FF920F931F93CF93DF9300
:1038A00080912801C2B7909128018913F9CFD0E007
:1038B000D82BF0E1FF2E80914504F81A0E94FA0FF0
:1038C0001EE517B90E9434150E94B71817B9369A29
:1038D0003699FECF84B195B1049640910001509184
:1038E000010167E0649F9001659F300D1124820FF4
:1038F000931FE3E096958795EA95E1F79093010190
:103900008093000180917D0C833019F4A89510926A
:103910007D0C2091280182B7909128012913F9CFBD
:1039200090E0922B8C1B9D0B209192063091930678
:103930002817390720F4909393068093920680917C
:103940000C01823078F480910F01882309F497C12B
:103950008091170590911805019690931805809312
:1039600017052FC110920C018091EA0D882309F4EC
:1039700056C04091D501842F807C09F1803819F41C
:10398000C0E9D1E002C0CAE7D0E08091680D909113
:10399000690D2091900630919106820F931F6AE085
:1039A00070E00E944979CB0143FD03C045FD0E94B0
:1039B000191FC817D9071CF481E00E940E7200E09D
:1039C0001CED90E0C0E0D0E08091410D0817B0F40C
:1039D000E02FF0E0EE5BF24F8081C80FD11D811720
:1039E00008F4182F911107C020914304821720F486
:1039F0008DE10E940E7291E00F5FE6CFCE0165E08F
:103A000070E00E9435797093AB0D6093AA0D1C3D58
:103A100031F0812F90E09093A70D8093A60D8091B7
:103A2000EB0D81110BC0809119058F5E982F977F48
:103A3000903608F048C09093190548C006E614E097
:103A40007CE7C72E7DE0D72EC0E0D0E0F801808172
:103A5000882371F1FE01EE0FFF1FEE0FFF1FE759E4
:103A6000FB4F80818295869586958370833001F522
:103A700020916F042223E1F0F6018081918156E0CC
:103A8000959587955A95E1F730E08217930784F072
:103A90008091050581FF05C081E390E00E948914B3
:103AA00007C046E46091700483E791E00E94907043
:103AB00021960C5F1F4FF2E0CF0ED11CC230D10512
:103AC00009F4B1CFC3CF877080931905C9ECD1E059
:103AD000D12CDF1409F437CF8E0103581D4FF801A4
:103AE0008081982F907C9034C9F4880F880F40E033
:103AF00060E0859585950E945517882379F080911F
:103B0000050580FF05C0FE01E258FD4F608101C040
:103B100061E046E483E791E00E949070F8018081C3
:103B2000982F907C9038D1F5880F880F85958595D2
:103B3000873114F1992787FD90954797813091053A
:103B400049F08230910561F0892B41F5809119058A
:103B5000837003C080911905807F81111FC005C04B
:103B60008091190587708230C9F4FE01E258FD4F3B
:103B700080810E94042012C09091190590FD0EC012
:103B800040E060E00E945517882341F0FE01E258B2
:103B9000FD4F8081805890E00E948914D394229632
:103BA00098CF0F2D10E0E801CC0FDD1FCA5BDB4F73
:103BB0008881D82ED294D69447E0D4228F7129F4EC
:103BC000F394FFE0FF1568F758C040E060E00E9402
:103BD0005517C82E80910F010B541E4F823009F4E7
:103BE00049C08D2D857051F4F8018081811106C086
:103BF000CC2021F0898190E00E9489148FEF8D0DF7
:103C0000823060F4F80180818130A1F5C11032C0AA
:103C10008981F2E0DF122BC08F5F29C085E08D150E
:103C200050F4F8018081811125C0CC2019F18981DF
:103C30000E9404201FC0F2E0FD15E0F4CC20D1F07A
:103C400084E0D81631F095E0D91631F066E970E0DD
:103C500005C06CE271E002C068E572E08091170572
:103C6000909118050E943579892B21F4898190E083
:103C70000E948914F801C082A3CF10920F01809195
:103C80000D018823D1F110920D010FE114E0C6E679
:103C9000D1E0DD24DA94F801F2808F2D8F700E943C
:103CA0001210833019F59881911104C0F8018081B8
:103CB000809508C097FF08C09F5F9883911106C048
:103CC000F8018181888302C0915098838F2D807F75
:103CD00069F08F2D82958F7089300CF08F5F40E0F6
:103CE00060E00E945517811101C0D8820D5F1F4FFF
:103CF0002196F1E0C237DF0771F6DF91CF911F9176
:103D00000F91FF90DF90CF9008951F93CF93DF9393
:103D1000182FD62FC42F80919607811101C0C2E0C1
:103D20004D2F50E02C2F60E08FE70E94CA67DA30F9
:103D300010F0DFE601C0D5E72C2F4FE260E08D2FB9
:103D40000E94C864412F50E04F5F5F4F2C2F60E00E
:103D50008FEF8D0FDF91CF911F910C94CA671F9346
:103D6000CF93DF93D82F162FC42FB9010E94D365AC
:103D7000112329F06FE08C2F0E945C14C82F4C2F68
:103D800050E0212F6D2F80E60E94CA678C2FDF91B3
:103D9000CF911F910895813649F40E94BD6981E059
:103DA0000E94E81B83E39EE40E940B1C69E17EE015
:103DB00080E10E94D36563E07EE080E20C94D365ED
:103DC000FF920F931F93CF93DF93182FF62E0AE0E5
:103DD0008AE0189FE0011124CD51DE4F2FE130E041
:103DE000211B3109029FA001039F500D1124BE0128
:103DF000CE010A960E94B379FF2049F0BE016A50B5
:103E000071094AE050E0CE010E94B3790AC0FE0178
:103E100011920A95E9F78091DB078883898384E60C
:103E20008A831093DD07DF91CF911F910F91FF904F
:103E300008959C01220F331F280F391F95958795F0
:103E400095958795280F391F959587959595879511
:103E500095958795820F931F0895429643E7489F53
:103E60009001499F300D1124C901E6E09595879591
:103E7000EA95E1F70895E82FF0E0ED5FFD4EE4915B
:103E8000EE2369F0E13021F48091EB0D811107C040
:103E900081E09091EA0D911103C080E0089581E0E6
:103EA0000895E82FFF27E7FDF095EE50FD4EE491D1
:103EB000772767FD7095CB0183589F4FEC307CF4DA
:103EC000EA30DCF5EF3F09F02CF4EE3F64F5E53F16
:103ED000E9F10895E43089F0E63079F00895E332AD
:103EE00091F134F4EC3009F1EE50E23050F10895E4
:103EF000E43239F1E7323CF10895803491059CF0C9
:103F0000880F991F80549109813C910564F0880FB6
:103F1000991F805C9109813C51E0950724F0880F3E
:103F2000991F885E91402AE001C024E6AC01249FDD
:103F3000C001259F900D11240895CB01815A9F4FF8
:103F4000089522E3F3CF880F991F0895F3E0880FB7
:103F5000991FFA95E1F70895E82FFF27E7FDF095FF
:103F6000EE50FD4EE491E53FA9F44091AC0D509127
:103F7000AD0D2091A00D3091A10D429FC001439F36
:103F8000900D529F900D112464E670E00E944979D3
:103F9000CB010895ED3F4CF4EE0FFF0BEC56FB4FB9
:103FA0008081992787FD90950895EF3F09F044F4AB
:103FB000EE3F8CF4ED3F09F58091020190E0089509
:103FC000E43081F0E332C9F48091A60D9091A70D01
:103FD000880F991F0895EE0FFF0BE556F84F838960
:103FE000948908958091680D9091690D20919006B3
:103FF00030919106820F931F0895EE0FFF0BE05A48
:10400000F24F808191810895CF92DF92EF92FF92DB
:104010000F931F93CF93DF931F92CDB7DEB7082F77
:1040200019820E94AC1F7C01802F0E943B1F8111CE
:1040300005C08AE30E94A41411E001C010E0E02F43
:10404000FF27E7FDF095EE50FD4E64916230E4F4F9
:1040500067FF3BC06D3F34F4663F5CF5653F09F494
:104060007BC030C06D3F09F47AC06CE370E0C701DB
:104070000E9449796B017C0146E260E0C6010E9422
:104080001D7260E045E377C0603209F46AC044F411
:104090006430D1F1BCF06A50623008F454C012C0F0
:1040A000633209F461C074F06552623008F457C09D
:1040B00009C0E62FEE0FFF0BEC56FB4FE080FF240C
:1040C000E7FCF09460E040E056C084E06802F00154
:1040D0001124EA59FB4F038102950695069503705A
:1040E000D08041E0023009F040E09E012F5F3F4F59
:1040F000C7010E9499117C01033099F1013011F33D
:1041000083E68D1588F52BC09091D501892F80729B
:1041100093FF03C0882349F006C0882331F0C7010C
:104120000E94191F7C0148E101C048E388EEE816AF
:1041300083E0F806E4F0C7016AE070E00E94497984
:104140007B0160E018C08091D50185FF12C0C701D6
:104150000E942D1F7C010DC060E04BE30CC061E0AC
:1041600004C061E043E307C062E044E204C061E0F0
:1041700002C060E04FE2111103C0C7010E941D722E
:104180000F90DF91CF911F910F91FF90EF90DF90F3
:10419000CF9008959F92AF92BF92CF92DF92EF920D
:1041A000FF920F931F93CF93DF93C82EB62EF42E5A
:1041B000E901102FAE2C8E2D8170982EE0FE15C0D7
:1041C00000E021E0240F43E153E18C2D0E949F6524
:1041D00012FD04C068E1D62EDC0C08C05CE1D52ECF
:1041E000DC0C88EFB80E0CE002C0DC2C06E08A2D57
:1041F0008870E82EA3FC1F7BEF2DFF27E7FDF095CD
:10420000EE50FD4EF49084E0F81609F468C08F1566
:104210009CF08FEF8F1564F08EEFF81664F585EF44
:10422000F81609F49AC08DEFF81609F478C07AC030
:1042300081E08F15B4F576C080E2F81609F46AC003
:104240008F1564F086E0F81609F449C0F8160CF4EE
:1042500069C0E6EFEF0DE230B8F164C083E2F81612
:1042600009F45BC0F8160CF45DC0EBEDEF0DE23025
:1042700008F455C057C012FD02C08CEFD80E99202B
:1042800011F08AE0D80E1770012F212FAE016B2D8F
:104290008AEF8D0D0E942E1003E30F0D8AEFC80EDA
:1042A0004BC0912F90684C2FEE2019F08DE38C0DB0
:1042B00002C08D2D801BEE24E394092F2F2D6B2D32
:1042C0000E94E111082F38C08091D50185FF47C0B9
:1042D000CE010E942D1FEC01D01A06E424C080916B
:1042E000D50185FF07C083FD07C0CE010E94191FBD
:1042F000EC0102C00DE601C006E6C83E83E0D80727
:1043000014F4106210C0CE016AE070E00E94497996
:10431000EB0109C0106201E406C0106301C0106225
:1043200006E701C000E2EE20E1F08DE38C0D212FC5
:10433000AE016B2D0E94CA678A2D8670A1F0A2FE85
:1043400004C08AE08C0D1B7F02C08091400C212F9D
:10435000402F6B2D0E94C86406C007E7E4CF03E43A
:10436000E2CF8D2DE4CF802FDF91CF911F910F9160
:10437000FF90EF90DF90CF90BF90AF909F90089507
:10438000DF92EF92FF920F931F93CF93DF93D82F7B
:10439000162FC42FD22E8E2D8370F82EA1F080916F
:1043A000AB01803881F48DE7840F8B3F40F0E42F20
:1043B000F0E0EE0FFF1FEC57FC4FC08101C0CEE7CD
:1043C00082E00E9410608DE78C0F2E2D8B3FE0F075
:1043D00040E851E1612F8EEE8D0F0E94B3652E2DC6
:1043E00043EB4C0F612F8AEF8D0F0E94C864FF20B2
:1043F00009F122E042E850E06EE770E08C2F90E097
:104400000E949A13C82F16C04C2F552747FD509570
:10441000612F8D2F0E94CA67FF2061F0402F6D2D04
:104420008C2FDF91CF911F910F91FF90EF90DF9034
:104430000C9459148C2FDF91CF911F910F91FF9005
:10444000EF90DF900895CF93DF939EE0899FE00186
:104450001124C753DE4FFE01EA54FE4F40E060E0F6
:1044600080810E945517882359F0C954DE4F40E0DF
:1044700060E088810E945517811104C081E003C06B
:1044800080E001C082E0DF91CF910895EF92FF922A
:104490000F931F93CF93DF93F82EE62EC42FD42FC4
:1044A000D695062F0D1B182F1D1B602F812F0E94E4
:1044B0006E666D2F6E0D4C2F812F0E946B664C2FF8
:1044C000602F8D2F8F0D0E946E664C2F602F812FD5
:1044D000DF91CF911F910F91FF90EF900C946B663D
:1044E00021E0AC0160E080E00C94B3651F93CF93B2
:1044F000DF93182FC0E1D1E083EA98E00E94702298
:104500001136B1F068F41036D1F48FEF8883198238
:10451000109293061092920687E10E940E720FC0CD
:10452000123619F0133621F00AC08BEE92E202C067
:104530008BE396E4DF91CF911F910C94731464E99F
:1045400078E088E00E94D3654981469550E068E0B4
:1045500084E50E94D96765E878E080E10E94D36530
:104560004881469550E060E184E50E94D96766E79E
:1045700078E088E10E94D365498150E08881481B3A
:10458000510957FF02C04F5F5F4F5595479568E14E
:1045900084E50E94D9676DE678E080E20E94D365E9
:1045A000809192069091930629E1289FA001299F6E
:1045B000500D1124569547955695479520E360E296
:1045C00084E50E94CA676AE578E088E3DF91CF91CD
:1045D0001F910C94D3650F931F93CF93DF93182FE4
:1045E000C7E9D7E085E598E00E947022113678F09F
:1045F000133628F0133659F486E792E202C08BE3B3
:1046000096E4DF91CF911F910F910C9473146CE499
:1046100078E088E00E94D3654A815B8100E020E079
:1046200068E08AE20E942E104C815D8120E068E003
:104630008EE40E942E1063E478E080E10E94D3654E
:104640004E815F8120E060E18AE20E942E10488561
:104650005985A4E056954795AA95E1F720E060E1D9
:104660008EE40E942E106EE378E080E00E94D36515
:104670004881598120E060E08EE40E942E104EE7D0
:104680006CE382E00E946B6643E26CE185E00E948D
:104690006E66CBE043E06BE38C2F0E946E66CA5FD0
:1046A000C338C1F71091950680919406893710F4AC
:1046B000C0E001C0C12FD6E00CE3EC2FF0E0EA56D9
:1046C000F94F4081602F641B8D2F0E946E66CF5F73
:1046D000C83708F0C0E0C11719F0DF5FDE3769F7AF
:1046E000DF91CF911F910F91089591E0211101C0A9
:1046F00090E0442319F041E553E002C045E553E062
:10470000292F0C94B3650F9301E0211101C000E043
:10471000242F48E751E10E949F650F9108956F9201
:104720007F928F929F92AF92CF92DF92EF92FF9201
:104730000F931F93CF93DF93EC01162F842F490122
:10474000602FD09040076090900770909107A091E3
:104750009207B0919307EEE3F1E0268137812619A5
:10476000370937FF02C0215C3F4F46E0359527955A
:104770004A95E1F7422F20936307208531852A1B54
:104780003B0B37FF02C0215C3F4F96E035952795E4
:104790009A95E1F7922F20936107442311F07782D5
:1047A0006682992311F0B187A087909162079111D9
:1047B00004C09091FC0495FF06C01092630710920C
:1047C00061071092620790916307911108C02091D0
:1047D0006107211104C022813381232B61F02091D4
:1047E000FE044AEF249F90011124220F331F3093BF
:1047F0003C0120933B0181149104B1F028812111E7
:1048000077C120919607222309F47BC1213009F456
:104810008AC191118FC1153609F4AFC1143609F45C
:10482000B6C141E00E94851EE114F10451F0988167
:104830008C2D9C1508F4892FF701E80FF11DE491E8
:1048400001C0E0E080919607813081F58091B4014C
:1048500018166CF4DE1610F4D39411F588818A15BD
:1048600018F48F5F888301C01882D12C19C0882367
:10487000B9F0D11014C08881882319F08150888341
:1048800001C0A882E114F10459F098818C2D9C1587
:1048900008F4892FF701E80FF11DD49001C0DA94D4
:1048A0001092B4011E3249F483E005C0833029F42C
:1048B0001E3219F481E080939607E114F10451F05F
:1048C00098818C2D9C1508F4892FF701E80FF11DB4
:1048D000549101C050E080916607811145C08091DC
:1048E0006107882301F14881481B47FD40E08A2D7C
:1048F00090E0242F332727FD3095281739070CF037
:104900004A2D4883E114F10459F0C41608F44C2DE3
:10491000F701E40FF11DE491ED1518F4DE2E01C04E
:10492000D12C1092610728812223F1F08091630736
:104930008823D1F0D81AD7FCD12C8D2D992787FD4B
:104940009095E114F10479F03C2D2C1508F4322FE8
:10495000F701E30FF11DE4912E2F30E0821793074A
:104960001CF0DE2E01C0D12C103669F190F4123407
:1049700009F473C028F41132A9F11E3221F197C055
:10498000143409F446C008F476C0153409F451C053
:104990008EC0153609F451C040F4133609F46EC0C8
:1049A000D8F5123609F45CC082C01E38C1F01F3B36
:1049B00031F0113809F07BC01092660721C01882CF
:1049C0001092660738C08881882309F470C081E09E
:1049D00090916607911180E08093660768C08EE829
:1049E0000E94BD6980916607882319F010926607BE
:1049F0005EC08881882311F0892831F410929607CF
:104A000080E00E94E81B53C087E10E940E7218826A
:104A10004EC0D51609F44BC0EF2809F448C0809168
:104A20006607811144C0D51610F4D39411C0D12C5F
:104A30000FC0D11002C0D12C3AC0EF28C1F1809133
:104A40006607811134C0DD2011F0DA9401C0D52E43
:104A5000552369F11092AB012AC088818A1539F17A
:104A600080916607811123C088818A1510F48F5FB9
:104A70000DC018820EC088818823C9F08091660716
:104A8000811115C08881882319F08150888301C065
:104A9000A882E114F10479F288818C1508F4C82EFB
:104AA000F701EC0DF11DE490ED1408F4DE2C80917B
:104AB000660781110AC021E0809140019091410177
:104AC000892B09F420E0822F01C081E080936507E3
:104AD000D0924007DF91CF911F910F91FF90EF90FF
:104AE000DF90CF90AF909F908F907F906F900895C0
:104AF00090916607911103C091E09093960740E072
:104B000091CE2091B401121624F0222319F015E65B
:104B100001C014E61092B4011E3209F07ACE21E0F1
:104B20002093960705C01E3209F073CE10929607A7
:104B300010E06FCE2091660721116DCEE82FE91BA2
:104B4000E7FDE0E0462F50E02E2F332727FD30957C
:104B50002417350714F0EFEFE60FFF27E7FDF09578
:104B6000282F30E0E217F30729F0EE0FFF1FE80DC2
:104B7000F91D1DC0109263074ECE811101C0862F12
:104B8000F401E80FF11DE80FF11D329710C0282F36
:104B900030E070E0615071092617370714F48F5F19
:104BA00001C080E0880E911C880E911CF401859153
:104BB0009491DF91CF911F910F91FF90EF90DF9033
:104BC000CF90AF909F908F907F906F900C947314C4
:104BD000AF92CF92EF92FF920F93AE2CC12CE12CAB
:104BE000F12C0E948F230F91FF90EF90CF90AF9008
:104BF0000895EF920F93E42E00E020E030E040E0D3
:104C00000E94E8250F91EF900895BF92CF92DF9216
:104C1000EF92FF920F931F93CF93DF93C82F87E1FB
:104C20009BE00E947022EE24E39406E024E931E147
:104C300044E06C2F8FEB97E00E94E825B090BF070F
:104C400010925501C8E8D7E010E000E0C12C54E014
:104C5000D52EE12CF12C41E4612F88E10E947A6588
:104C600041E3400F612F8EE10E947A65802F0E9400
:104C70008A15AC01612F8AE20E94DC65073081F061
:104C8000A881B98124E630E00E940B79A701960142
:104C90000E947F79A901612F8AE50E94D9670AC025
:104CA00081E0B81611F040E201C041E2612F8AE5CF
:104CB0000E949E100F5F185F2296083061F622E076
:104CC00044E15BE068E28CE60E94AD654091000142
:104CD0005091010160E388E70E94D96781E0B81232
:104CE0000AC0B09262074FE761E88091E6040E9433
:104CF00061148093E604DF91CF911F910F91FF9093
:104D0000EF90DF90CF90BF900895EF920F931F9395
:104D1000CF93DF93C82F8FE09BE00E947022E12C9D
:104D200006E024E931E143E06C2F8EEB97E00E942E
:104D3000E825D0E0C0E0C43018F018EF1D0F01C026
:104D40001D2F8FE08C0F0E946C69082FCF5F20E031
:104D50004C2F612F8AE20E94FA1040E3400F202F6F
:104D6000612F84E40E94C864D85FC93021F7D8E37A
:104D7000C0E08C2F0E946C69182F00E02C2F4FEEA2
:104D80005AE06D2F80E00E949F6540E3410F212F84
:104D90006D2F80E20E94C864CF5FD850C63049F7BB
:104DA00047EE5AE068E184E50E94D96516E0C0E26A
:104DB000D0E02D2F48EB51E16C2F84E50E948364F5
:104DC000812F0E946C6940E3480F282F6C2F8CE6DE
:104DD0000E94C86481E0810F0E946C6940E3480F23
:104DE000282F6C2F88E70E94C864DF5FC85F1E5FB2
:104DF000D430F9F6DF91CF911F910F91EF90089584
:104E0000EF920F93CF93C82F8FED9AE00E947022FC
:104E1000E12C06E024E931E142E06C2F8DEB97E0D4
:104E20000E94E8256FE877E080E10E94D3656FEB90
:104E300077E088E10E94D3656EEA77E080E20E9425
:104E4000D3656FE977E088E20E94D3656BE777E08E
:104E500080E3CF910F91EF900C94D3652F923F9206
:104E60004F925F926F927F928F929F92AF92BF927A
:104E7000CF92DF92EF92FF920F931F93CF93DF9326
:104E800000D000D000D0CDB7DEB7D82E84E391E1BA
:104E90000E947022B7E0AB2E16E0C12E0DE2E02E8C
:104EA00001E1F02E0CE020EA31E149E06D2D83EDC7
:104EB00097E00E948F236090D307109140078EEDFA
:104EC0008D0D843028F48091660781110E94E87668
:104ED00080916607882319F022E0298302C031E01F
:104EE000398364E271E188E00E94D3658091D50145
:104EF00083FB882780F991E069120DC011110BC066
:104F000061E00E945C149091D50180FB93F990932D
:104F1000D50101E001C000E0282F48E151E168E03F
:104F20008CE30E949F658091D50185FB882780F9DD
:104F3000E1E06E120DC0113059F461E00E945C1482
:104F40009091D50180FB95F99093D50101E001C0C6
:104F500000E0282F40E151E168E080E60E949F6573
:104F600026E634E03E832D83EEEC8E2EEDE09E2E81
:104F700031E33A83F2E07F2EA0E1FA2E8981806846
:104F80008C8365E071E18F2D0E94D3659A819153E6
:104F90009B834A816F2D86E00E947A65671004C06A
:104FA000111102C00C8101C000E8E12C2B81ED81C0
:104FB000FE8140816F2D80E60E94E111EE24E39492
:104FC00000E82B81F40140816F2D8EE70E94E111F2
:104FD000671002C0113011F000E001C00981ED81BD
:104FE000FE81238122952695269523704FEF50E16F
:104FF0006F2D80E60E949F65671031C08091660723
:10500000811106C08091400190914101892B39F1B5
:105010001123B9F0113019F5ED81FE81838163E030
:1050200082958695869583700E945C148295880F80
:10503000880F807CED81FE8193819F73982B9383F1
:105040000EC0ED81FE81808122E04FEF50E060E0F4
:1050500070E090E00E949A13ED81FE8180834424E9
:105060004394470C78E0572E5F0CAD80BE80C12C76
:10507000D12CED81FE818381982F9F70492F50E0C4
:105080009601220F331F02C0559547952A95E2F7E6
:10509000F42FF3702F2E8295837090E00C2C02C0B9
:1050A000959587950A94E2F7282F2170322E641483
:1050B00011F0E12C01C0E98020E04AEF50E1652DBC
:1050C00084E00E94B365112311F000E001C00E2DB1
:1050D000222D40E952E1652D84E20E949F65113046
:1050E00011F000E001C00E2D232D46EF50E1652D9B
:1050F00082E40E949F65123019F40E2D006801C0F1
:1051000000E83FEFA31AB30AEE24E3942B81ED816C
:10511000FE81EC0DFD1D4181652D80E60E94E111AF
:10512000641060C080916607811107C080914001C2
:1051300090914101892B09F455C0113079F180F02B
:10514000123009F04FC0F501808122E04FEF50E0AE
:1051500060E070E090E00E949A13F501808342C005
:1051600022E043E060E0822D0E944D14ED81FE813B
:105170002381C114D10439F0F4E08F9FC0011124C0
:10518000922F937002C0922F9C70982B9F70ED818C
:10519000FE818381807F892B838324C022E041E0CC
:1051A00060E0832D0E944D14ED81FE8123812295C4
:1051B0002370C114D10429F0982F990F2D7F922BC1
:1051C00003C0922F9E7F982B93709295907FED81D4
:1051D000FE8183818F7C892B83838091480181119B
:1051E0000E94E8764394F8E05F0E2FEFC21AD20ACD
:1051F00032E0C316D10409F03CCF83E0780E98E189
:10520000F90EEA81EF5FEA832D813E812C5F3F4FEB
:105210003E832D8337E0830E911C7F12B2CE2696FB
:105220000FB6F894DEBF0FBECDBFDF91CF911F91B7
:105230000F91FF90EF90DF90CF90BF90AF909F9035
:105240008F907F906F905F904F903F902F90089538
:105250004F925F926F927F928F929F92AF92BF9286
:10526000CF92DF92EF92FF920F931F93CF93DF9332
:10527000C82F80E890E10E94702297E0A92ECC24EC
:10528000C3942EE7E22E20E1F22E0CE020EA31E179
:105290004BE06C2F81ED97E00E948F236090D10747
:1052A0008090400731E8E32E34E0F32EC0E8D4E0EC
:1052B000AA24A394B12C18E0712C992487FC909413
:1052C000C12CD12C80E3482E4A0C0C2D6BE770E1E9
:1052D000812F0E94D365442D612F8CE00E947A6556
:1052E0006A147B0449F48C149D0431F480916607A0
:1052F000811105C021E001C020E0512C03C022E053
:1053000055245394013099F0022FF701208142E295
:1053100050E1612F88E40E949F655520C1F06CE147
:10532000F70180810E945C14F701808310C04881DE
:10533000552747FD5095612F8CE60E94CA6755207E
:1053400031F04DE763E888810E9459148883FFEFAC
:10535000CF1ADF0A82E0C816D10409F0B6CFE2E026
:10536000EE0EF11C2296185FFFEFAF1ABF0A103441
:1053700009F0A6CFDF91CF911F910F91FF90EF9091
:10538000DF90CF90BF90AF909F908F907F906F9065
:105390005F904F9008957F928F929F92AF92BF92AD
:1053A000CF92DF92EF92FF920F931F93CF93DF93F1
:1053B000D82E87ED9AE00E947022B6E0AB2EC5E0B1
:1053C000CC2ED1EDED2EDAE0FD2E06E024E931E120
:1053D00041E06D2D8CEB97E00E948F23C090BC07BD
:1053E000809040078091630081FF04C06AEC7AE0FE
:1053F00088E1FCC0CA9480916607882319F0A3E075
:105400009A2E02C099249394C0EFD4E0B12C10E1FD
:10541000AA24A394AB0C20E04A2D612F80E00E94C7
:10542000A310F12CCB1002C08F1411F000E001C0CA
:10543000092D802F8270782E92E0F91609F444C06D
:10544000E3E0FE1609F455C0F1E0E980FF16D1F063
:10545000E294E694E694F3E0EF222E2D4FEB5AE02F
:10546000612F88E10E949F65772009F45AC062E0AD
:105470008E2D0E9464148295880F880F807C9981FC
:105480009F731FC0EE0CEE0CE594E5948E2D9DE00D
:105490008902F0011124F7FD3396AF015595479528
:1054A00055954795202F612F82E40E94CA67772087
:1054B000C1F14FE161EE8E2D0E9461148F739981CD
:1054C000907C982B99832DC0E880EE2DE770EE2E0E
:1054D0002E2F41EB5AE0612F88E40E949F657720D0
:1054E00001F163E08E2D0E94641487709881987F8B
:1054F00016C0E880E594E594E594202F4E2D612FA9
:105500008AE50E94FA10772061F046E16AEE8E2D5E
:105510000E946114880F880F880F98819770982BCC
:105520009883F394F4E0FF127DCF185F2296AF16B4
:1055300011F0BA2C6DCF66EA7AE080E30E94D36561
:1055400084E0C8120AC048E266EF809100050E941C
:1055500061148093000521E201C020E24091000522
:10556000552747FD5095465F5F4F60E38EE40E94EC
:10557000CA67EE24E39495E0C912E12C2E2D42EA8D
:105580005AE068E380E00E94B3650AE211E0C8EEE9
:10559000D4E070E3F72EF801419151918F016991A8
:1055A0007991461B570B440F551F20E268E38F2D5E
:1055B0000E94CA67F8E1FF0E80E9F812ECCFEE20F6
:1055C00091F090E6D9120FC088E0EAE2F1E0A8EE8F
:1055D000B4E001900D928A95E1F781E00E9410609D
:1055E00087E10E940E7262E97AE088E0DF91CF9154
:1055F0001F910F91FF90EF90DF90CF90BF90AF90F1
:105600009F908F907F900C94D365FF920F931F9380
:10561000CF93DF93F82EEB018A0147E16CE20E9401
:10562000462243E06BE28F2D0E946E6643E06CE2FF
:105630008FEF8F0D0E946B66C8016FE87FEF0E94AD
:1056400049792CE2260FCE0161E770E00E9449798A
:10565000862F45E0622F8F0DDF91CF911F910F9123
:10566000FF900C944622CF92DF92EF92FF920F931D
:105670001F93CF93DF93C8E8D7E04A815B816881AD
:1056800079818AE20E94052B4C815D816E817F8148
:1056900086E50E94052B28961AE3F12E0DE510E011
:1056A00087E3C82E899199919C5FB8010E9449793E
:1056B000DD24D394D60EEC2CE61A4D2D6E2D8F2DB5
:1056C0000E946E664D2D6E2D81E08F0D0E946E66DC
:1056D0004D2D6E2D82E08F0D0E946E6685E0F80ED6
:1056E00089E4F812DFCFDF91CF911F910F91FF90E6
:1056F000EF90DF90CF900895DF92EF92FF920F939B
:105700001F93CF93DF93F82E8CE49BE00E947022CE
:10571000EE24E39406E024E931E145E06F2D80ECCE
:1057200097E00E94E8251092C007C1E2D7E010E0A0
:10573000812F0E948A1548815981841795070CF49E
:10574000AC01499359932C853D85281739070CF4F2
:105750009C013D872C87143060F0FE017097240F68
:10576000351F37FF02C02F5F3F4F35952795318397
:1057700020831F5F1730E1F680913D078093620719
:1057800090E2F91621F08FEBF8120EC00BC08F5F7C
:1057900080933D07833041F487E10E940E7281E0DF
:1057A0000E94106010923D0780913D078130E1F02A
:1057B000A8F0823009F07BC0109255016BE17BE0CC
:1057C00080E10E94D36543E851E168E182E10E94F3
:1057D000D965C7EBD4E0E1E2F7E028C06BE37BE0FA
:1057E00088E10E94D36563C06DE27BE080E10E94A6
:1057F000D36543E851E168E182E10E94D965C3E1E4
:10580000D7E0D12CB8E9EB2EBAE3FB2E08E615EC75
:10581000FF86EE861D8F0C8F8D2D0E948A15899331
:105820009993D39497E0D912F3CF41C061917191CC
:10583000848595859B01281B390B37FF03C0319563
:1058400021953109233331053CF1DF0150974D910A
:105850005C91598348839A01261B370BB90137FFA6
:1058600002C0615C7F4FA6E075956795AA95E1F748
:10587000261B370B3F872E87841B950B9C0197FFB8
:1058800002C0215C3F4F46E0359527954A95E1F7E8
:10589000821B930B9D8F8C8F229687E0EF32F80747
:1058A00029F60E94725E9093E2048093E104DF91F6
:1058B000CF911F910F91FF90EF90DF900C94332BBD
:1058C000FF920F931F93CF93DF93182F062FEA01B8
:1058D000F22E222321F061E00E946414182FBE01F1
:1058E000802F0E94D3652F2D412F602F86E60E94C6
:1058F0007523812FDF91CF911F910F91FF90089514
:10590000FF920F931F93CF93DF93182F062FEA0177
:10591000F22E222321F061E00E945C14182FBE01B8
:10592000802F0E94D3652F2D412F602F86E60E9485
:105930007523812FDF91CF911F910F91FF900895D3
:105940007F928F929F92AF92BF92CF92DF92EF920F
:10595000FF920F931F93CF93DF93C82F8BEE90E1AD
:105960000E947022DDE0AD2E14E0C12E06EEE02E86
:1059700000E1F02E0CE020EA31E14AE06C2F82EDEC
:1059800097E00E948F231091D2079090400790914A
:105990006607C23278F0C63230F0CF3B59F48091BE
:1059A0003B0D806405C0992351F080913B0D8063CD
:1059B00080933B0D992319F0B2E0FB2E02C0FF2427
:1059C000F394183008F02EC1E4ECAE2EEDE0BE2EBC
:1059D000F2ECCF2EFDE0DF2EE50188248394A8E0D1
:1059E0007A2E6BED70E1872D0E94D3658C2F8A197A
:1059F000813029F442E5672D80E00E947A65181114
:105A000002C0992011F000E001C00F2DF6012081A5
:105A100040E952E1672D82E40E949F65181103C09E
:105A2000F1E09F1611F000E001C00F2D288130E059
:105A300040E050E073E0E72E672D86E60E94BA66EC
:105A4000181120C080916607811106C08091400125
:105A500090914101892BB1F091100AC022E043E0FE
:105A600060E0F60180810E944D14F60180830AC037
:105A7000F1E09F1207C022E048E760E088810E94C1
:105A80004D148883839488E0780E2196EFEFCE1A28
:105A9000DE0AF3E08F12A5CFC0916F0480E4C89FA7
:105AA000E001112461ED70E188E10E94D3651330BB
:105AB00041F4911006C080916607882321F002E02E
:105AC00003C000E001C001E0202FAE0168E184E5E1
:105AD0000E94CA67023061F480916F0422E048ECB2
:105AE00050E060E070E090E00E949A1380936F04B1
:105AF000133049F4E1E09E1206C0809166078823C6
:105B000021F0C2E003C0C0E001C0C1E00C2F209131
:105B1000700444E252E168E18AE50E949F65C23068
:105B200039F46FE0809170040E945C1480937004DB
:105B300066EC70E180E20E94D365143051F442E3D8
:105B400061E0809171040E9459148093710421E0F6
:105B500001C020E04091710450E060E284E50E94C1
:105B6000CA67C091D501C295C695C695C3706DEB45
:105B700070E188E20E94D365153091F462E08C2FC9
:105B80000E945C14C82F982F9295990F990F907CC2
:105B90008091D5018F73892B8093D5010F2D01C082
:105BA00000E02C2F42EB50E168E282E40E949F6506
:105BB00066EA70E180E30E94D365163069F4809153
:105BC000430422E042ED50E060E070E090E00E948B
:105BD0009A138093430401C0F12C209143040F2DAC
:105BE000006330E0220F331F442737FD4095542FC8
:105BF00064E0E62E60E384E50E94BA6621E0173097
:105C000009F020E08091D5014BE950E168E38295ED
:105C100081700E94802C9091D50180FB94F9909323
:105C2000D50124C06CE870E188E00E94D365CAE722
:105C3000D4E080E1F82E98E0D92EDC1A8C2F8D0D5F
:105C4000181307C061E288810E945C14888301E018
:105C500001C000E0299143E153E16F2D80E00E94F3
:105C60009F6588E0F80EE0E4FE12E8CFDF91CF9167
:105C70001F910F91FF90EF90DF90CF90BF90AF906A
:105C80009F908F907F9008951F93CF93DF93D62F8F
:105C9000122F0E94802CC82F212F482F6D2F86E6AF
:105CA0000E9483238C2FDF91CF911F910895CF9372
:105CB000482FCAE02AE0829FC00111248D519E4FD7
:105CC0002FE130E0241B3109C29FA001C39F500D7A
:105CD0001124BC01665F7F4F0E94B379E9E1F3E0D4
:105CE000DF011D92CA95E9F782E00E941060CF9112
:105CF0000C94AF600F93CF93C42F0E94FA1000232F
:105D000039F046E16AEE8C2FCF910F910C94591423
:105D10008C2FCF910F9108950F931F93CF93DF9303
:105D2000D82F162FC42F022F47FF08C041E28AEF59
:105D30008D0F0E94C86486E08C1BC82F2C2F4EEE5E
:105D40005EE0612F8D2F0E949F65DF91CF911F91A3
:105D50000F9108950F931F93CF93DF93162F8132E6
:105D6000C0F5811103C0611108C033C0803219F43D
:105D7000662329F02EC0662311F001E001C00FEF69
:105D8000080F0E942010EC01802F0E942010FC01BF
:105D900098818FEF890F8031E0F420812131C8F4A0
:105DA000291302C08BE009C0112329F0903188F437
:105DB0009F5F98830EC088830CC0815029F090812A
:105DC000288121939993F9CF82E00E94106000937B
:105DD000DC07DF91CF911F910F91089580911903F6
:105DE000882329F08BEC9EE10E940B1C81E0089532
:105DF0006BEF7DE088E20E94D3656CEE7DE080E38E
:105E00000C94D365CF93C82F813669F08F3B39F05E
:105E1000803699F4809112070E94572E04C080E0CA
:105E20000E940E720AC08C2F0E94BD6981E00E9400
:105E3000E81B83E39EE40E940B1C60EE7DE088E09B
:105E40000E94D365CF910C94F82E0F93CF93C82F57
:105E500080910F07882319F062E47DE002C065E3BA
:105E60007DE088E00E94D3654FE063E177E08091B8
:105E70000E070E94D45E00E12AE043E157E060E1B2
:105E800081E00E947D654FE360E182E40E947A65D3
:105E90000E94F82EC13609F44EC0CF3B21F0C03627
:105EA00009F055C005C080E0CF910F910C940E729F
:105EB00080910F078823A9F083E29DE00E940913D7
:105EC00080910E070E94495F882339F087E10E9484
:105ED0000E7282E080930F072CC080E00E940E7249
:105EE00028C08091E3048F5F0E940062C091E304A8
:105EF00081E08C0F0E94D061811109C0C150C13175
:105F000008F0CFE08091E304C813F2CFC0E0C09363
:105F1000E30481E00E9410600E94AF608091E3047E
:105F20000E940B5F8091D3010E949F1482E08093B6
:105F30000F0180E601C081E60E94BD6981E00E94F8
:105F4000E81B80E297E3CF910F910C940B1CCF914B
:105F50000F9108959091B40181E0191624F09111E8
:105F600001C080E081951092B4010895CF93C82FAD
:105F70000E94AA2F909111072091AB01223671F057
:105F800028F4203639F02136A9F006C0233661F016
:105F90002E3611F481E00FC0181624F49C1730F44B
:105FA0009F5F04C0882311F09111915090931107C5
:105FB00080E001C082E0CF91089566ED7DE088E049
:105FC0000E94D3656CEC7DE080E10E94D36562ECB9
:105FD0007DE088E10E94D36568EB7DE080E20E946D
:105FE000D3656EEA7DE088E20E94D3652AE240E351
:105FF00067E082E10C94DC67CF93DF9380E00E943E
:10600000DD2F84E00E94B62FD82FC09111076C2F8E
:10601000660F660F660F685F20E044E288E10E9429
:106020000166D130B9F5C13089F40E94EE2E81119C
:106030000FC0C093DA078091DD078F5F8093DD0783
:1060400060E00E94E01E1092100702C0C23018F4F7
:106050008BED9BE40EC08091DD07C43069F4809322
:1060600012078091AB010E94BD691092AB0182E0E2
:106070009FE20E940B1C0BC0C23031F48F5F8093F3
:10608000DD0761E00E94E01E81E08093100710921E
:106090003F070AC0D23041F410923F078091AB0114
:1060A0000E94BD691092AB018091DD078093DC07EF
:1060B000DF91CF910895CF92DF92EF92FF92CF932D
:1060C000DF93FC01EB019C01DC010E94FC789B0149
:1060D000AC01DE010E941279272F382F492F552756
:1060E000DF010E9412796B017C013CE0F694E79499
:1060F000D794C7943A95D1F724E630E02C1B3D0B9A
:106100000E94FC786E5C7F4F8F4F9F4F6C0D7D1D02
:106110008E1D9F1D24E630E040E050E00E945D7936
:10612000C901DF91CF91FF90EF90DF90CF9008955C
:106130001F93CF93DF936115710529F1192F111F5B
:106140001127111F19F091958195910977FF10C0C2
:10615000719561957109C0E0D4E09E01281B390B4F
:10616000C9010E945B309E01281B390BC90102C086
:106170000E945B30112329F022273327281B390B7B
:1061800001C09C01C901DF91CF911F9108956F92C9
:106190007F928F92AF92CF92EF920F93CF93DF9334
:1061A000CDB7DEB7382F562F822F602F9C2D44237A
:1061B00021F0552329F022E00AC020E000E008C0C9
:1061C000E0914001F091410121E0EF2BB9F301E0B2
:1061D000442311F0311121E03EE0E39E300111240F
:1061E000A3014D585C4F3A01933639F4FA014485C6
:1061F0000E947A2EF30184872AC0923639F4FA017C
:1062000045850E947A2EF301858721C04A2D50E0F2
:10621000490F511D490F511D440F551F480D511D68
:10622000460D571DFA013F01A11007C04081E22E23
:1062300004E62CE90E94C02108C040814C59E22E9E
:1062400004E620E00E94C0218456F3018083DF91A0
:10625000CF910F91EF90CF90AF908F907F906F90F4
:1062600008952F923F924F925F926F927F928F92FA
:106270009F92AF92BF92CF92DF92EF92FF920F93D5
:106280001F93CF93DF9300D000D000D0CDB7DEB7FF
:10629000182F8BE99DE00E94702293E0A92EC12C5B
:1062A0002AE9E22E2DE0F22E00E020E030E040E08E
:1062B000612F8CEC97E00E948F2310925501409142
:1062C000D9074F5F20E060E080E30E94A310F090C8
:1062D000CC078091D9070E942322182F8091D907DB
:1062E000E82FF0E0EE0FFF1FE857F84F20813181D3
:1062F0002A3131051CF01092CB0706C0273E3F4FD4
:106300001CF491E09093CB070E94321781111092F8
:10631000CB0765E97DE080E10E94D36541E0F110A3
:1063200040E08090CB07A12CC12EE090D90700E17E
:1063300026E361E081E00E94C7306EE87DE088E1FD
:106340000E94D36541E0F41240E08090CB07AA247C
:10635000A394C12EE090D90708E126E361E081E033
:106360000E94C73068E87DE080E20E94D36541E08A
:10637000E2E0FE1240E0812CA12C83E6C82EE090E2
:10638000D90700E22EE161E081E00E94C73062E8B7
:106390007DE088E20E94D36541E0F3E0FF1240E037
:1063A000812CA12C02E6C02EE090D90708E22EE154
:1063B00061E081E00E94C730113029F0123031F4E1
:1063C00064E77DE005C06BE77DE002C06CE67DE040
:1063D00080E30E94D3652091D9078EE0289F900129
:1063E000112494E0199F200D311D112427533E4F95
:1063F000F901E655FE4FD901A555BE4F1C91D901B3
:10640000A455BE4FFC9084E6F80ED901A355BE4FAB
:106410000C910C5980810E942417682E812F0E94B4
:106420002417382E44E660E08F2D0E940B17782E3B
:1064300044E660E0802F0E940B17582E8091D90708
:106440000E943217E62DFF27E7FDF095FE83ED83CE
:10645000E72CFF24E7FCF094882309F464C0812C26
:10646000912C540110E0A4E6CA2ED12CB0E44B2E9E
:106470006D817E81D501C401B595A79597958795C6
:106480000E949830880F991F61E270E00E9449795C
:106490006E9DC0016F9D900D7E9D900D11240FE3A8
:1064A000010FB6010E943579F42DF61B6F2F802F56
:1064B0000E941E66812F837051F46FE3802F0E942B
:1064C0001E66612F6695605E8FE30E941E661F5FE9
:1064D00021E2820E911CA11CB11C1E3349F6E091F1
:1064E000D907F0E0EE0FFF1FE857F84F0081118148
:1064F0004801AA2497FCA094BA2CC501B40121E25A
:1065000030E040E050E00E947F794EE361E08EE5AC
:10651000820F0E946E668091D9070E9432178823ED
:1065200009F4ABC06CC000E010E0912C31E2C32E46
:10653000D12C44E6A42EB12C50E2252E832D992790
:1065400087FD90959A838983E52DFF27E7FDF095D8
:10655000FC83EB836D817E81C8010E949830B60177
:106560000E9449796E9DC0016F9D900D7E9D900D9A
:1065700011242EE5822E890CB5010E943579F22D69
:10658000F61B6F2F882D0E941E66292D2370422E28
:1065900049F460E2882D0E941E6660E2690D8EE576
:1065A0000E941E6669817A81C8010E949830B601F6
:1065B0000E944979EB81FC816E9FC0016F9F900D15
:1065C0007E9F900D1124BEE58B2E8918B5010E9487
:1065D0003579605E882D0E941E66411009C060E218
:1065E000882D0E941E66622D69198EE50E941E6626
:1065F00093940F5D1F4FFFE19F12ACCF70CFC50189
:10660000B4017C5F8F4F9F4F22E030E040E050E0CC
:106610000E947F796D817E81C9010E9498309C0122
:10662000220F331FA72D77FCAD5FA595A595BB273E
:10663000A7FDB0950E94F47829E130E040E050E0F9
:106640000E947F7969017A01CA01B9012FED3FEFFC
:106650004FEF5FEF0E947F7960E4620F4EE38FE3BC
:106660000E946B66C701B60122E030E040E050E0D6
:106670000E947F7969017A0135C0181419041A043F
:106680001B040CF0632C662D772767FD7095C801FD
:106690000E949830181419041A041B0414F4A72D2E
:1066A00001C0A52DA7FDAD5FA595A5959C01BB27B4
:1066B000A7FDB0950E94F47829E130E040E050E079
:1066C0000E947F7969017A01CA01B9012FED3FEF7C
:1066D0004FEF5FEF0E947F7960E2620F4EE38FE33E
:1066E0000E946B6629E130E0D8010E940B79412CB1
:1066F000512C32015394A30192010E947F79A90188
:1067000060E382E70E94D967A9E1B0E0A7019601A2
:106710000E941279A30192010E947F79A90168E089
:1067200084E50E94D967181419041A041B045CF448
:106730006D817E81C80144970E9498309601281B84
:10674000390BC9010AC0632D772767FD7095C80111
:1067500044960E9498308C199D0945E0489F90010D
:10676000499F300D1124442737FD4095542FE3E015
:10677000EE2E00E360E184E50E94BA6626960FB62D
:10678000F894DEBF0FBECDBFDF91CF911F910F9167
:10679000FF90EF90DF90CF90BF90AF909F908F9041
:1067A0007F906F905F904F903F902F9008952F9221
:1067B0003F924F925F926F927F928F929F92AF9291
:1067C000BF92CF92DF92EF92FF920F931F93CF93DE
:1067D000DF93CDB7DEB72B970FB6F894DEBF0FBEB1
:1067E000CDBF182F84E69DE00E947022F4E0AF2E0A
:1067F000CC24C394A2E6EA2EADE0FA2E0CE020EA07
:1068000031E143E0612F8AEC97E00E948F23809171
:10681000CA07FF24FA94F80E2091400729838111BA
:1068200010925501103871F480E80E94BD691092F1
:10683000AB01F7FC52C181E391E30E940B1CF09283
:10684000D9074BC142E55DE068E085E10E94D9656A
:1068500076EC672E77E0772E88E897E09F838E832B
:1068600010E11B861A86EEE05E2EEF2DFF27E7FD76
:10687000F095FB83EA83BA848B2D0E942322982E05
:1068800084E0989E900111243D832C83EA85FB854A
:106890005E9EC0015F9E900D1124820F931F87534F
:1068A0009E4FDC01A355BE4FFC01E455FE4F3C91C9
:1068B000208132130DC0FC01E555FE4FDC01A655C9
:1068C000BE4F31E020818C91281330E0432E01C06F
:1068D000412CEE81FF8181919191FF83EE839C0198
:1068E000275E3F4F2333310508F0412C79866886B7
:1068F000F301F0808A31910534F4873E9F4F24F4F0
:10690000FF24F39401C0F12C8B2D0E9432178823B1
:1069100019F0F12C44244394F301F08220E041E08B
:106920004B0D612F80E00E94A31033243394F110AB
:10693000312C8091660781110AC021E080914001CD
:1069400090914101892B09F420E0D22E02C0DD2470
:10695000D3942A813B818A859B852817390731F496
:1069600081E09981911180E0282E01C0212CF30152
:106970008080A12CC92CEB2C012F27E2422D6D2DFC
:1069800080E00E94C7302220C9F0DD20B9F0442009
:10699000A9F02A853B85529EC001539E900D11247B
:1069A000EC81FD818E0F9F1F8D589C4FFC01EF0DD8
:1069B000F11D2081FC01E30DF11D20832A813B8123
:1069C0008A859B852817390739F481E099819130B0
:1069D00009F080E0282E01C0212CEFEF6E1A7E0A0C
:1069E000E885F9858080AA24A394C92CEB2C012F7B
:1069F00029E3422D6D2D80E00E94C7302220C9F08E
:106A0000DD20B9F04420A9F02A853B85529EC001C3
:106A1000539E900D1124EC81FD818E0F9F1F8B588A
:106A20009C4FFC01EF0DF11D2081FC01E30DF11DD8
:106A300020832A813B818A859B852817390721F489
:106A400041E09981923009F040E0812CA12C63E66D
:106A5000C62EEB2C012F2FE36D2D80E00E94C73056
:106A6000EA81FB812A853B85E217F30721F441E0A7
:106A70003981333009F040E0812CA12C52E6C52E3B
:106A8000EB2C012F27E56D2D80E00E94C7304110CF
:106A900004C0FF2029F04FE701C04DE28AE302C0A5
:106AA0004EE78BE3612F0E947A6581E0981629F00A
:106AB00092E0991204C04CE403C04DE401C048E4E4
:106AC000612F85E70E947A65EA85FB853196FB8711
:106AD000EA87185F103309F0CECE2B960FB6F894E4
:106AE000DEBF0FBECDBFDF91CF911F910F91FF9001
:106AF000EF90DF90CF90BF90AF909F908F907F905E
:106B00006F905F904F903F902F90089590E0E92F05
:106B1000FF27E7FDF095E155FD4EE491E81302C033
:106B2000892F0895EE2311F09F5FF1CF80E0089543
:106B3000823430F4E82FF0E0E155FD4E8491089561
:106B400080E20895FF920F931F93CF93DF93C82F96
:106B5000D62FF42E122F622F842F0E940E13FC01C9
:106B6000E53F81E0F80794F09BE09E0F9F1510F041
:106B70009CE09E0F40E3490F202F6D2F8C2FDF915B
:106B8000CF911F910F91FF900C94C864212F40E981
:106B90005BE06D2F8C2F0E949F65DF91CF911F913D
:106BA0000F91FF900895BF92CF92DF92EF92FF92E4
:106BB0000F931F93CF93DF93C82F83E79BE00E942F
:106BC000702206E0E02E0CE020EA31E142E06C2F7A
:106BD00083EC97E00E94E825B090C307C03611F01F
:106BE000CE3669F48FEF8B0D843048F48093DF0745
:106BF0008C2F0E94BD6981E496E30E940B1C6AE61B
:106C00007BE088E00E94D365C9ECD1E010E1F12E71
:106C100011E0CC24C3941B11C12C67E67BE08F2DBF
:106C20000E94D36540E3410F6F2D8CE00E947A658E
:106C30002C2DFE01E353FD4F40816F2D8AE20E940F
:106C4000FA10BAE5DB2EE12C0C2D2E2D412F6F2DE5
:106C50008D2D0E94A235E39486E0D80E84E0E812E0
:106C6000F3CF1F5F88E0F80E2A96153091F6DF917A
:106C7000CF911F910F91FF90EF90DF90CF90BF9039
:106C800008956F927F928F929F92AF92BF92CF9210
:106C9000DF92EF92FF920F931F93CF93DF93C82F52
:106CA0008090DF072AE0829E40011124C4018257B0
:106CB0009B4F4C0188E89BE00E947022AA24A39479
:106CC000CC24C39426E8E22E2BE0F22E00E020E054
:106CD00030E040E06C2F84EC97E00E948F234091DD
:106CE000DF074F5C60E080E30E947A65C090C407D4
:106CF0006090660718E0E12CF12CDD24C7FCD094ED
:106D00008E2DCE14DF0429F416142CF492E0A92E53
:106D100004C0A12C02C0AA24A394813081F06FE7A3
:106D20007BE0812F0E94D3650A2D2A2DF401408536
:106D3000612F80E30E947A2EF401808751C069E7B9
:106D40007BE0812F0E94D36580E3782EB12C809167
:106D500040078B1511F000E001C00A2D4091DF07BC
:106D60004F5F2B2D612F872D0E94A235AA2091F114
:106D7000209140072B112EC0161434F08091400151
:106D800090914101892B31F1E401C20FD11DC20F55
:106D9000D11DE881F981CF018B509E4F843FF1E0F6
:106DA0009F0714F484EF91E022E048EF51E064EF94
:106DB00071E00E949A13AC0180914801882351F040
:106DC000443F21E0520711F440E050E0455F51405C
:106DD00059834883B39486E0780E94E0B912B7CF14
:106DE000EFEFEE1AFE0A185F183109F089CFDF9134
:106DF000CF911F910F91FF90EF90DF90CF90BF90B8
:106E0000AF909F908F907F906F900895CF93C62FF3
:106E10000E94BD690E94AF60C093E3048C2F0E9462
:106E20000B5F8091D3010E949F1482E080930F0139
:106E300081E00E9410600E94AF6081E0CF910895D0
:106E4000BF92CF92DF92EF92FF920F931F93CF9357
:106E5000DF93D82F8EE59BE00E9470228091660719
:106E6000811110C0E0916307E7FF0CC0E195EC30A1
:106E700008F0EBE0F0E0EE0FFF1FE056FE4E8591CC
:106E800094915BC01091C2074FE06D2F82EC97E0A8
:106E90000E94F92568E57BE080E00E94D3650E94AE
:106EA0002361AC0160E086E60E94D96741E06CE0B6
:106EB00080E00E94851EC091C20780910F0782303A
:106EC00021F41092C10710920F07D63638F4D43649
:106ED000F0F4D036E9F1D13659F05EC0D13809F47A
:106EE00040C0DF3B09F44FC0D03809F055C03DC069
:106EF0008091C107882359F01092C10787E10E9451
:106F00000E726091C20781E60E94063745C08091EB
:106F1000E3048C1739F06C2F8D2F0E94063781E027
:106F20000E940E72D53629F488E299E20E94731409
:106F300033C0D43689F589ED96E5DF91CF911F9165
:106F40000F91FF90EF90DF90CF90BF900C9473144F
:106F500081E08093C1071092660787E10E940E725C
:106F60001BC081E00E94E81B17C08091C1078823E5
:106F700099F081E080930F07C0930E0785E29FE2AE
:106F80000E940B1C09C01092C1078091E3048093FA
:106F9000C20781E00E9422608091C107882341F0EE
:106FA0001C1731F061E06C0F81E0810F0E94DE61FF
:106FB000DD27C7FDD095809167079E01281B310909
:106FC000C901181619065CF0CE01019797FF02C09F
:106FD00080E090E08093670710E1B12C0BC0253072
:106FE0003105D4F3CE0104978B3091059CF38AE0F0
:106FF00090E0F0CFF0906707FB0CCF2CD12CCC1594
:10700000DD0511F401E101C000E196012F5F3F4F62
:10701000442737FD4095542F62E0E62E612F82E130
:107020000E94BA668091E304F81205C04AE2612F1B
:1070300081E00E947A654FE063E177E08F2D0E9446
:10704000D45ECC15DD0531F48091C107882311F0A1
:1070500001E101C000E12FE043E157E0612F88E149
:107060000E947D65B394185F36E0B312C3CFDF9101
:10707000CF911F910F91FF90EF90DF90CF90BF9035
:107080000895DF92EF92FF920F931F93CF93DF93B8
:10709000E82E0091D401C7E9D7E010914404202FD5
:1070A000332727FD309537FF03C0319521953109EE
:1070B0002532310554F12D853E854F855889242B85
:1070C000352B4B855C85242B352B8989282B8A8988
:1070D000282B232B29F4802F881F8827881F8A8B31
:1070E000101614F48CED01C084E2800F40E060E0E3
:1070F0000E945517882341F09A89911105C091E0AB
:107100002989211190E0998B8A8B112339F040E075
:1071100060E0812F0E945517882319F0FF24F39413
:1071200002C0F12CE12C2D853E852F5F3F4F3E871D
:107130002D872F8538892E0D311D388B2F87F89498
:107140002091420C3091430C78948B859C85281BB0
:10715000390B2436310508F423C18C599F4F9C8785
:107160008B872F853889ED85FE85C901BF010E9477
:107170003579E62ED62E6E9FC0016F9F900D11249B
:10718000281B390B388B2F871E861D868FE0800FBA
:107190008F3110F4198A0DC094E2900F993448F49D
:1071A000101614F481EF800F40E060E00E94551744
:1071B000898B2091D401332727FD309537FF03C0F9
:1071C000319521953109622F8881998101969983A2
:1071D0008883EA81FB813196FB83EA83DD2029F0F5
:1071E0008E819F8101969F838E83613009F4698B24
:1071F0008989882341F0FF2031F04C815D814F5F08
:107200005F4F5D834C83E694488559854E0D511D33
:1072100059874887E090D601F090D701FC8AEB8A25
:10722000611102C01A8620C0613031F4111114C0FE
:10723000C7018E1B9F0B16C0603170F420FF06C083
:10724000E4E056954795EA95E1F702C04E815F81EB
:10725000C701841B950B06C08C819D819701281B5B
:10726000390BC9019C8B8B8B8A850B891C898130DA
:1072700049F018F0823069F017C08091D40188235A
:1072800099F010C017FF10C0E114F10469F082E01A
:107290000AC0053C3FEF130714F483E08A87E1142A
:1072A000F10411F481E08A87898D9A8D8017910706
:1072B00009F46AC08A85813009F057C08091FC04C6
:1072C00082FF31C0E114F10471F10E31110519F49E
:1072D00069E289E10BC00431110519F46AE28AE11F
:1072E00005C00A30110531F46BE28BE10E94147283
:1072F00081E00DC0063011054CF417FD03C0602F6E
:107300008CE1F4CF8CE10E940E72F2CF80E090917C
:10731000FC0493FF08C0882331F082E390E090934F
:107320003C0180933B018091D50180FF04C0C701DF
:10733000801B910B01C0C8016CE370E00E94497989
:10734000DC01CB014091FC0441FF1EC0AB2BE1F4FA
:107350004091050541FF07C0009761F046E260E0FB
:107360000E941D7207C080E003C0823069F48CE186
:107370000E940E728091FC0483FF06C082E390E0BD
:1073800090933C0180933B018B899C899A8F898FD4
:107390002091D50120FF04C0E81AF90AFC8AEB8A83
:1073A000DF91CF911F910F91FF90EF90DF900895A3
:1073B0009091D40197FD91958EEF890F8E3020F535
:1073C000892F85959A3024F40E947F6A90E003C04B
:1073D000992787FD90950197FC01EE0FFF1FE85755
:1073E000F84F208131818091D40187FF05C080E072
:1073F00094E0821B930B02C0C9019C5F26E0969526
:1074000087952A95E1F702C080E090E00E9441381C
:1074100083E00E947F6AE82FF0E0EE0FFF1FEA573B
:10742000F84F808191819C5FB6E096958795BA95DB
:10743000E1F72091D50122FF0AC08530910538F08F
:107440002091AE07211103C023E02093AE072091C5
:10745000B9073091BA072F5F3F4F3093BA07209397
:10746000B9072091B7073091B807280F391F30931B
:10747000B8072093B707F8948091420C9091430C81
:1074800078942091B5073091B607AC01421B530B9D
:107490009A01283E3340D8F19093B6078093B50700
:1074A0008091D801823039F440E060E085E10E94AB
:1074B0005517811128C08091B7079091B807609146
:1074C000B9077091BA070E9435791092B8071092E7
:1074D000B7071092BA071092B907809194068937BE
:1074E00018F48F5F80939406E091950681E08E0FEB
:1074F00080939506F0E0EA56F94F6083883738F0BC
:1075000010929506089587E00E940E72D4CF0895D8
:10751000E7E9F7E01286138212821782168215823B
:107520001482118610868091D6019091D701928F96
:10753000818F0895EF920F93562F642F22FF02C080
:1075400095E001C093E0022F0064E82FF0E0EE0F19
:10755000FF1FEE58F24F2081318148E0480FE92E9D
:10756000852F0E94CA200F91EF900895CF92DF924D
:10757000EF92FF92CF93DF936B017C01C0E1D0E0EB
:1075800040E050E8E0E0F0E89A01DA010E94FC787F
:10759000C616D706E806F90610F44E275F27F695BB
:1075A000E7952197209719F04E2B5F2BEDCFCA015D
:1075B000DF91CF91FF90EF90DF90CF9008951F93D0
:1075C00041E0262F30E0683050F440E055E0529F13
:1075D000F001539FF00D1124E155FC4F0AC02850D3
:1075E000310959E0529FF001539FF00D1124E952E7
:1075F000FC4F9C5F97FD0DC0811528E0920784F039
:10760000442319F088E090E002C084E090E0E80FA5
:10761000F91F2081332727FD3095322F222725C0DF
:10762000442329F0492F9927880F991F03C0492F18
:1076300046959170242F30E0E20FF31F608140E007
:1076400052E0481B590B5595479564039001659F7F
:10765000300D11241181BC01759567951603A001A9
:10766000179F500D1124240F351FC90169E170E0E7
:107670000E944979CB011F9108953F924F925F92EA
:107680006F927F928F929F92AF92BF92CF92DF9232
:10769000EF92FF920F931F93CF93DF93982EBB240B
:1076A000B3948091DE07883008F4B12C82E791E131
:1076B0000E947022BB2011F08AE001C086E0A82E53
:1076C000CC24C394F0E7EF2EF1E1FF2E00E020E0A0
:1076D00030E040E0692D87ED97E00E948F234091D4
:1076E000DE0750E04F5F5F4F21E060E084E20E94E0
:1076F000CA67C091DE07BB2061F08C2F90E008972D
:1077000029E0289FE001299FD00D1124C952DC4FA8
:1077100006C025E0C29FE0011124C155DC4F6090F6
:10772000D7076A94A090400741E6941681F0491566
:1077300038F054E49516E1F085E4981689F02EC0EF
:10774000E4E69E16A9F0F5E69F1651F027C0AA20A0
:1077500029F11092400781E60E94BD69A12C1EC04C
:10776000809166078823D1F01A14C4F48FEF13C0F8
:1077700080916607882391F02A2D332727FD3095C5
:10778000BB2019F089E090E002C085E090E0281766
:10779000390724F481E08A0D8093400780914007E7
:1077A000809366078C2E7D2ECC2EDD2E05E010E01A
:1077B000E0E15E2EE62CFF24E7FCF094F601419117
:1077C0006F0121E0C8010597E816F90609F020E0ED
:1077D000552747FD5095652D88E10E94CA67BB205B
:1077E00091F0093081F021E0E016F10609F020E087
:1077F000FE01E00FF11F4081552747FD5095652D93
:1078000080E30E94CA67F8E05F0E0F5F1F4F28E316
:107810005212D4CF4FEF641202C021E0A11020E039
:1078200049E651E168E08CE00E94B365BB2019F0A5
:1078300089E090E002C085E090E021E0E816F906DA
:1078400009F020E042E651E168E38CE00E94B36574
:10785000BB2019F089E090E002C085E090E0E816D6
:10786000F9066CF467FC50C0EC0EFD1E44E66CE9B2
:10787000F70180810E945914F701808345C01614D6
:107880000CF042C020E044E06CEF8091D6070E94EB
:107890004D148093D607909148019923A9F1BB20FC
:1078A00021F090E164E049E003C098E062E045E047
:1078B000F4E68F028001112470E0719561957109E1
:1078C000582F56039001579F300D112484E6829F54
:1078D0006001839FD00C1124E82DF72D20E030E0CB
:1078E000E92EF12CC9018C0D9D1DB7010E9449792B
:1078F0006193200F311F8E2F8819841798F382E02F
:107900000E9410600E94AF6080916607882309F48E
:1079100059C0712C7CE9E72EFF24FA94CA2CDD248F
:10792000C7FCD094892D8F7DA82EEEEBAE0E40C003
:10793000C90155E0880F991F5A95E1F7BB2009F45A
:107940004AC064E070E00E944979462E4E01820EE2
:10795000931EF4018081F0E28F02C0011124B7016F
:107960000E944979662E40E2542E560E2F5F3F4FFB
:10797000052D10E0C216D30609F05EC002341105D1
:107980006CF12FE3251530F045E0652D8AE3840D79
:107990000E946B660F331105A4F180914001909114
:1079A0004101892B09F03FC051E05A15E0F573946D
:1079B000272D30E0BB2061F089E090E028173907DF
:1079C0000CF4B6CFC0E0DCEF10E060E2F62E52C05F
:1079D00085E090E0F3CF62E070E0B5CF3AE3332E7C
:1079E000340C45E06EE1660D832D0E946B66013418
:1079F000110539F245E06FE1660D832D0E946B663B
:107A0000C0CF4AE3440E45E061E2660D842D0E943A
:107A10006B660E33110509F262E2660D45E0842DB6
:107A20000E946B66BACF44E66CE9F40180810E9443
:107A30005914F4018083BBCFFBE34F0E01341105D1
:107A400034F443E06FE1660D842D0E946B662FE3F2
:107A5000251528F043E0652D842D0E946B660F33B9
:107A600011050CF0A4CF61E2660D43E0842D0E9465
:107A70006B669DCF6091DE07CE010E94DF3A0CE37A
:107A8000010F25E0969587952A95E1F76F2D681BE4
:107A9000802F0E941E66812F837021F460E2802F68
:107AA0000E941E661F5FA096103421F740E460E03C
:107AB0008CE5DF91CF911F910F91FF90EF90DF90B8
:107AC000CF90BF90AF909F908F907F906F905F907E
:107AD0004F903F900C946E662F923F924F925F9220
:107AE0006F927F928F929F92AF92BF92CF92DF92CE
:107AF000EF92FF920F931F93CF93DF93CDB7DEB733
:107B00006E970FB6F894DEBF0FBECDBF8D8F9E8FE0
:107B1000698780913D01882309F44EC080916407F4
:107B2000882319F08150809364070E949A15209150
:107B30004B0630914C068217930761F090934C06E8
:107B400080934B0610924E0610924D0681E0809372
:107B50003A0132C06091FB04665F71F180910201CD
:107B6000823350F180914F068F5F80934F068031B2
:107B700018F180914D0690914E06019690934E0615
:107B800080934D0610924F0647E751E0649F9001A5
:107B9000659F300D11242817390770F48F719927CC
:107BA000019751F486EF9FEF0E9489146DE280E106
:107BB0000E9414720E94A7140E942D1C809331050C
:107BC0008091FA04282F2170822E839481FF02C0B5
:107BD000612C02C033E0632E4091E1014423F1F1B6
:107BE000E82DF0E0EE0FFF1FE857F84FA081B181BC
:107BF000E62DF0E0EE0FFF1FE857F84F0190F081FF
:107C0000E02D9D010E94F4786B017C019F01DF0152
:107C10000E94F478C60ED71EE81EF91E642F70E08D
:107C200080E090E02AE0660F771F881F991F2A9551
:107C3000D1F724E630E040E050E00E947F79CA01AD
:107C4000B9010E9425796C157D058E059F0530F4DC
:107C5000C701B6010E94B63A7C0102C0E12CF12CAA
:107C60009701A4E6B0E00E94FC786D8B7E8B8F8B31
:107C7000988FB7EB4B2EB4E05B2E42EF55E05C875C
:107C80004B87BE016F5F7F4F7E876D8788E897E0E7
:107C90009A8B898BC12CD12C712C99859170998FDD
:107CA000A985AE70AA8FB985BA70BB8FE985E670D9
:107CB000EC8F9C2C8C2D0E948A1592012E5F3F4FD9
:107CC000388B2F87D2012D913C91821B930B9C0105
:107CD000BC01882777FD8095982FAAE0660F771F53
:107CE000881F991FAA95D1F7EF85F88912161306F8
:107CF0001CF4228D338D02C0248535852436310550
:107D000014F424E630E0442737FD4095542F0E94B8
:107D10007F7989012130FCEF3F073CF0011524E019
:107D200012072CF000E014E002C000E01CEF80918C
:107D3000FC0480FF11C08091FA0481708B8B1C8A37
:107D400082E090E04B895C89841B950BC816D906AC
:107D500019F4119501951109A989BA890D931D93FB
:107D6000BA8BA98B580117FF03C0BFE0AB0EB11C43
:107D7000F4E0B594A794FA95E1F73A2CE4E0CE1636
:107D8000D1045CF481E0890D0E947F6A815091E00A
:107D900001C0990F8A95EAF706C091E00C2C01C04A
:107DA000990F0A94EAF737FE02C03A2C3194F1E0B9
:107DB000F31544F0311002C0892F03C080914A06A8
:107DC0008923782A23E0291508F422C1398D31113D
:107DD0004DC08091D50181FF49C0520149E3A40EF5
:107DE000B11CF5018181807C09F440C0F20181ADB4
:107DF00040E061E08595859585950E94551788231B
:107E0000A9F1D501EC91E770F0E0DF01AA0FBB1FEB
:107E1000A65DBE4FEE0FFF1FE851FB4F8D919C9169
:107E200020813181821B930B97FD0196AC01559502
:107E30004795F5012181322F330F330F3595359555
:107E40003403C001359F900D11246FE170E00E9452
:107E50004979660F771F660F771F2295269526951D
:107E60002370213009F08FC6060F171FE114F104AB
:107E7000C1F0981411F0961014C02091E10130E087
:107E8000D8010E940B79EAE0660F771F881F991FBF
:107E9000EA95D1F72D893E894F89588D0E947F79C7
:107EA0008901892D0E942322A82E892D0E94321734
:107EB000EA2DF0E0882311F1EE0FFF1FEE0FFF1FF8
:107EC0002EE02C9DC0012D9D900D1124E80FF91F6F
:107ED000ED58FC4F80810E942417682F772767FD9B
:107EE0007095C8019C5F97FD0196959587950E94B6
:107EF00098308C01000F111FB12C24C081E01016A6
:107F000011060CF480E0B82E3EE03C9DC0013D9D82
:107F1000900D1124EE0FFF1FEE0FFF1F8E0F9F1FFE
:107F200087539E4F8B0D911DFC01E655FE4F8081BE
:107F30000E942417682F772767FD7095C8010E945B
:107F400098308C014EE04C9DC0014D9D900D112448
:107F500054E0A59E800D911D112487539E4F8B0DDB
:107F6000911DFC01E455FE4F808144E660E08C5990
:107F70000E940B179801A82FBB27A7FDB0950E9460
:107F8000F47824E630E040E050E00E947F798901F7
:107F9000892D0E94321781111450892D0E942817B3
:107FA000811106C0692D809131050E9454132AC0A9
:107FB0008091DA0180FFF6CF692D809131050E9412
:107FC0005413282F8091FC0480FD2195332727FD31
:107FD0003095432F532F23583F4F4F4F5F4FA0E013
:107FE000B4E0A01BB10B0E941D7920E038E040E016
:107FF00050E00E947F79211568E036074105510560
:1080000089F2C901880F991FAD85BE858D939C9318
:10801000EB85FC8511830083FA8DFF23F9F023E0C3
:108020002915E0F0892D0E942817811113C03B8D7E
:10803000332349F0065F1F4F0531110520F0AB8552
:10804000BC851D921C92BC8DBB2321F0ED85FE8565
:1080500011821082EB85FC85118E108EFFEFCF1AF6
:10806000DF0A2B853C852E5F3F4F3C872B874D8554
:108070005E854E5F5F4F5E874D8757E0C516D10422
:1080800019F04F84588815CE1091DE011721809188
:108090004A068095812319F088E10E940E721093A0
:1080A0004A0680E094E09093010680930006909346
:1080B00003068093020682E10E946C69811108C068
:1080C00083E10E946C69882331F080E090E005C074
:1080D00080E09CEF02C080E094E090933B068093A8
:1080E0003A062AE231E00AE016E0E8EEF4E060E069
:1080F000D9018D919D919D01643020F44081518181
:10810000841B950B880F991FD8018D939D938D012A
:108110006F5F3296683061F72AE136E0E0E5F6E01D
:108120004191519161917191D9014D935D939D015F
:10813000B6E0E039FB07A1F7E0E8F4E0ACE3B6E035
:10814000808128E08202C00111248D939D93329694
:1081500034E0EE38F307A1F7A090E101AA2009F47A
:108160006EC0E82CF12CEE0CFF1CA7014E505A4FAC
:108170007A01DA01CD90DC90062D10E0000F111F7E
:108180000E501A4FF801408151819601D6010E948C
:10819000F4781B012C019A01DA010E94F478260E72
:1081A000371E481E591E6A2D70E080E090E0EAE01C
:1081B000660F771F881F991FEA95D1F724E630E0F4
:1081C00040E050E00E947F79CA01B9010E94257900
:1081D000621573058405950590F5C201B1010E94F1
:1081E000B63A9C01A4E6B0E00E94FC781B012C0189
:1081F000B12C9501D6010E940B792AE0660F771FFA
:10820000881F991F2A95D1F7A20191010E947F79B9
:10821000D7012D933C93F801A081B18195010E9473
:108220000B793AE0660F771F881F991F3A95D1F7AF
:10823000A20191010E947F79D8012D933C93609116
:10824000DF01862F807E09F4F8C089858A7089F461
:10825000E82DF0E0EE0FFF1FEE50FA4F2081318144
:10826000E62DF0E0EE0FFF1FEE50FA4F8081918176
:1082700004C080E090E020E030E049854670A1F441
:10828000FE013196E80DF11DE80DF11D408151818F
:10829000240F351FFE013196E60DF11DE60DF11D8F
:1082A00040815181840F951FE091E001EE2341F060
:1082B000F0E0EE0FFF1FE051FA4F4081518102C004
:1082C00040E050E062FF03C031952195310963FF22
:1082D00003C091958195910964FF03C05195419523
:1082E0005109629566956770623009F451C018F4BF
:1082F0006130E1F0A2C0633009F489C0643009F054
:108300009CC0FA01E21BF30BF0930506E093040610
:108310009A01280F391F3093070620930606481B41
:10832000590B509309064093080687C0BC0197FF7C
:1083300002C0695F7F4FB3E075956795BA95E1F725
:10834000FC01E61BF70BBC0197FF02C061587F4F91
:10835000660F672F661F770BE61BF70B97FF02C0B0
:1083600081509E4FBC01672F770F770B6595CF012A
:10837000861B970BBA01621B730B70930506609303
:10838000040637FF02C02F5F3F4F3595279546C043
:10839000B90137FF02C0695F7F4F13E0759567959C
:1083A0001A95E1F7F901E61BF70BB90137FF02C097
:1083B00061587F4F660F672F661F770BE61BF70B21
:1083C00037FF02C021503E4FB901672F770F770B5F
:1083D00065959F01261B370BBA01681B790B7093BB
:1083E00005066093040697FD019695958795840F81
:1083F000951FAC01420F531F50930706409306068A
:10840000821B930B909309068093080616C0BA014D
:10841000621B730B7093050660930406240F351FCF
:10842000A901480F591F5093070640930606281BC1
:10843000390B309309062093080680913D01811184
:108440000E94D83980E4E0E5F6E0DF011D928A95CC
:10845000E9F78BEA93E090930401809303018CEA9F
:1084600093E090930601809305018DEA93E0909349
:108470000801809307018EEA93E090930A018093AC
:108480000901E2EDF5E0FA87E98722E735E0388B6C
:108490002F8742E355E05E874D87312C212C832DB9
:1084A0000E9420107C01FC0182810E9424178B878E
:1084B000D7018C918150803108F06AC240E061E0C0
:1084C000F70183810E945517811116C0A985BA85CD
:1084D000DC901C92F701918188EF890F823008F0BF
:1084E00041C287818670843009F43CC2993009F01A
:1084F00047C000E01CEF46C0DD24D394A985BA85AF
:108500008C918111D12C81E0E985FA858083F70176
:1085100021818FEF820FA82FB0E0FD01EE0FFF1F2A
:10852000EE50FA4F00811181843150F0831540F4F0
:10853000AA0FBB1FAA0FBB1FA05BB94F0D911C91C7
:10854000F7013781832F807361F0832F82958370C9
:10855000815041E050E002C0440F551F8A95E2F778
:10856000242A36FF0FC0253068F4E22FF0E0EE0F2A
:10857000FF1FEF5FFE4FC70108969183808302C003
:1085800000E010E0F7018781887459F48085882322
:1085900041F04DE763E80E940B170E944017080F57
:1085A000191FF701F681FB8B2B85332727FD3095AB
:1085B0003A8B298BF11105C0F7018581882309F4D5
:1085C000F0C0AD85BE85AD90BC90EF85F889808107
:1085D0009181A2819C014A2F552747FD5095290181
:1085E0003A01D1100AC0BB2757FDBA95A52F942F89
:1085F000832F6801C81AD90A3EC0F70187818670A7
:108600008430D9F4E081F0E0EE0FFF1FE85EF94F0F
:10861000A081B18120E034E60E940B792B013C015E
:10862000FB85FF2351F02F2F332727FD3095432F54
:10863000532F0E947F7929013A01C301B20120E042
:1086400031E040E050E00E947F79509540953095B0
:1086500021953F4F4F4F5F4F6801C20ED31EC1148B
:10866000D10449F0F7018581D7FE82958F70F4E639
:108670008F9F50011124A114B10491F080913D010C
:10868000882331F021E0A21AB108A114B10441F00D
:10869000332777FC3A95272D162D052DC12CD12C8B
:1086A000AD85BE85AD92BC92C114D10409F474C0ED
:1086B0004801AA2497FCA094BA2CBB89BB2309F4D7
:1086C00067C080913D01882309F443C0EB85EE2308
:1086D000A1F029893A8937FF03C0319521953109E5
:1086E000442737FD4095542F60E070E080E293E02E
:1086F0000E947F79CA01B90104C060E070E080E2A5
:1087000093E0F70126811C141D0444F09095809598
:10871000709561957F4F8F4F9F4F22952F7030E05E
:108720002115310591F0E4E6E29FA001E39F500D91
:1087300011249A01442737FD4095542F0E947F79D8
:10874000420E531E641E751E04C04424582C692C0E
:108750007A2CBB2777FCBA95A72D962D852D1C1456
:108760001D0434F488169906AA06BB0634F009C025
:1087700088159905AA05BB0524F44424582C692CB6
:108780007A2C332777FC3A95272D162D052D04C01A
:108790004424582C692C7A2CAF85B8894D925D926F
:1087A0006C92F701878187FF28C044E66CE98481D9
:1087B0000E940B17A82FBB27A7FDB0951A161B0602
:1087C00044F417FF6AC024E630E02A1B3B0BD901B2
:1087D00009C0109709F461C0101611060CF05DC0B5
:1087E000AC59BF4F98010E94F47824E630E040E095
:1087F00050E00E947F79890150C0F7016481862F83
:10880000992787FD9095A92FB92F8730910590F56D
:10881000FC01EC5AFF4F0C949E79F701818189305D
:1088200021F417FD35C012500BC017FF36C01BC016
:10883000F7018181893039F41016110664F11E5F49
:10884000000F111F2AC0101611066CF026C017FF6A
:1088500024C011950195110920C010161106DCF0F5
:1088600002C017FD15C000E010E017C01016110679
:1088700094F00EC067FF06C0119501951109F6E04E
:10888000F61B6F2F6750C8010E94DF3A8C0105C0AC
:1088900000E01CEF02C000E014E0F701478140FD5A
:1088A00010C081819FEF980F943058F4FE013196EB
:1088B000E80FF11DE80FF11D329780819181080FBB
:1088C000191F9801A989BA890E94F4784B015C01AB
:1088D0004874483051F4F7018085882331F04DE722
:1088E00063E80E940B170E944017D7010C9110E01B
:1088F00001501109F701878186958370000F111FC0
:10890000000F111F813071F0823029F1F801E05B16
:10891000F94F80819181A281B381880E991EAA1E90
:10892000BB1E19C0C501B40124E630E040E050E0B0
:108930000E947F79F801E05BF94F6081718182814B
:1089400093810E94257920E034E040E050E00E94CD
:108950007F7949015A01F801E05BF94F80829182E9
:10896000A282B382339429853A852F5F3F4F3A879D
:1089700029874F8558894D5F5F4F588B4F876D858D
:108980007E856E5F7F4F7E876D8770E2371287CD61
:108990001091410C20FE05C0111103C08EE10E9410
:1089A0000E7221FE07C0812F877F803419F48FE17A
:1089B0000E940E7222FE09C0812F877F803811F03D
:1089C000103919F480E20E940E7288E697E09E87C3
:1089D0008D879D8D9987AE8DAA8737E4232E34E04D
:1089E000332EE0E5F6E0FC87EB87E12CF12CEF86F7
:1089F000AB85BC854D905D906D907C90C301B201BC
:108A000024E630E040E050E00E947F79EB85FC8571
:108A10002193319341935193FC87EB87AD85BE85BC
:108A20002D933D93BE87AD878E2D0E9427104C015C
:108A3000FC01838194812181FAE02F0260011124DD
:108A400028E1C21A2CEFD20AD4012C91BAE02B02F1
:108A500050011124E8EEAE1AE3E0BE0A3C2D2D2DA4
:108A60008C159D0514F4382F292F032F122F0A156A
:108A70001B050CF485014114510461047104A9F033
:108A800077FE04C0D801AA19BB0903C0D601A01BF8
:108A9000B10BA30192010E941D7920EA36E841E062
:108AA00050E00E947F7929013A01C8010E94F51621
:108AB0008C01040D151DC6010E94F5166C01C5013F
:108AC0000E94F516C016D1060CF486010817190786
:108AD0000CF48C01F4018281882319F01195019521
:108AE000110980914504F0E1F81B2F852F17F8F448
:108AF000F701EE0FFF1FEA5BFB4F9081892F880F74
:108B0000880F8595859599F0929596959695937091
:108B10009D5F9370923058F040E060E00E945517DE
:108B2000882329F0D1018C910E9440178C01F89480
:108B3000E985FA8501931193FA87E9877894FFEF25
:108B4000EF1AFF0A22E0220E311C30E1E316F10495
:108B500009F04DCF6E960FB6F894DEBF0FBECDBFB5
:108B6000DF91CF911F910F91FF90EF90DF90CF9009
:108B7000BF90AF909F908F907F906F905F904F903D
:108B80003F902F900895223009F070C98B016EC973
:108B9000FF920F931F93CF93DF93CDB7DEB7C054EF
:108BA000D1090FB6F894DEBF0FBECDBF63E0CE0192
:108BB00081960E946C3D61E0CE0101960E946C3D61
:108BC000E5E2F3E09E012F5D3F4F8E010F5F1F4FE7
:108BD000418152818081882329F0D9018D919C9116
:108BE000D80104C0D8018D919C91D9016D917C91DF
:108BF000861B970B840F951F883EB3E09B073CF4C0
:108C000089314CEF94073CF0482F892F02C048EE81
:108C100083E0942F02C098E18CEF91838283359694
:108C20002E5F3F4F0E5F1F4F83E0E537F80781F659
:108C30000BEA13E0F12C8F2D0E942817811102C03E
:108C4000D8011C92F3940F5F1F4FB4E0FB12F3CFD7
:108C500086E00E94106081E00E940E72C05CDF4FCF
:108C60000FB6F894DEBF0FBECDBFDF91CF911F913D
:108C70000F91FF9008958F929F92AF92BF92CF92E3
:108C8000DF92EF92FF920F931F93CF93DF93C82F42
:108C9000D091F8041D2F1F70D073109255018038A9
:108CA00009F43FC098F4833209F4A3C030F4803251
:108CB00071F1823209F4AAC0F4C0853209F482C08D
:108CC00008F472C0813609F4C4C0EBC0843809F4DA
:108CD00062C058F4823809F4A7C008F4CAC08BEE09
:108CE00092E20E94731483E8A6C08E3809F44AC049
:108CF0008F3B09F4C8C0853809F0D3C081E0809368
:108D0000620789EF9FE40E940B1C85E86FC0133057
:108D100009F0C7C08091AE0791E089278093AE0724
:108D2000AEC0143079F5D03261F48091680D909125
:108D3000690D919581959109909391068093900684
:108D4000B0C0D11114C080916904807C803C21F4B2
:108D50008EEC9DE00E94687480916D04807C803C64
:108D600009F09FC085ED9DE00E9468749AC0D033E1
:108D700049F410925F0D10925E0D10925B0D1092EF
:108D80005A0D8FC081E0809362070E9469140E948F
:108D90000B1C8C2F2BC081E08093620780E297E34D
:108DA0000E940B1C84E822C0123039F48091D8074D
:108DB0008F5F833074F080E00CC0143009F071C014
:108DC00080E10EC0123041F48091D807815087FDB8
:108DD00082E08093D80765C0143009F062C080EF4C
:108DE0008D0F807384608093F80449C00E94BD6930
:108DF00058C01F5F153008F010E0812F8D2B809335
:108E0000F80481E00E94106083E13AC0112311F060
:108E1000115001C014E0812F8D2B8093F80481E064
:108E20000E94106084E12CC0D460D093F80487E1E4
:108E30000E940E7282E8DF91CF911F910F91FF90F7
:108E4000EF90DF90CF90BF90AF909F908F900C9459
:108E5000BD698091A107823021F483E08093A1074E
:108E60000EC0133019F40E94821409C01430C9F4E2
:108E700004C00E94883A0E9482140E94BD7587E156
:108E80000E940E720EC081E00E94BD6983E00E94C4
:108E9000BD6982E00E94BD6981E08093B4071092B1
:108EA000D80740E060E08091DD010E945517C82F8F
:108EB000882331F08091B407811102C00E94C84517
:108EC000C093B407143009F49DC0909102018091C1
:108ED000E504981710F4C6E001C0C4E080E00E94E9
:108EE000D1124C2F406860E185E20E949E1046E559
:108EF00068E186E20E947A658091A1078823A1F04B
:108F0000823011F426E001C024E04091AA0750917C
:108F1000AB07022F60E18DE50E942E1020E040E0BB
:108F200068E183E30E942F1100E02091DB014DE214
:108F300058E060E186E20E949F658091DA0180FF3F
:108F400006C049E258E060E188E30E94D965C0E0CC
:108F5000D0E00FE1C02EFC2EFE01EB5DF74FE49058
:108F60006C2F809131050E94541397FD03969C014C
:108F70003595279535952795243E0CF424EE022F40
:108F80002D310CF00CE18FEF8F0D46E38230E0F4D1
:108F900064E08E2D0E946E668091FA048F2580FD1C
:108FA00004C08091DA0180FD0CC043E06EE18FEFD8
:108FB0008E0D0E946E6643E06EE181E08E0D0E9490
:108FC0006E666C2D601B14C06BE385EE8E0D0E94E7
:108FD0006B66FF24FA94FE0C43E06AE38F2D0E9437
:108FE0006B6643E06CE38F2D0E946B66E00E6BE3D3
:108FF00047E08E2D0E9446222196C430D10509F00B
:10900000AACF29C001E12AE049EC51E060E080E00C
:109010000E947D65909102018091E504981710F4FB
:1090200042E001C040E060E084E50E949E10809133
:10903000A107882309F491C0823011F422E001C015
:1090400020E04091AA075091AB07022F60E08FE625
:109050000E942E1082C0123008F004C3E1E4EE2E0C
:10906000E7E0FE2E00E0F9E1CF2EABE1BA2EF701EA
:10907000C191D1917F01802F8370113041F19E0108
:10908000D7FF02C0215E3F4F75E0359527957A9551
:10909000E1F7AE01421B530B9A01D7FF02C0C15842
:1090A000DF4FAE01440F452F441F550B420F531F96
:1090B000602F66956695660F660F660F685D8B9DDF
:1090C000802D112420E28F5D0E94CA6741C00430C8
:1090D00018F422E2822E02C09EE5892EA82EAA0C48
:1090E000AA0CA80E9E01D7FF04C0222733272C1BF1
:1090F0003D0BC29EA001C39E500D11249A013E5FFC
:10910000932E9594959459E1591514F489E1982E6C
:1091100025E543E366E26A0D87EE880D0E943B6613
:1091200045E064E26A0D882D0E946E661C161D06DD
:1091300014F4839401C0891867E26A0D492D882DC3
:109140000E946B666A2D6B5D492D882D0E946B66AF
:109150000F5F083009F08BCF01C380E00E940374D9
:109160008093B20781E00E9403748093B307D031EB
:1091700009F4BEC1D03209F08FC08091EA0D882376
:1091800069F124E040E160E081E00E949A3A20E049
:1091900048E364E582E00E949A3A4CE158E060E1DD
:1091A0008CE30E94D9654091780D5091790D24E4AB
:1091B00068E08EE40E94CA672091680D3091690DC5
:1091C0008091900690919106280F391FA5E0EA2E14
:1091D00004E446E060E280E00E94CA2080916604D8
:1091E0008823B1F08091B207882311F003E001C019
:1091F00000E068E178E080E30E94D3650464EE2437
:10920000E39420E04091CE0D68E280E10E94E111FC
:1092100080916A048823B9F08091B307882311F004
:1092200003E001C000E044E158E060E380E40E9414
:10923000D9650464EE24E39421E04091D50D68E201
:1092400082E50E94E11167EA72E188E30E94D3653A
:109250004091640D5091650D20E468E382E10E9425
:10926000CA674BEA52E168E380E30E94D965409106
:10927000660D5091670D20E468E382E4DF91CF91A1
:109280001F910F91FF90EF90DF90CF90BF90AF9024
:109290009F908F900C94CA67D03309F0E6C08091FC
:1092A000EA0D811102C0C2E001C0C0E06FE078E0C9
:1092B00080E10E94D3652091940D3091950D442753
:1092C00037FD4095542F6BEFE62EDC2FD0610D2F2C
:1092D00060E180E30E94BA664EE260E180E30E94B2
:1092E0007A652091960D3091970D442737FD409572
:1092F000542F7CEFE72E60E188E40E94BA666AE0B2
:1093000078E088E10E94D36520918E0D30918F0D19
:10931000442737FD4095542FEBEFEE2E68E180E3B4
:109320000E94BA664EE268E180E30E947A6520916D
:10933000900D3091910D442737FD4095542FFCEF4F
:10934000EF2E68E188E40E94BA666CEF77E080E275
:109350000E94D36540915A0D50915B0D60E288E701
:109360000E94D9676EEE77E088E20E94D365C090D4
:109370005E0DD0905F0D8091D50185FF12C069EE22
:1093800077E088E20E94D3658DE492E0A601489FD1
:109390006001499FD00C589FD00C1124CD2CDD24A6
:1093A000C6942C2FA60168E288E70E94CA678091C4
:1093B000EA0D882309F4D2C140916C0D50916D0DD6
:1093C00060E280E30E94D9674091700D5091710D69
:1093D0008091D50185FF0DC08DE492E0FA01E89FF0
:1093E000A001E99F500DF89F500D1124452F5527DE
:1093F000469568E280E30E94D9676DED77E080E3EF
:109400000E94D36561ED77E088E30E94D365C2E4F2
:10941000DDE010E000E3D02E84E2F82E8091410DD3
:10942000181708F09BC1133021F4A8E3DA2EB4E238
:10943000FB2E299180914304281710F000E301C00E
:1094400002E330E0220F331F442737FD4095542FAD
:10945000F4E0EF2E6D2D8F2D0E94BA66FAE2FF0E1A
:10946000153009F47BC11F5FD9CF40E368E08FE37B
:109470000E946E66CAE7D4E010E0F990FF20B1F0D8
:10948000FA948F2D0E94AC1F9C01612F6E70660FA5
:10949000660F660F605F10FF02C080E401C080E0CD
:1094A0007FE0E72E04E04F2D0E94CA201F5F163098
:1094B00021F722E047EA52E168E380E00E94AD65CF
:1094C0000091640D26E041E369E38EE00E940268AA
:1094D00022E04BEA52E168E384E70E94AD65009127
:1094E000660D26E041E369E381E40E94026836C12B
:1094F00046E6842E44E0942E51EDC52E5DE0D52E37
:109500006CE7A62E6DE0B62EC0E0D0E010E0F401CE
:109510008081882309F44FC001E0FE01EE54F84F2A
:109520008081811101C000E04CE852E168E1812FA7
:109530000E94D965FC2E4C2F4F5C68E186E0810FBC
:109540000E947A650464EE24E3942C2FF60133978D
:10955000408160E180E1810F0E94E111FE01EE0F88
:10956000FF1FEE0FFF1FE759FB4F908192959695D5
:109570009695937088E1810F933039F4F50140811D
:10958000518160E20E94D9670AC0EE24E39400E0B2
:109590002C2FF6013197408160E20E94E111EE2408
:1095A000E39400E42F2DF601408160E284E2810F14
:1095B0000E94E11110E42196F4E08F0E911C27E047
:1095C000C20ED11C32E0A30EB11CC230D10509F08D
:1095D0009ECF8091EA0D882369F060E278E088E010
:1095E0000E94D36500917A0D26E046E669E089E1A4
:1095F0000E94026867EA72E180E30E94D3654091AD
:10960000DC0D50E024E468E280E10E94CA674091EA
:10961000DE0D50E068E388E10E94D9674091DF0DDC
:1096200050E020E468E384E20E94CA674BEA52E11A
:1096300060E380E40E94D9654091E30D50E024E4AA
:1096400068E280E50E94CA674091E50D50E068E35A
:1096500088E50E94D9674091E60D50E020E468E378
:1096600084E60CCE123009F06FC00E94332B80913B
:10967000D807882329F0982F990F890F880F8D5FBD
:10968000182FC82FDD27C7FDD0955E0122E0A20E5E
:10969000B11CC12EDD24C7FCD094AC14BD04FCF079
:1096A000FF24F394F10E40E060E08F2D0E945517E7
:1096B000082F0E942C11AC0133E01302400D511D04
:1096C0001124B6016C1B7D0B6C5F7F4F660F660F1C
:1096D000660F23E08AE00E947D651F2DDACF80911E
:1096E000D8078F5F182F110F180F110FC12FDD270B
:1096F000C7FDD0955E0142E0A40EB11CC12EDD2451
:10970000C7FCD094AC14BD044CF1FF24F394F10ECB
:1097100040E060E08F2D0E945517082F0E942C1109
:10972000AC01E3E01E02400D511D1124B6016C1B7B
:109730007D0B6C5F7F4F660F660F660F23E084E63C
:109740000E947D651F2DDACF4091AC075091AD0787
:1097500004E024E068E28CE30E942E10DF91CF91B8
:109760001F910F91FF90EF90DF90CF90BF90AF903F
:109770009F908F900895982F809167071916BCF4D9
:10978000292F332727FD3095281B3109462F50E01C
:10979000421753071CF4892F861B0AC046505109F3
:1097A000241735072CF4892F861B8A5F01C080E0BF
:1097B000809367070895BF92CF92DF92EF92FF9256
:1097C0000F931F93CF93DF93C82E4EE0682F8EEC3C
:1097D00097E00E94F9258091DA07882319F082EE3C
:1097E0009EE002C088ED9EE00E947022182F8091BA
:1097F000DD070E942010EC0120E0488160E086E057
:10980000810F0E94D810D090CE0766E08D2D0E9467
:10981000BB4B18E0F12CBB24B394409167074F0D6C
:10982000EE24E394D412E12C50E04F30510508F0BF
:1098300045C1FA01E55AFF4F0C949E7960ED7EE038
:10984000812F0E94D3652E2D20614981612F84E5EF
:109850000E94A310EE2009F431C14CE261E089813D
:109860000E94591489832AC168EC7EE0812F0E94EE
:10987000D3650DE723E84A81612F80E60E94C0216D
:109880008A831CC18F8186FF03C04EEB5EE002C05D
:1098900047EB5EE0612F8CE00E94D9650DE723E87D
:1098A0004885612F80E60E94C021888707C18F818B
:1098B0002E2D4BEA5EE0612F83FB882780F90E9402
:1098C000802C9F8180FB93F90DC08F812E2D4FE955
:1098D0005EE0612F86FB882780F90E94802C9F81A3
:1098E00080FB96F99F83EAC08F8181702E2D49E914
:1098F0005EE0612F9B2D981B892F0E94802C9B2D51
:10990000981B8F8190FB80F98F83D8C00F8107FB54
:10991000002700F9002319F043E95EE002C04DE89A
:109920005EE02E2D612F8CE00E94B365EE2059F091
:109930008F8187FB882780F961E00E945C149F81FA
:1099400080FB97F99F838F8187FB882780F9081711
:1099500009F4B4C01C82B2C08F8187FF09C004E63D
:109960002CE94C81612F80E60E94C0218C83A6C027
:109970002E2D4C81612F82E10E948C2EEE2009F465
:109980009DC046E160EF8C810E9459148C83873022
:109990000CF494C090E6C91291C087508093DE0702
:1099A0008DE39BE30E940B1C89C065E87EE0812F5C
:1099B0000E94D3650E2D2E2D4B81612F8EE40E94C7
:1099C0007A2E8B837BC06CE77EE0812F0E94D3656B
:1099D0000F810295037049F0402F50E02E2D206436
:1099E000612F84E50E94CA6707C02E2D45E553E02C
:1099F000612F8EE40E94B365EE2009F45FC063E03E
:109A0000802F0E945C1483708295807F9F819F7C51
:109A10001CC064E77EE0812F0E94D3652F812695CC
:109A200023700E2D4AE55EE0612F8EE40E949F6553
:109A3000EE2009F443C08F81869562E083700E9416
:109A40005C148370880F9F81997F982B4BCF4D8139
:109A500042954F702EE43EE06E2D812F0E94AF1E86
:109A60008295807F9D819F700BC04D814F7024E453
:109A70003EE06E2D812F0E94AF1E8F709D81907FE2
:109A8000982B9D831BC04E8142954F7028E33EE08A
:109A90006E2D812F0E94AF1E8295807F9E819F70C8
:109AA0000BC04E814F702EE23EE06E2D812F0E9442
:109AB000AF1E8F709E81907F982B9E83F394185FCA
:109AC00087E0F812AACEDF91CF911F910F91FF90FE
:109AD000EF90DF90CF90BF9008956F927F928F921A
:109AE0009F92AF92BF92CF92DF92EF92FF920F932D
:109AF0001F93CF93DF93C82F8BE591E10E947022D3
:109B000040E1E42E0CE020EA31E146E06C2F85EDE7
:109B100097E00E94E825E090D507EA9466E08E2D54
:109B20000E94BB4BC03611F0C43641F4E7FC06C0BE
:109B3000E092DE078DE39BE30E940B1CA12CB12C6D
:109B4000CC24C39498E0D92EFF24E7FCF09425E0C0
:109B5000922E39E0832EC0916707CA0D0C2F10E0BA
:109B6000D1E0E016F10609F0D0E077247394C83014
:109B700028F4712C87E08C1528F45FC0E6E0EC1522
:109B800008F45BC0B11002C0BD2E02C0BB24B39468
:109B90002D2F48E551E16D2D80E00E94B365A801AD
:109BA0004F5F5F4FC93010F482E101C087E12D2F74
:109BB0006D2D0E94CA67772051F008501109809ED0
:109BC000E001819ED00D1124C952DC4F07C0909E48
:109BD000E001919ED00D1124C155DC4F8E018AE227
:109BE000682EF80141918F01552747FD50956D2D45
:109BF000862D0E94D967F5E16F0E83E96812F1CFD7
:109C000008E00D0D711002C0C39411C025961AE230
:109C10004991552747FD5095602F812F0E94D967A4
:109C20001B5E1E37A9F700E10D0DC394C394A394E6
:109C3000E7E0AE1611F0D02E8ECFB11005C08091A6
:109C400067078F5F80936707DF91CF911F910F9117
:109C5000FF90EF90DF90CF90BF90AF909F908F904C
:109C60007F906F9008952F923F924F925F926F92E4
:109C70007F928F929F92AF92BF92CF92DF92EF929C
:109C8000FF920F931F93CF93DF9300D000D0CDB7F7
:109C9000DEB7282E88EA9DE00E947022809110078E
:109CA000882321F00E94AA2F182F01C010E0809174
:109CB0003F0781110BC0E0903E070CE020EA31E144
:109CC00044E0622D8DEC97E00E94E8256090CD077E
:109CD0008091AB01803621F08F3B31F08E32A1F4C0
:109CE00090911007992319F0109210070DC09091D0
:109CF0003F07911109C00E94BD691092AB0161102C
:109D000007C01092100702C06620D9F3198202C062
:109D100081E0898367E0862D0E94BB4B382E8091BD
:109D20003F0781111092AB0180911007882369F0E1
:109D300011160CF456C1111156C18091AB01823637
:109D400009F44FC1833609F44EC14424439411E011
:109D5000512CA32CB12C852D0E9420107C01311692
:109D600078F4612F70E06A197B096830710544F45A
:109D7000660F660F660F20E0442D81E00E94D81028
:109D80009FE1951508F4C8C0F701F081FA83F4113A
:109D9000C3C0C7010A969C838B83F52CCB80DC80E3
:109DA0009AE0C91AD108311608F0A3C0812F90E0BB
:109DB0008A199B09883091050CF08CC0782E770C9D
:109DC000770C770C80911007811113C0611211C0BC
:109DD000F092DD07EA81E093DB07F981FF2359F078
:109DE0001092110781E080933F07EE24E394212C29
:109DF00004C0E12C02C0EE24E3945F1459F0F60194
:109E000027812695237000E043EA5DE0672D83E11A
:109E10000E949F6520E1EB81FC8139974081672D8D
:109E200080E30E94A3100DE723E88B809C80F8E07C
:109E30008F1A9108F4014081672D8DE20E94C021A4
:109E4000F4018083EB81FC8137974081442329F022
:109E500020E0672D88E40E94FA10EB81FC813697A0
:109E60004081442379F0F601878120E087FF06C016
:109E700044E6672D80E60E94C86404C0672D80E632
:109E80000E948C2EF6018681811102C040E201C041
:109E900043E5F6018581882329F0433511F44AE230
:109EA00001C044E4672D89E70E947A65809110071C
:109EB0008823F9F08091DC078F111BC020E046E673
:109EC000672D88E10E940166F092DD071093CD07AF
:109ED000612E0FC0089769F480911007882349F01C
:109EE0008091DC078F1105C08091CD078F5F809333
:109EF000CD071F5FF394F0E2FF1609F448C08B8191
:109F00009C810A969C838B83FC013A9780819A817D
:109F1000891709F443CF3BC0611237C04092DB0779
:109F20005092DD07662D6A19660F660F660F615045
:109F300029E049E180E00E94DC67E981EE2329F114
:109F40000E94EE2E811121C060E08091DD070E9409
:109F5000E01E109210078BED9BE40F900F900F9076
:109F60000F90DF91CF911F910F91FF90EF90DF90B5
:109F7000CF90BF90AF909F908F907F906F905F90A9
:109F80004F903F902F900C940B1C1F5FF52C439427
:109F9000F1E14F1611F05F2CDECE80913F07882350
:109FA00031F02092AB010E94FC2F109266071150F5
:109FB00010933E070F900F900F900F90DF91CF916D
:109FC0001F910F91FF90EF90DF90CF90BF90AF90D7
:109FD0009F908F907F906F905F904F903F902F90C9
:109FE000089561E001C060E08091DD070E94AA2E23
:109FF000ACCE6F927F929F92BF92CF92DF92EF9200
:10A00000FF920F931F93CF93DF93D82E86E89AE0A9
:10A010000E947022FFE1EF2E06E024E931E140E0EA
:10A020006D2D8BEB97E00E94E8251091BB07E09027
:10A03000400767E0812F0E94BB4BF82E88E1F812A1
:10A0400008C01B3110F48FEF01C081E0E8E1FE2E63
:10A05000F80E91E6D916B1F09D1558F084E4D816A3
:10A0600061F18D1520F092E4D916E0F541C085E448
:10A0700006C094E6D91609F1D916A0F185E6D816DE
:10A0800059F036C080916607882391F110926607D7
:10A0900081E60E94BD692CC0113039F4EE2041F1F7
:10A0A00080916607882321F104C0163109F5EE205E
:10A0B000F9F08091400781500CC0113069F498E0AC
:10A0C0009E15B0F080916607882391F0809140073B
:10A0D0008F5F809340070CC0163151F486E08E15D7
:10A0E00038F0F4CF80916607811102C010924007CA
:10A0F000F1107EC06BE77AE088E00E94D3651130F2
:10A1000031F480916607811102C001E101C000E1D4
:10A110002AE047E055E068E082E40E947D65809196
:10A12000660781110BC08091630787FF07C081E03C
:10A13000809366071092630710924007809166072C
:10A14000882381F020916307332727FD30958E2DDA
:10A1500090E08217930734F4109266071092630719
:10A1600010924007113009F091C48091660788234E
:10A1700009F48CC48091400790916307891B87FD87
:10A1800003C08093400702C01092400780914007AF
:10A190008A301CF089E08093400710926307CE2D2F
:10A1A000D0E0CA54DB4FFE01EF5AFF4F80810E947E
:10A1B00086352091400130914101232B29F49D2DBA
:10A1C0009F7D9254923018F461E40E9464140E94BE
:10A1D0009835CF5ADF4F88839E2D990F9E0D990F8A
:10A1E00021E0482F68E082E4890F0E94C8644EC4D1
:10A1F00091E09F1548F1D8E0C091F904C695C69545
:10A20000C695C77064E77AE08D2F0E94D36512303F
:10A2100089F466E08C2F0E946414C82F8770880F21
:10A22000880F880F9091F904977C982B9093F904EC
:10A2300001E001C000E02C2F48E45AE06D2F8CE5CE
:10A240000E949F65D85F04C082E0F8121DC0D8E06C
:10A25000C09105056DE37AE08D2F0E94D365133020
:10A2600049F463E08C2F0E946414C82F8093050585
:10A2700001E001C000E02C2F43E15AE06D2F82E4A1
:10A280000E949F65D85F04C093E0F91231C0D8E006
:10A29000C0911205C95F6CE07AE08D2F0E94D365F2
:10A2A000143039F467E08C2F0E946414C82F21E425
:10A2B00001C020E44C2F50E06D2F86E60E94CA6753
:10A2C00040911205552747FD50952C2F332727FD28
:10A2D0003095275031094217530729F0C750C093D2
:10A2E00012050E94A714C8E0CD0FC93328F0D0C3CF
:10A2F00084E0F8121EC0C8E06DEF79E08C2F0E9458
:10A30000D365153051F444E661E0809103050E9465
:10A3100061148093030521E401C020E4409103050A
:10A3200050E06C2F86E60E94CA67C85FC93328F0E8
:10A33000AFC395E0F9121DC0C8E06CEE79E08C2F38
:10A340000E94D365163049F465E0809104050E94AF
:10A3500064148093040521E401C020E440910405C5
:10A3600050E06C2F86E60E94CA67C85FC93328F0A8
:10A370008FC386E0F81220C0C8E063EE79E08C2F2E
:10A380000E94D365173061F44DE26AE08091E404E5
:10A390000E9461148093E4040E948A6821E401C051
:10A3A00020E44091E40450E06C2F86E60E94CA67E6
:10A3B000C85FC93328F06CC397E0F9121DC0C8E02C
:10A3C00063ED79E08C2F0E94D365183051F448E793
:10A3D00068E28091E5040E9461148093E50421E421
:10A3E00001C020E44091E5046C2F86E60E948810AD
:10A3F000C85FC93328F04CC388E0F81222C0C8E017
:10A4000060EC79E08C2F0E94D365193051F44EE650
:10A4100066EF8091FB040E9461148093FB0421E0AD
:10A4200001C020E04091FB04552747FD5095465F51
:10A430005F4F6C2F80E70E94CA67C85FC93328F05E
:10A4400027C399E0F91217C0C8E021E01A3009F0DB
:10A4500020E08091FC044FEA59E06C2F81700E944B
:10A46000602C9091FC0480FB90F99093FC04C85FF1
:10A47000C93328F00DC38AE0F81218C0C8E021E003
:10A480001B3009F020E08091FC0443EA59E06C2F76
:10A49000869581700E94602C9091FC0480FB91F95C
:10A4A0009093FC04C85FC93328F0F2C29BE0F91214
:10A4B00019C0C8E021E01C3009F020E08091FC04C4
:10A4C00044E959E06C2F82FB882780F90E94602CB8
:10A4D0009091FC0480FB92F99093FC04C85FC9330F
:10A4E00028F0D6C28CE0F81219C0C8E021E01D3077
:10A4F00009F020E08091FC0446E859E06C2F83FBD2
:10A50000882780F90E94602C9091FC0480FB93F9CD
:10A510009093FC04C85FC93328F0BAC29DE0F912D9
:10A520001DC0C8E069E779E08C2F0E94D3651E301A
:10A5300051F446E16AEE8091E7040E946114809331
:10A54000E70421E001C020E04091E7046C2F80E6A1
:10A550000E94FA10C85FC93350F09AC28EE0F81614
:10A5600029F0D8E000E070E1B72E4CC0C8E021E04F
:10A570001F3009F020E08091020548E659E06C2F79
:10A5800086FB882780F90E94602C9091020580FB51
:10A5900096F990930205D8E0DC0FD93318F378C20E
:10A5A000011133C068E579E08D2F0E94D365011158
:10A5B0002FC0C091FE041B112EC068E78C2F0E9493
:10A5C0006414C82F21E0CC2341F1206495E0C99F99
:10A5D000A00111246D2F86E60E94CA6743E76D2F04
:10A5E0008091400C0E947A6501111EC0C093FE0448
:10A5F000D85FD93308F04CC281E08B0D0F5F8231F8
:10A60000B1F0B82EFB14C0F7CBCF68E479E0CCCF23
:10A61000C0910605D0CF20E0D6CF45E553E06D2FA1
:10A6200086E60E94B365E0CFC0930605E1CF81E1E5
:10A630008F15E0F021E0123109F020E08091FC0458
:10A6400082958170C1E04AE359E06D2F9C2F981BE1
:10A65000892F0E94602CC81B8091FC04C0FB84F9E8
:10A660008093FC04D85FD93308F012C282E08B0DCE
:10A67000F816D8F421E0181320E0809102058295A5
:10A680008170C1E04EE259E06D2F9C2F981B892FFD
:10A690000E94602CC81B80910205C0FB84F9809346
:10A6A0000205D85FD93308F0F3C183E08B0DF816AB
:10A6B000D0F421E0181320E08091F9048170C1E00A
:10A6C0004DE159E06D2F9C2F981B892F0E94602C23
:10A6D000C81B8091F904C0FB80F98093F904D85F0E
:10A6E000D93308F0D5C184E08B0DF816D8F421E0F9
:10A6F000181320E08091F90486958170C1E04DE93E
:10A7000053E16D2F9C2F981B892F0E94602CC81B32
:10A710008091F904C0FB81F98093F904D85FD933A3
:10A7200008F0B6C165E0C62ECB0CFC1408F079C069
:10A7300062E179E08D2F0E94D3655EE9652E52E1DA
:10A74000752EC2E49924939480911105892101E02A
:10A7500009F400E021E0A3016D2F8C2F0E947D659C
:10A76000990CCA5F8FEF681A780AC23769F71C1113
:10A7700054C08091400790916307891B87FD03C0F7
:10A780008093400702C010924007809140078A30B2
:10A790001CF089E080934007109263074E2D50E033
:10A7A00042565D4E8E2D880F8E0D880F02E021E0FF
:10A7B0006D2F8E5B0E947D6590E6D91649F08EE67E
:10A7C000D81631F08091400190914101892B29F1F7
:10A7D0008D2D0E94BD691092660721E030E002C015
:10A7E000220F331FEA94E2F7409111054227C90175
:10A7F00088739927892B19F44093110509C0842F78
:10A80000822319F0276C242301C0242B20931105E7
:10A8100081E00E9410600E94AF60D85FD93308F0D9
:10A8200037C186E08B0DF816E0F421E0181320E024
:10A830008091F90482FB882780F9C1E043E059E068
:10A840006D2F9C2F981B892F0E94602CC81B809114
:10A85000F904C0FB82F98093F904D85FD93308F07A
:10A8600017C187E08B0DF816E0F421E0181320E003
:10A870008091F90487FB882780F9C1E045EF58E013
:10A880006D2F9C2F981B892F0E94602CC81B8091D4
:10A89000F904C0FB87F98093F904D85FD93308F035
:10A8A000F7C088E08B0DF816E0F421E0181320E0E3
:10A8B0008091FC0485FB882780F9C1E04BEE58E0CD
:10A8C0006D2F9C2F981B892F0E94602CC81B809194
:10A8D000FC04C0FB85F98093FC04D85FD93308F0F1
:10A8E000D7C089E08B0DF816B8F421E0181320E0EA
:10A8F0008091020587FB882780F94FED58E06D2F86
:10A900000E94602C9091020580FB97F990930205BC
:10A91000D85FD93308F0BCC08AE08B0DF816E0F49C
:10A9200021E0181320E08091FC0486FB882780F941
:10A93000C1E047ED58E06D2F9C2F981B892F0E9496
:10A94000602CC81B8091FC04C0FB86F98093FC043A
:10A95000D85FD93308F09CC08BE08B0DF816B8F4A3
:10A9600021E0181320E08091020549EC58E06D2F9A
:10A9700085FB882780F90E94602C9091020580FB5E
:10A9800095F990930205D85FD93308F081C08CE027
:10A990008B0DF816A8F421E0181320E0809116051D
:10A9A0004FEB58E06D2F81700E94602C909116053E
:10A9B00080FB90F990931605D85FD93308F068C0F2
:10A9C0008DE08B0DF816E0F4C091FC04C7FBCC279A
:10A9D000C0F921E0181320E04EEA58E06D2F8C2FCB
:10A9E0000E94602C9091FC0480FB97F99093FC04EA
:10A9F0008170C8130E94E876D85FD93308F048C048
:10AA00008EE0B80EFB1408F043C049EA58E06D2F01
:10AA100086E00E94D965D83328F008E00D0F09338D
:10AA200078F036C004E2C0E02C2F48EB51E16D2FE6
:10AA3000802F0E948364CF5F085EC430A9F7EDCFFA
:10AA40001B110DC080916607882359F063E0809147
:10AA5000FA040E9464148093FA0422E003C020E008
:10AA600001C021E04091FA044F5C602F82E10E9416
:10AA7000C864D4E2C0E0CF5F20E04C2F602F8D2F60
:10AA80000E94A310D85EC430B1F702C0D0E1B4CBAD
:10AA9000DF91CF911F910F91FF90EF90DF90CF90BA
:10AAA000BF909F907F906F9008958F929F92AF92EA
:10AAB000BF92CF92DF92EF92FF920F931F93CF93AB
:10AAC000DF93C82F89EA9FE00E9470229CE0A92EA4
:10AAD000CC24C39427EAE22E2FE0F22E0CE020EAE9
:10AAE00031E147E06C2F8FEC97E00E948F23C090FC
:10AAF000CF07CA94F090400766E08C2D0E94BB4BB4
:10AB0000A82E18E0DD24C7FCD0942A2D30E0C21610
:10AB1000D30639F480916607882329F082E0B82EA5
:10AB200004C0B12C02C0BB24B394E901CC0FDD1FDB
:10AB3000C20FD31FC15EDB4F64EA7FE0812F0E940A
:10AB4000D36588E08A1510F448E301C041E34A0D5B
:10AB5000612F8CE00E947A65FF2011F000E001C0B7
:10AB60000B2D2A812F7049E35FE0612F83E10E9462
:10AB70009F658A818F700E941210982E81E091103B
:10AB80002EC0F81611F020E001C02B2D4881612F56
:10AB90008DE30E94A31088818532B4F0BBED8B2E2B
:10ABA000880E6981882D0E94511F9C0182E0F81651
:10ABB00011F000E001C00B2DA2E0EA2E482D612F1C
:10ABC0008AE60E94CA2062C082E0F81611F020E0F6
:10ABD00001C02B2D4981552747FD509553C0981230
:10ABE00016C0F81611F020E001C02B2D4881612F0E
:10ABF0008DE30E94FA1082E0F81611F020E001C007
:10AC00002B2D4981612F84E50E94FA103FC082E01C
:10AC1000981217C081E0F81611F020E001C02B2D2A
:10AC20004881612F8DE30E94A31082E0F81611F095
:10AC300020E001C02B2D4981612F87E50E94A310E0
:10AC400025C065E37FE0812F0E94D36581E0F8167F
:10AC500011F020E001C02B2D4881552747FD50956C
:10AC60004F5F5F4F612F8FE40E94CA6782E0F81642
:10AC700011F020E001C02B2D4981552747FD50954B
:10AC80004F5F5F4F612F8CE60E94CA674A814295F1
:10AC90004F7049300CF04F5F83E0F81203C02B2D4A
:10ACA000286001C028E0612F89E60E94FA10809197
:10ACB0006607811107C08091400190914101892B65
:10ACC00009F465C0BB2009F462C081E0F81639F1CF
:10ACD000F816A0F082E0F81609F43EC083E0F812FE
:10ACE00056C08A816FE082958F700E945C148295B5
:10ACF000807F9A819F70982B9A8349C08A816EE0E9
:10AD00008F700E945C148F709A81907F982B9A8329
:10AD10000E9412109816D9F11882198238C081E069
:10AD2000981661F0981640F082E0981651F083E092
:10AD300098122DC063E60BC065E409C046E16AEED7
:10AD400002C045E460E088810E94591403C08881F4
:10AD50000E945C1488831BC081E0981669F09816E5
:10AD600040F082E0981671F083E0981210C063E61C
:10AD70000AC04DE763E802C046E16AEE89810E949D
:10AD8000591404C065E489810E945C148983A394EA
:10AD9000185F103409F0B9CEDF91CF911F910F9158
:10ADA000FF90EF90DF90CF90BF90AF909F908F90EB
:10ADB0000895AF92BF92CF92DF92EF92FF920F93DE
:10ADC0001F93CF93DF93B82E8DE19DE00E947022F8
:10ADD00063E1A62E7DE0C72EEFE0EE2EEDE0FE2E25
:10ADE0000CE020EA31E141E06B2D85EC97E00E9418
:10ADF0008F231091C507D090400767E0812F0E94F4
:10AE0000BB4BC82F2091E30430E02F5F3F4F442716
:10AE100037FD4095542FF2E0EF2E01E160E08AE229
:10AE20000E94BA66C1113BC06AE07DE088E00E94E2
:10AE3000D36500E12AE049EC51E068E082E40E9439
:10AE40007D65113009F0AEC329E040E467E08AE394
:10AE50000E94DC678D2D880F8D0D880F209166076D
:10AE600046E068E0845C0E94016680916607882362
:10AE700009F498C3CD2DD0E0C753DE4F88810E94DE
:10AE8000863561E40E945C140E9498359881981779
:10AE900009F488C3888382E00E94106083C3C230B3
:10AEA00020F5C8E069EF7CE08C2F0E94D36512305A
:10AEB00081F420E6B21204C08091D3010E949F1455
:10AEC00061E38091D3010E945C148093D30121E05F
:10AED00001C020E04091D30150E04C5F5E4F6C2FE9
:10AEE00088E50E94CA67C85F03C0C23091F4C8E019
:10AEF00066E872E18C2F0E94D365133009F0B1C36C
:10AF000081E0D81251C3809166078111ACC301E082
:10AF1000ABC3C330D1F4C8E061EF7CE08C2F0E945A
:10AF2000D365143051F449E367EC8091D4010E9459
:10AF300059148093D40141E001C040E021E06C2F1E
:10AF40008CE30E942F11C85F03C0C430E1F4C8E055
:10AF500068EE7CE08C2F0E94D365153051F445E1FA
:10AF60006BEE809144040E9459148093440441E0A4
:10AF700001C040E022E06C2F8CE30E942F11C85FDB
:10AF8000C93320F073C3C53021F5C8E066E872E12B
:10AF90008C2F0E94D365163071F48091D50161E049
:10AFA00081700E945C149091D50180FB90F9909380
:10AFB000D50101E001C000E02091D501217042EDF2
:10AFC0005CE06C2F8CE30E949F65C85FC93320F062
:10AFD0004DC3C630B9F4C8E021E0173009F020E0D5
:10AFE0008091DA014BEC5CE06C2F81700E94802C28
:10AFF0009091DA0180FB90F99093DA01C85FC93330
:10B0000020F034C3C730C1F4C8E021E0183009F0A3
:10B0100020E08091DA0144EC5CE06C2F8295817035
:10B020000E94802C9091DA0180FB94F99093DA01D0
:10B03000C85FC93318F01AC3C830E9F46BEB7CE081
:10B040008C2F0E94D365193049F464E08091DB01B4
:10B050000E945C148093DB0101E001C000E02091BC
:10B06000DB014BE95CE06C2F8CE30E949F65C85FBD
:10B07000C93320F0FBC2C930D1F4C8E063E97CE0F9
:10B080008C2F0E94D36521E01A3009F020E0022FB6
:10B090004091DD016C2F86E30E947A2E8093DD01C2
:10B0A00058E0E52EEC0E88E38E1530F4DFC2CA308E
:10B0B00009F050C048E0E42E6AE87CE08E2D0E9442
:10B0C000D3653CE3C32EC0E0D0E0DC1202C01B30ED
:10B0D00061F02091DE0130E00C2E02C035952795FD
:10B0E0000A94E2F7022F017001C002E0AE014E5750
:10B0F000534F21E06E2D8C2D0E947D65219626E018
:10B10000C20E86E6C812E1CF1B30F9F420E6B21673
:10B1100031F02091400130914101232BB1F08B2D72
:10B120000E94BD691092660721E030E00D2C01C03D
:10B13000220F0A94EAF78091DE0182278093DE01D4
:10B1400082E00E9410600E94AF60C8E0CE0DC9335B
:10B1500028F08CC2CB3009F0DAC0C8E06CE77CE0A4
:10B160008C2F0E94D3651C3041F4D11006C0809111
:10B170006607882321F002E003C000E001C001E07F
:10B180004091D80186E0489FA0011124435A534FB3
:10B1900026E06C2F84E20E947D658091D80188238F
:10B1A00059F09DEF980F9230F0F563E57CE08C2F1D
:10B1B0000E94D365D8E406C067E57CE08C2F0E942E
:10B1C000D365DCE31C3049F421E0D21206C0809143
:10B1D0006607882321F002E003C000E001C001E01F
:10B1E0002091D9012E5F45E35CE06C2F8D2F0E94EA
:10B1F0009F651C3049F482E0D81206C08091660732
:10B20000882321F022E003C020E001C021E040912A
:10B21000DC0182E34802A0011124445D5E4F6C2FE3
:10B2200088E28D0F1EC08130F1F46EE27CE08C2F3D
:10B230000E94D3651C3049F421E0D21206C08091EF
:10B240006607882321F022E003C020E001C021E04E
:10B250004091D901552747FD50954F5F5F4F6C2FA7
:10B260008EE70E94CA671C3009F04DC080916607C6
:10B27000811107C02091400130914101232B09F435
:10B2800042C0D091D8018091020585FF02C064E0E0
:10B2900001C063E081E0D81661F0D81620F022E00A
:10B2A000D216F1F02BC08D2F0E945C148093D80130
:10B2B00025C0DD2321F08DEF8D0F823038F444E07E
:10B2C0006EEF8091D9010E94591407C0D130B1F4BA
:10B2D0006CE78091D9010E945C148093D9010EC063
:10B2E000DD2321F08DEF8D0F823040F44AE06CEFCA
:10B2F0008091DC010E9459148093DC018091D80177
:10B300008D131092D901C85FC93328F0AFC1CC307A
:10B3100009F077C0C8E08091D801882321F09DEF23
:10B32000980F923010F56FE17CE08C2F0E94D3656E
:10B330001D3011F421E201C020E24091E20185E0DC
:10B340004802A00111244F515F4F6C2F8CE40E94E2
:10B35000CA671D3009F051C044E16CEE8091E201F2
:10B360000E9459148093E20148C08130B9F4D1E0C1
:10B370001D3009F0D0E02D2F49E05CE06C2F80E01B
:10B380000E94B365DD23C9F120E8B21236C081E026
:10B3900080937B0C80E00E940E722FC060E07CE006
:10B3A0008C2F0E94D3654091D90147FD04C04330E2
:10B3B0001CF042E001C040E04093D9011D3031F45F
:10B3C00080916607882321F002E003C000E001C0FD
:10B3D00001E089E04802A00111244C51544F29E0BA
:10B3E0006C2F8CE30E947D651D3039F462E0809102
:10B3F000D9010E945C148093D901C85FC93320F041
:10B4000035C1CD3051F5C8E067ED7BE08C2F0E944F
:10B41000D3651E3099F48091DA0167E082958695B4
:10B4200087700E945C148295880F807E9091DA016B
:10B430009F71982B9093DA0121E001C020E04091A8
:10B44000DA014295469547704F5C6C2F82E70E9467
:10B45000C864C85FC93320F009C1CE3021F5C8E007
:10B460006DEC7BE08C2F0E94D3651F3071F48091CE
:10B47000DF0161E081700E945C149091DF0180FB2C
:10B4800090F99093DF0101E001C000E02091DF011D
:10B49000217045EC5BE06C2F8CE30E949F65C85FD8
:10B4A000C93320F0E3C0CF30C1F4C8E021E010314F
:10B4B00009F020E08091DF014BEB5BE06C2F86957B
:10B4C00081700E94802C9091DF0180FB91F9909314
:10B4D000DF01C85FC93320F0C9C0C031C1F4C8E082
:10B4E00021E0113109F020E08091D50143EB5BE0D0
:10B4F0006C2F869581700E94802C9091D50180FBE5
:10B5000091F99093D501C85FC93320F0AFC0C13124
:10B51000D1F4C8E021E0123109F020E08091D5019A
:10B520004AEA5BE06C2F82FB882780F90E94802C1E
:10B530009091D50180FB92F99093D50168E06C0F52
:10B54000693328F093C0C23109F090C068E080915F
:10B550006407811103C021E0133109F020E046E9BE
:10B560005BE080E00E94B365133109F07FC020E802
:10B57000B2127CC01092660789E18093640780E86C
:10B580000E94BD6910920F0785E29FE2DF91CF9183
:10B590001F910F91FF90EF90DF90CF90BF90AF90F1
:10B5A0000C940B1CC0E17ECCD1105BC0809166076F
:10B5B00000E0882311F022E001C021E04091D60193
:10B5C0005091D7016C2F87E40E942E10133009F0A0
:10B5D00046C080916607811106C0209140013091DC
:10B5E0004101232BE1F16CE370E08091D601909151
:10B5F000D7010E944979962FD82FDD2021F021E034
:10B60000D21691F02CC06BE3892F0E945C142CE3BE
:10B610008202C00111248D0F911DD7FD9A95909340
:10B62000D7018093D6011BC04EE361E082E08D0F0D
:10B630000E945914D81BDE5F2091D6013091D701AA
:10B640002D1B3109D7FD339537FD05C03093D70148
:10B650002093D60104C01092D7011092D601C85F82
:10B660005BCC00E001C002E020E0A8CFDF91CF91E9
:10B670001F910F91FF90EF90DF90CF90BF90AF9010
:10B6800008955F926F927F928F929F92AF92BF9236
:10B69000CF92DF92EF92FF920F931F93CF93DF939E
:10B6A000D82E81E591E10E94702271E1A72ECC2471
:10B6B000C394EFE4EE2EE1E1FE2E0CE020EA31E14E
:10B6C00045E06D2D84ED97E00E948F23C090D40754
:10B6D000CA94B090400766E08C2D0E94BB4B982E18
:10B6E00080E8D81227C09FE09C1520F14C2D5527EB
:10B6F00047FD5095FA01E919F109EE0FFF1FEF5BC5
:10B70000F84F20813181B11015C085E0849FF00190
:10B71000859FF00D1124ED5DFC4F8281882319F087
:10B720003195219531093483238382E00E94106092
:10B730000E94AF6048E0A42EEC2CFF24E7FCF094BC
:10B7400080E1981609F4BEC0892D0E942710EC01F3
:10B75000092D10E0F801EE0FFF1FEF5BF84F20817D
:10B7600031818A81EB81FC81882319F0F195E19583
:10B77000F1092E1B3F0B233331051CF081110AC048
:10B780009EC02E3C3F4F1CF4882321F098C02DE230
:10B79000822E02C09FE7892E939420E0492D6A2DC6
:10B7A00080E00E94D810482D6A2D8BE40E947A65B3
:10B7B0008091DF0181FF03C08DE7682E02C0B4E6EF
:10B7C0006B2E812C562C5194E016F10641F4B810E2
:10B7D00006C080916607811105C021E004C020E009
:10B7E000712C09C022E0809165078823C9F3772472
:10B7F00073941092550182E0881691F193E08916B6
:10B8000009F443C081E08816B1F020624B815C816D
:10B810006A2D80E30E94CA67772009F446C022E0BF
:10B8200048EE53E068E17CEF8B819C810E949A1383
:10B830009C838B833AC048814456552747FD5095D9
:10B840006A2D88E40E94CA67772079F1888184563E
:10B85000888349E1652D0E9459148C59888325C03D
:10B8600049814C59552747FD50956A2D86E60E941F
:10B87000CA677720D1F089818C598983462D67EE7C
:10B880000E9459148456898310C04A816A2D8CE61F
:10B890000E948323772049F061E08A810E945C1432
:10B8A00091E0811101C090E09A83839494E0891221
:10B8B0008BCF88E08A0D803491F1A82E41CFAEE77E
:10B8C0008A2E6ACFC1E090E1C912C0E0809164077E
:10B8D000811123C02C2F4EE351E16A2D82E10E9499
:10B8E000B365CC23E1F080E8D81219C089E18093D8
:10B8F000640780E80E94BD69DF91CF911F910F918D
:10B90000FF90EF90DF90CF90BF90AF909F908F907F
:10B910007F906F905F900C94C84520E0DCCFDF9162
:10B92000CF911F910F91FF90EF90DF90CF90BF903C
:10B93000AF909F908F907F906F905F9008956F92DF
:10B940007F928F929F92AF92BF92CF92DF92EF92AF
:10B95000FF920F931F93CF93DF93C82F82E190E163
:10B960000E947022D1E1AD2E12E0C12E0FE0E02E38
:10B9700000E1F02E0CE020EA31E148E06C2F80ED90
:10B9800097E00E948F23A090D007AA949090400740
:10B9900066E08A2D0E94BB4BB82E18E0CA2CDD242D
:10B9A000C7FCD094B11020C06FEF7FE0812F0E94C0
:10B9B000D365A1100FC080916607882311F0C2E003
:10B9C00001C0C1E060E1809145040E945C14809355
:10B9D000450401C0C0E04091450450E02C2F612F88
:10B9E0008CE60E94CA6759C180E18B1508F455C1E5
:10B9F00000E180914504081BEB2CF12CE701CC0FF2
:10BA0000DD1FCC5BDB4F20E04B2D612F80E00E94DF
:10BA1000D8100B1508F4C3C0812CCE14DF0441F4F8
:10BA2000981006C080916607811105C001E004C02E
:10BA300000E0712C07C002E0809165078823C9F3FC
:10BA4000772473948881811021C0807C803421F018
:10BA5000803821F446E503C041E401C043E5202FCE
:10BA6000612F8EE10E94C864772009F493C0888119
:10BA700062E082958695869583700E945C1482951B
:10BA8000880F880F807C98819F7330C091E0891265
:10BA900030C0982F907C903819F0A6E16A2E02C031
:10BAA000F9E16F2E482F440F440F459545954731D6
:10BAB0004CF029EE240F48EE5FE0612F8AE20E94ED
:10BAC0009F6505C0202F612F8AE20E94FA1077201F
:10BAD00009F460C08881880F880F462D6AEE85952D
:10BAE00085950E9459148F739881907C982B988328
:10BAF00051C0982F907C4981903491F447FD03C048
:10BB00004F3024F401C040E0242F01C02FE02983EE
:10BB100044E252E1612F80E60E949F654FE017C02A
:10BB2000903841F5880F880F89359CF047FD04C097
:10BB300040321CF040E201C040E0498321E0240F84
:10BB400043E153E1612F80E60E949F6540E260E09F
:10BB50001BC04F360CF04FE64983552747FD5095E3
:10BB600040585F4F202F612F80E60E94CA674FE642
:10BB700060E80AC0552747FD5095202F612F80E6C9
:10BB80000E94CA674DE763E8772021F089810E940F
:10BB900059148983839483E088123FCF7EC065EE79
:10BBA0007FE0812F0E94D365812CCE14DF0441F405
:10BBB000981006C080916607811105C001E004C09D
:10BBC00000E0712C07C002E0809165078823C9F36B
:10BBD000772473948881811013C0482F4F71202FD0
:10BBE000612F8EE10E94FA10772009F452C08881FB
:10BBF00065E18F710E945C148F719881907E1BC0EB
:10BC000091E089121BC0282F22952695277049EBB9
:10BC10005FE0612F8CE30E949F657720D1F18881DE
:10BC200066E08295869587700E945C148295880FE5
:10BC3000807E98819F71982B98832BC082958695E2
:10BC4000877090E04981069774F0403208F040E236
:10BC5000498321E0240F43E153E1612F80E60E94F4
:10BC60009F6540E20BC04A3F08F04AEF498350E02D
:10BC7000202F612F86E60E94CA674AEF772049F09D
:10BC800050E0898122E060E070E090E00E949A1329
:10BC90008983839483E0881288CFB394185F10342B
:10BCA00009F080CEDF91CF911F910F91FF90EF901F
:10BCB000DF90CF90BF90AF909F908F907F906F90CC
:10BCC00008951F93CF93DF93EC011AE088810E94BF
:10BCD00086350E94983589931150C1F7DF91CF9135
:10BCE0001F910895E7EBF4E080E090E0219131911D
:10BCF000820F931F24E0EF3CF207C1F7089581E61D
:10BD0000E6EBF4E0DF011D928A95E9F78AE0809383
:10BD1000B60489E18093E4048AE58093E50481E038
:10BD20008093FA04E7EBF4E020E032E080E891E071
:10BD30002193319395878487938F828FB4E0E53C7C
:10BD4000FB07B1F74AE050E068EE73E187E095E069
:10BD50000E94A4790E94725E9093E2048093E104B1
:10BD60000895CF93C82F2DEE32E0E9ECF1E0DF012A
:10BD7000C9011D920197E9F74AE050E06DED73E1CA
:10BD8000CF010E94A4798C2F90E06AE070E00196C8
:10BD90000E944979605D6093CE01805D8093CF0100
:10BDA00080E0CF910C948C6A0F931F93CF93DF9315
:10BDB000EB01042F803138F561E0680F83EF97E0E5
:10BDC0000E94296210E0A80160E270E0CE010E94AA
:10BDD000C5794AE050E0BE0183EF97E00E94AD6272
:10BDE0000A9789F483EF97E00E941B62C00FD11F6E
:10BDF000009749F06AE070E00E944979805D8A937B
:10BE0000862F972FF5CFDF91CF911F910F91089536
:10BE10008F5F0C94D061CF93C82F8031C0F561E063
:10BE2000680F83EF97E00E9429622DEE32E0E9EC83
:10BE3000F1E0DF01C9011D920197E9F74DEE52E0F3
:10BE4000BF0183EF97E00E94AD628F3F910509F03B
:10BE500018F48C2F0E94B15E89EC91E00E94615E23
:10BE600080917104811107C08091DA0186958370F9
:10BE70008E5F809371040E94883A0E9482148091A0
:10BE80003B0D806480933B0DCF910C94E876CF916D
:10BE90000895FF920F931F93CF93DF93CDB7DEB733
:10BEA0002F970FB6F894DEBF0FBECDBF01E0080F8D
:10BEB000102F1031C8F4FF24F394F10E8F2D0E943F
:10BEC000D06181110FC0602F83EF97E00E9429623B
:10BED00061E0610F28E532E042E08AEE97E00E94DF
:10BEE000956306C01F2DE5CF103169F780E01AC0B9
:10BEF0004FE050E0BE016F5F7F4F83EF97E00E94FD
:10BF00004662882351F0482FBE016F5F7F4F8AEE53
:10BF100097E00E941263A895EBCF8AEE97E00E940B
:10BF2000C06381E02F960FB6F894DEBF0FBECDBF81
:10BF3000DF91CF911F910F91FF900895EF920F9392
:10BF40001F93CF93DF930E94BD61882381F10E94EC
:10BF5000336187FD2CC060E083EF97E00E94296287
:10BF600081E6E6EBF4E0DF011D928A95E9F741E610
:10BF700050E0BF0183EF97E00E94AD6287E095E05B
:10BF80000E94615E8091B6048A3028F4809172012B
:10BF90008160809372018AE08093B604C091E104CD
:10BFA000D091E2040E94725EC817D90781F161E066
:10BFB0008DEC93E10E94A61B8BEB93E10E94091389
:10BFC0000E9498610E947F5E88ECE82E01E610E0F6
:10BFD00026EB34E041E060E083EF97E00E94F163FC
:10BFE0008136910529F060E08CEA93E10E94A61B5E
:10BFF00080E00E94B15E98ECE92E0DEE12E029EC93
:10C0000031E042E061E083EF97E00E94F1638091CC
:10C01000E304DF91CF911F910F91EF900C940B5F90
:10C02000882379F09091FE07982B9093FE07F8945F
:10C030008091420C9091430C78949093FD078093EB
:10C04000FC070895EF920F931F93CF934091FE0743
:10C05000442309F47FC0811110C0F8948091420CF0
:10C060009091430C78942091FC073091FD07821B3E
:10C07000930B8436910508F46DC08091E00781111F
:10C0800069C0C42FC47042FD02C081E001C083E0DA
:10C090008093E0071092FE0740FF26C034E1E32EB4
:10C0A00001E610E026EB34E041E061E181EE97E04B
:10C0B0000E94F1638136910519F461E180E029C0A5
:10C0C0008091E707823051F48091FE0781602BC098
:10C0D0008091E707823001F1C1113AC060E083EF3F
:10C0E00093E10E94A61B34C041FF32C024E1E22E3E
:10C0F0000DEE12E029EC31E042E061E181EE97E0E3
:10C100000E94F1638D3E924019F78091E30461E152
:10C110008F5F0E94DE611CC08091FE07C11102C0CA
:10C12000826001C086608093FE07F8948091420C83
:10C130009091430C7894845691099093FD078093D5
:10C14000FC0780917D0C833019F4A89510927D0C2A
:10C150001092E007CF911F910F91EF900895809179
:10C16000FE07882359F081E00E94226080917D0CB7
:10C170008330A9F7A89510927D0CF1CF089540E483
:10C1800050E060E070E08FEF97E00C94C86841E009
:10C1900050E062E070E081E098E00C94C868CF93D2
:10C1A000DF931F92CDB7DEB7698390E1899FB0011D
:10C1B000112441E050E0CE0101960E94C8680F9022
:10C1C000DF91CF910895CF93DF931F92CDB7DEB764
:10C1D00090E1899FB001112441E050E0CE01019629
:10C1E0000E94CC7989810F90DF91CF910895CF93F0
:10C1F000DF93D82FC82F8C2F0E94E360882329F06B
:10C200008C2F0E94E360C82FF6CF609101088C2F1D
:10C210000E94CF60D0930108DF91CF910C94C7604A
:10C22000CF93C0910108CC2359F08C2F0E94E3607A
:10C23000809301080E94C76060E08C2F0E94CF604D
:10C240008C2FCF910895CF93DF9380910108C0E0A8
:10C25000D0E0882321F02F960E94E360FACFCE0130
:10C26000DF91CF910895DF92EF92FF920F931F938A
:10C27000CF93DF9380E8E9ECF1E0DF011D928A952E
:10C28000E9F7C3E0D8E0F12CB4E1FB1205C08091DE
:10C29000010801E018E002C08E01888190E0E12CE5
:10C2A000DD24D394DF0C009701F19C012450310967
:10C2B0002C37310530F4FC01E753FE4F2081222357
:10C2C00071F0EE2029F060E08E2D0E94CF6004C056
:10C2D000F80110820E94BF6080E090E0E4CFD0823D
:10C2E000E82E0E94E36090E0DECFF3942396F5E120
:10C2F000FF12CACFC4E0D0E0FE01E753FE4F8081B9
:10C30000811109C0609101088C2F0E94CF60C093F9
:10C3100001080E94C7602196C038D10569F780E006
:10C32000DF91CF911F910F91FF90EF90DF900895D3
:10C33000CF9380E4EFEFF7E0DF01982F1D929A95FD
:10C34000E9F794E09093FF078093000880E18093E1
:10C35000020884E0C1E0C80F6C2F0E94CF60CF3785
:10C3600011F08C2FF7CF60E08FE70E94CF6084E060
:10C3700080930108CF910C94BF6040E450E060E0EE
:10C3800070E08FEF97E00E94CC798091FF078430B6
:10C3900029F481E090910008903409F080E008953C
:10C3A00090E0FC01EE0FFF1FE80FF91FE150F84F7E
:10C3B00081E09481911101C080E00895CF93DF93D3
:10C3C00090E0EC01CC0FDD1FC80FD91FC150D84F32
:10C3D0008C819D81AE8170E0FB01EE0FFF1FE60FA7
:10C3E000F71FE150F84F2481358146812C833D832E
:10C3F0004E8384839583A683DF91CF910C94BF6095
:10C40000CF9390E09C01220F331F280F391FF901B1
:10C41000E150F84FC481F901ED5FF74F10821182AE
:10C4200012820E94BF60CC2321F08C2FCF910C94FC
:10C43000F760CF910895FC01808190E0FC01EE0F40
:10C44000FF1FE80FF91FEC5FF74F918180819F700C
:10C450000895CF93DF93FC0160831282118270E014
:10C46000CB01880F991F860F971FEC01C150D84F41
:10C470002C812383148215821682FC01EB5FF74F17
:10C48000808182958F70DF91CF910895AF92BF9296
:10C49000CF92DF92EF92FF920F931F93CF93DF9390
:10C4A0001F92CDB7DEB78C01FC01808190E0FC01CA
:10C4B000EE0FFF1FE80FF91FEC5FF74F808121811E
:10C4C000922F9F70F80121813281821B930B7A0198
:10C4D0008417950708F47C015B016701C114D1043E
:10C4E00029F1F8018381882309F164816F5F6483F6
:10C4F00070E0F0E18F9F600D711D112441E050E06C
:10C50000CE0101960E94CC798981F50181935F016A
:10C51000F80184818F3030F0148283810E94E360BF
:10C52000F8018383F1E0CF1AD108D8CFF8018181D7
:10C5300092818E0D9F1D8C199D09928381838E2D72
:10C540008C190F90DF91CF911F910F91FF90EF9079
:10C55000DF90CF90BF90AF9008957F928F929F927F
:10C56000AF92BF92CF92DF92EF92FF920F931F9301
:10C57000CF93DF934C016B018A01C0E0D0E05C01F6
:10C5800025E0A20EB11CC017D107E8F5F4018581A2
:10C590008F7781F0F4014581F42FFF777F2E2F2FC5
:10C5A00030E0C8018C1B9D0B8217930760F4702E3E
:10C5B0007C1A09C041E050E0B501C4010E94466206
:10C5C000813041F320C0E72CF12CC6018C0F9D1F58
:10C5D00047FF06C0A70160E070E00E94C5790CC06B
:10C5E000A701BC01C4010E944662871529F0FE0123
:10C5F000E80FF11DCF0108C0CE0DDF1DF4018581CC
:10C6000087198583C0CFCE01DF91CF911F910F9104
:10C61000FF90EF90DF90CF90BF90AF909F908F9062
:10C620007F900895AF92BF92CF92DF92EF92FF92E8
:10C630000F931F93CF93DF93EC018B01D42E8B814B
:10C64000811111C089819A81892B69F4E880F12CCC
:10C650000E9410618B83F701EE0FFF1FEE0DFF1D8F
:10C66000E150F84F8483CD2C8FE0A82ECC2009F424
:10C6700045C02F813885F8948091420C9091430CED
:10C680007894281B390B37FF02C082E004C08B81ED
:10C69000811103C081E08E8331C09C819F3078F08E
:10C6A0001C820E94E360811106C00E941061682F05
:10C6B0008B810E94CF608B810E94E3608B838B8192
:10C6C000882341F36C819A2D961BBC2C9C1508F491
:10C6D000B92EEB2CF12C70E090E1899F600D711D5B
:10C6E00011246F5F7F4FA701C8010E94C8680E0D1B
:10C6F0001F1D8C818B0D8C83CB18B8CF6D2D70E0F6
:10C700006C19710929813A81260F371F3A832983D1
:10C710008D2D8C19DF91CF911F910F91FF90EF908C
:10C72000DF90CF90BF90AF900895EF92FF920F935C
:10C730001F93CF93DF93EC01F62EE42E89010E9424
:10C7400029626F2D70E0FB01EE0FFF1FE60FF71F50
:10C75000EC5FF74F1082E29430EFE322E182F8942D
:10C760004091420C5091430C7894400F511F5887D0
:10C770004F83DF91CF911F910F91FF90EF9008951C
:10C780001F93CF93DF93EC01888190E0FC01EE0FC3
:10C79000FF1FE80FF91FEC5FF74F898180839A81B3
:10C7A0009F708181807F892B81838B81882329F0F1
:10C7B0000E94E360182F81110BC010E00E94BF603F
:10C7C000112359F0812FDF91CF911F910C94F760C5
:10C7D00060E08B810E94CF60F1CFDF91CF911F91FC
:10C7E00008957F928F929F92AF92BF92CF92DF92E5
:10C7F000EF92FF920F931F93CF93DF931F92CDB7CA
:10C80000DEB76C0159012E2D30E00E94956319822C
:10C810004501E12CF12C77247394F40181914F01AF
:10C820009981811108C071104EC08081811105C0AD
:10C83000772473941CC071100AC080E09F3718F4ED
:10C84000E016F10679F5772089F0782E01C0712C79
:10C85000992341F19068998341E0BE016F5F7F4F5A
:10C86000C6010E9412638130E1F027C0782E99231F
:10C87000C9F041E0BE016F5F7F4FC6010E941263A5
:10C880008130D9F44981B701641B71096A0D7B1DA0
:10C89000C6010E9412639981891719F0981B998328
:10C8A0000CC0198289818F5F8983FFEFEF1AFF0A1D
:10C8B0000E151F0508F0B1CF08C089818F77870159
:10C8C000081B110902C0872DB9CFC6010E94C063A1
:10C8D000C8010F90DF91CF911F910F91FF90EF90C2
:10C8E000DF90CF90BF90AF909F908F907F900895F2
:10C8F00080E094E0E0E4F8E0DF019C011D9221502B
:10C900003040E1F70895FF920F931F93CF93DF9389
:10C91000FA0174913196A491B0E0179693E0B59521
:10C92000A7959A95E1F71A2FDA011396FA01329634
:10C930004491249FA00DB11D1124669566956695BE
:10C9400090E0F0E86F9F800D911D112420E030E011
:10C9500060E0805C974F472F50E0611798F40A2FF2
:10C96000EC01C20FD31FFD01FE2EF01AF71620F4C2
:10C97000F490F9923196F8CFA40FB51F6F5F20584D
:10C980003F4FEBCFDF91CF911F910F91FF90089513
:10C99000FF920F931F93CF93DF9346312CF4842F94
:10C9A000880F840F880FA0C076E0780FA42FBB27D4
:10C9B000A7FDB09520FD08C021FD02C090E005C094
:10C9C0009091410C96FFFACF91E066956695669539
:10C9D000C82FD0E030E8639FC00DD11D1124C05C8A
:10C9E000D74FFE0122FF53C04E3211F07CE0780F8A
:10C9F0008AE04802F0011124E054F1409D012052E8
:10CA0000310937FF03C09D0121513109A90124E0FB
:10CA1000559547952A95E1F780EA849F9001859F77
:10CA2000300D11242E0F3F1F2A5F3B4E85E08823D7
:10CA300081F0F9010491E056FF4F6491A9014F5F25
:10CA40005F4FFA011491F901EF55FF4FF4909A01ED
:10CA500004C010E060E000E0F12C2F5F3F4F99230D
:10CA600021F0009510956095F094DE01AF57BF4F0F
:10CA7000FCE0A034BF0740F408831983FE01E058AE
:10CA8000FF4F6083FC922296815088F62CC023FFD2
:10CA900008C02196292F2195208375E0780F51E059
:10CAA00001C050E025E04202F0011124E751F54EAB
:10CAB00085E04491552311F0843059F03CE0C034B6
:10CAC000D30738F49E012F5F3F4F91114095488363
:10CAD000E901815031968111ECCF4CE0C034D4078C
:10CAE00010F491959883872FDF91CF911F910F912B
:10CAF000FF90089520E00C94C864EF92FF920F938A
:10CB00001F93CF93DF93F62E122F902F9071E92E63
:10CB1000EA01112369F0EE2011F0488102C0FE0104
:10CB20004491202F6F2D0E94C86411502196F1CF9F
:10CB3000DF91CF911F910F91FF90EF9008950F9388
:10CB4000FA0194914F5F5F4F929F400D511D112448
:10CB5000292F0E947D650F9108950F9300E00E9498
:10CB60007D650F910895FF920F931F93CF93DF93ED
:10CB7000062F122F922F9071F92EFA01FF2011F03B
:10CB8000408101C04491EF012196442331F0212FCF
:10CB9000602F0E94C864FE01F1CFDF91CF911F91F9
:10CBA0000F91FF900895AB0120E0682F80E00C9476
:10CBB000B36520E00C94B365FF920F931F93CF935E
:10CBC000DF93082FF62EEA0114E1180F15504C2FB1
:10CBD0004F704A301CF0495C28E002C0405D20E004
:10CBE0006F2D812F0E94C86434E0D695C7953A9581
:10CBF000E1F71013EBCFDF91CF911F910F91FF90D1
:10CC00000895222321F09091410C96FD0895480F3C
:10CC1000669566956695E82FF0E090E8699FE00DCF
:10CC2000F11D1124E05CF74F8E1B982F9E0F941777
:10CC300020F4908190959193F8CF0895962F969532
:10CC400096959695E82FF0E080E8989FE00DF11D0D
:10CC50001124E05CF74F8CE0E034F80758F467707B
:10CC600081E090E0062E01C0880F0A94EAF79081D7
:10CC700098279083089547FF02C0840F4195962F0F
:10CC8000969596959695E82FF0E080E8989FE00DB0
:10CC9000F11D1124E05CF74F677031E001C0330FE4
:10CCA0006A95EAF74423B1F08CE0E034F80790F499
:10CCB000822F90E020FF08C02081232720839595B4
:10CCC0008795282F206803C095958795282F415078
:10CCD0003196E8CF08952FEF0C943B66962F9695EA
:10CCE00096959695282F30E0F90180E8989FE00D01
:10CCF000F11D1124E05CF74F962F940F96959695B1
:10CD0000969580E8989F200D311D1124205C374FA7
:10CD1000862F8770A1E0B0E001C0AA0F8A95EAF7DC
:10CD2000A1958081A827A083E217F30750F4E0586B
:10CD3000FF4F8CE0E034F807E0F490819095908309
:10CD4000F3CF8CE0E034F807A0F4842F992787FD17
:10CD50009095860F911D68E070E00E94497921E06E
:10CD600030E001C0220F8A95EAF721958081822761
:10CD7000808308953F924F925F926F927F928F923D
:10CD80009F92AF92BF92CF92DF92EF92FF920F935A
:10CD90001F93CF93DF93182FB62E802F05FF04C06B
:10CDA00004FF04C002E003C000E001C001E0982FCE
:10CDB0009F77C92EE7FE04C0E1946624639401C006
:10CDC000612C57FF0AC050954095309521953F4FF3
:10CDD0004F4F5F4F7724739401C0712C82FF06C0C0
:10CDE0009CE09093400CCAE0DC2E05C096E0909346
:10CDF000400CB5E0DB2E86FF28C071101D0D283ECB
:10CE000083E038074105510514F01D0D05C0243697
:10CE100031054105510514F01D0D05C02A303105BD
:10CE2000410551050CF01D0D002381F0023031F455
:10CE300024363105410551054CF41D0D2A303105CC
:10CE4000410551051CF41D0D01C01D198091400CB8
:10CE5000810F8093400C023011F490EFC90E8824AA
:10CE60008394F2E09F2EA12CFF24E7FCF094A6E02F
:10CE70005A2E5B0CE82DF0E0EE16FF060CF460C0B5
:10CE80006AE070E0C9010E944979382EEB01E0E3C5
:10CE90004E2E480E2C2D442D6B2D812F0E94C864E0
:10CEA000081131C0C2FE1AC08FEF830D833008F421
:10CEB0009394CE016AE070E00E944979823011F0CB
:10CEC0008430E9F484E3481204C0AA24A394A10E98
:10CED00017C0AA24AA94A10E939412C07EEF472EE5
:10CEE000410E8FEF810FC0FE05C047E06B2D0E9401
:10CEF0006E6603C0652D0E941E66142D01C0A12E12
:10CF0000209709F000E09E01442737FD4095542FFB
:10CF1000211531054105510581F4002331F002301E
:10CF200059F491E0981540F008C0C4FE09C06110A2
:10CF300004C080EFC80E01C000E01D1983949ACF91
:10CF4000AA2061F0492D6CE06B0D8A2D0E946B6662
:10CF5000492D6DE06B0D8A2D0E946B66772039F0AC
:10CF60002C2D4DE26B2D812F8D190E94C86480E01D
:10CF7000DF91CF911F910F91FF90EF90DF90CF90B5
:10CF8000BF90AF909F908F907F906F905F904F90E9
:10CF90003F900895EF920F93022F9A01442737FD97
:10CFA0004095542F95E0E92E0E94BA660F91EF90BC
:10CFB000089520E00C94CA670F931F93CF93DF93DB
:10CFC000182FC62F042FD22F422F0E946E660230D8
:10CFD00038F04D2F6C2F8FEF800F810F0E946E66FF
:10CFE00002501F5F6FEF6C0F6D0F402F812F0E945B
:10CFF0006B66402F6C2F812FDF91CF911F910F9186
:10D000000C946B660F931F93CF93DF93182FC62F4B
:10D01000D22FE42FF0E03297053608F004E60E9F99
:10D02000C0010F9F900D112464E670E00E944979C1
:10D03000062F2D2F6C2F812F0E94DC67002369F0B3
:10D04000D150DC0FCF5F1F5FCD1738F4402F6C2F0E
:10D05000812F0E946B66CF5FF7CFDF91CF911F9139
:10D060000F910895A998AB98AC988BBBAD9AAD98E9
:10D07000AB9AA99A089581E080933F08AA9825E089
:10D080002A95F1F7000085E08A95F1F70000AA9A49
:10D090008CED95E025E02A95F1F7000001970097C7
:10D0A000C9F782EE0E9432688EEA0E94326881EAF5
:10D0B0000E94326886EA0E94326884EA0E943268DE
:10D0C00082EA0E94326880EC0E9432688FE20E94FD
:10D0D000326885E20E94326881E80E94326882E20A
:10D0E0000E9432688FEA0E94326882E28093E404F0
:10D0F00010923F080895CF93C82F81E080933F0896
:10D1000081E80E9432688C2F0E94326810923F089A
:10D11000CF9108958091E4040C947B681F93CF9382
:10D12000DF9381E080933F0810E0C0E4D8E084E022
:10D130000E94326880E10E943268812F806B0E94D9
:10D140003268A998AB9AAC98FE01CE0180589F4FE7
:10D1500020812BBBAD9AAD9821812BBBAD9AAD98A8
:10D1600022812BBBAD9AAD9823812BBBAD9AAD9894
:10D170003496E817F90761F7EF01AB9AA99A1F5F98
:10D180001830A9F610923F08DF91CF911F910895B2
:10D19000BF92CF92DF92EF92FF920F931F93CF93A4
:10D1A000DF937B018A01080F191FEC01E81AF90AC5
:10D1B0006701CC0EDD1EC017D107C1F0B990809178
:10D1C000E0078270E19B05C08823E1F30E94491CBF
:10D1D000F6CFDFBACEBAE09A8DB3B81649F3BDBA2E
:10D1E0008FB7F894E29AE19A8FBFE2CFDF91CF91A7
:10D1F0001F910F91FF90EF90DF90CF90BF90089517
:10D200008091710C1092710C0895FC0180818F70D7
:10D21000880F611181608F709081907F982B90832F
:10D2200081818F5F81838281882351F09F7041F4D7
:10D23000833621F0842F80628093710C11821282D8
:10D240008281883069F148F4813091F188F0823030
:10D2500039F1843009F03FC023C08F35C1F018F494
:10D260008031F1F00895813649F0823671F10895E8
:10D2700080818F708F3079F581E62BC040664093B6
:10D28000710C10924E0610924D068FE522C08181DE
:10D29000803211F4406816C08832E9F480E119C088
:10D2A0009181903328F090E0959587958283118243
:10D2B000828190E00197218130E082239323892BA2
:10D2C00051F440644093710C08958181803418F0CA
:10D2D00088E0828311820895282F30E02F303105B5
:10D2E0006CF4F901EE0FFF1FE20FF31FEC5BF34F3D
:10D2F00090819F7081E09F3071F52EC090E0FC011D
:10D300003F97E930F10538F5E659FF4F0C949E79C7
:10D3100091B194701DC093B390781AC0909163003E
:10D32000917016C0909163009095987011C0809193
:10D33000630083FF10C091B102C091B190959074C9
:10D3400007C091B1907104C093B3F9CF91B19072BD
:10D3500081E0911101C080E008958F7090E08F30DE
:10D36000910551F0FC01EE0FFF1FE80FF91FEC5B78
:10D37000F34F82E68283118208958F7090E08F30A0
:10D38000910549F0FC01EE0FFF1FE80FF91FEC5B60
:10D39000F34F83E682830895EF92FF920F931F93DA
:10D3A000CF93DF938091420C9091430C0196909320
:10D3B000430C8093420C8093410C16B31095C4E447
:10D3C000DCE0F12C11FB662760F94F2DCE010E94A5
:10D3D0000569F3941695239686E0F812F3CFE0B230
:10D3E000E094C9E6DDE100E010E0FC1AFE01849162
:10D3F0004C2F4F0D8E2161E009F460E0C8018A5A7C
:10D40000934F0E94056921960D5F1F4F083111054A
:10D4100069F79091B00161E0C92FC07295FF60E09B
:10D420004EE08EE69CE00E94056986B390E0809510
:10D4300090958E7799278C2B19F089E08093540171
:10D44000DF91CF911F910F91FF90EF900895EF9290
:10D45000FF920F931F93CF93DF93F82E80E04AE063
:10D46000282F30E0429FF001439FF00D1124E75335
:10D47000FE4F928DF91650F5803261F18AE0E82E68
:10D48000E29E8001E39E100D1124E801CD51DE4F94
:10D490006FE170E0621B730BE69EA001E79E500DEA
:10D4A00011242F5F3F4FE29EC001E39E900D112497
:10D4B000BE018D519E4F0E94B379FE011192EA94F4
:10D4C000E9F7F801E753FE4FF28E06C09923A1F267
:10D4D0008F5FC6CFC3EED1E0CE01DF91CF911F9118
:10D4E0000F91FF90EF90089580E491E0E3EEF1E07A
:10D4F000DF019C011D9221503040E1F70895909189
:10D50000FA04E82FF0E084E0989FE00DF11D11246B
:10D51000E05CFC4F84910895FF920F931F93CF938B
:10D52000DF9300D000D0CDB7DEB719821A821B82FC
:10D530001C82E091FF04F0E0E75AFC4F66E070E0E7
:10D5400091E0E4910E2F10E041E050E09801062EAA
:10D5500002C0359527950A94E2F723703327D90145
:10D560001196E1E0F0E0EC0FFD1F2E0F3F1FA41716
:10D57000B50711F4F90190834F5F5F4F45305105B6
:10D58000B1F79F5F625071099530F1F681112CC09F
:10D590000E94746A89810E94276A8C0181E00E943E
:10D5A0007F6AF801818394E6F92EF2828A810E94D3
:10D5B000276A8C0182E00E947F6AF8018183F282EF
:10D5C0008B810E94276A8C0183E00E947F6AF801A8
:10D5D0008183F2828C810E94276A8C0184E00E9400
:10D5E0007F6AF8018183F2820F900F900F900F9065
:10D5F000DF91CF911F910F91FF9008950F931F938B
:10D60000CF93DF939091DF0191FF03C060E075E05D
:10D6100002C060E074E01091DA011295169517705F
:10D62000882331F0A6ECBCE0833021F420E103C074
:10D63000AEE7BCE028E09091D901990F910F920FCD
:10D640004091DC0124E64202A0011124485A5D4FBA
:10D650000091E201E8EEF3E09F010203E001039F85
:10D66000D00D11249E0128533045241B350BFD019C
:10D67000882339F032964D935C93833011F418EF80
:10D68000190FCC27DD27C61BD70B1917F0F4A12FD4
:10D69000B0E0AA0FBB1FAF5BB84F0D90BC91A02D9F
:10D6A0006A177B070CF4DB01AC17BD070CF4DE0135
:10D6B000A854B44F2A1B3B0BA41BB50BB183A0830A
:10D6C000538342831F5F3496E0CF31832083DF0191
:10D6D000882371F01296285E334030937A0C2093A1
:10D6E000790C1D921C92DF91CF911F910F9108959B
:10D6F000149653834283F5CFE0912601F0912701E0
:10D7000029E090E130E0482F4170341302C0905F6F
:10D7100004C091509083319690E1869580682150A5
:10D7200011F0342FF0CF915F9193F0932701E093A4
:10D73000260108951F93CF93DF93182F2EE73CE027
:10D740003093270120932601C09114018C2F8774F8
:10D7500061F08091D901882321F0813021F4C0E962
:10D7600006C0C0E804C0C8E902C0C7FF06C087E120
:10D770000E946C69882309F45AC0C7FD5AC040E072
:10D7800060E085E10E945517882309F452C0C06209
:10D79000C09314018091E3048F5F80931501E7E14A
:10D7A000F1E0A1E4B7E090E06DE0911729F14D912F
:10D7B0005D91649F9001659F300D112485E0359542
:10D7C00027958A95E1F73E5F37FD06C02F3F83E03E
:10D7D00038072CF4822F05C080E030E002C08FEFC4
:10D7E00033E0EF012197292F220F220F232B2883CB
:10D7F00080839F5F3296D9CFC4E1D1E089910E94A6
:10D800007C6B81E0C232D807C9F7E0912601F09124
:10D810002701108231978FEF80838EE79CE09093F1
:10D82000250180932401DF91CF911F910895CF7737
:10D83000A4CFCF7DADCF1F920F920FB60F921124C0
:10D840002F938F939F93EF93FF9388B391E0892752
:10D8500088BBE0912401F0912501CF0101969093BE
:10D860002501809324012081822F90E097BD86BD01
:10D87000293C08F0C09A80917D0C816080937D0CDA
:10D88000FF91EF919F918F912F910F900FBE0F906D
:10D890001F9018951F920F920FB60F9211242F937D
:10D8A0003F938F939F93EF93FF9388B391E08927E2
:10D8B00088BBE0912601F0912701808128B539B518
:10D8C00080FD03C0205E3F4F02C0205F3F4F39BD47
:10D8D00028BD90E095958795009791F4CF0101962A
:10D8E0009093270180932601818181110AC0809144
:10D8F0007800909179008053984F99BD88BD01C000
:10D90000808380917D0C816080937D0CFF91EF91ED
:10D910009F918F913F912F910F900FBE0F901F906D
:10D920001895EDE7F0E08081857E808317981F9A37
:10D93000AAE8B0E01C9210928B0082E88C93808160
:10D94000806280830895EDE7F0E080818F7D8083A1
:10D95000179AAAE8B0E01C9210928B008AE08C9390
:10D9600080818861808308951F920F920FB60F9275
:10D9700011248F939F93EF93FF9380910E0D882333
:10D9800021F01F9A10920E0D04C01F9881E0809321
:10D990000E0DE0911201F09113018081918190931D
:10D9A0008700809386008091790C90917A0C9093F7
:10D9B00085008093840082819381892B11F03296B7
:10D9C00007C08091DF01817080930E0DE6ECFCE0D2
:10D9D000F0931301E093120180917D0C816080939C
:10D9E0007D0CFF91EF919F918F910F900FBE0F9043
:10D9F0001F901895E2E7FCE0208126952695282BBC
:10DA0000208381818F5F8183843048F0A281B3813C
:10DA1000CD010196938382832C9310821182089505
:10DA2000882339F08091780C8F5F8093780C80E8A0
:10DA300003C01092780C80EC0E94FA6C8091780CF4
:10DA40008530B8F70895CF93DF93C82FE091760C17
:10DA5000E827F0E0EE0FFF1FEF58F24E25913491CA
:10DA60004091770C50E0242735273093770C209392
:10DA7000760CD8E08C2F80780E94106DCC0FD1509E
:10DA8000C9F7DF91CF910895CF9380EC0E94FA6C93
:10DA9000C6E080E80E94FA6CC150D9F780ECCF91C3
:10DAA0000C94FA6CEF92FF920F931F93CF93DF9336
:10DAB000C091D8018091020585FF04C08091C50105
:10DAC0008111C4E080917C0C8C1709F48EC0C09346
:10DAD0007C0C1EBC1DBC1CBC87B7837C87BF80919F
:10DAE0007D008E7F80937D008CE386BF8FE38093E3
:10DAF0007C00C23079F118F4C130A1F006C0C33007
:10DB000009F444C0C43009F45DC00E94916C80E403
:10DB10009CE99BBD8ABD87B7806187BF1FBC8AE037
:10DB20008EBD63C00E94916C80E797E199BD88BD6E
:10DB300080EA9FE0909379008093780087B78860AF
:10DB400087BF80917D00816080937D001FBC82E053
:10DB50008EBD56C00E94916C88EC90E09093790045
:10DB6000809378008CE291E09DBD8CBD80EE9BEAB5
:10DB700097BD86BD87B7806287BF80917D00816039
:10DB800080937D001FBC8AE18EBDB9C080E49CE912
:10DB90009BBD8ABD87B7806187BF1FBC8AE08EBDF1
:10DBA00083E00E94FE6A80E593EC90938700809367
:10DBB000860088E893E190938500809384000E941A
:10DBC000A36CA7C084E00E94FE6A80E593EC90936A
:10DBD00087008093860088E893E190938500809386
:10DBE00084000E94A36CC0989DC0C13049F008F425
:10DBF00090C0C23009F483C0C33009F48AC092C017
:10DC00007894E2E7FCE08EE79CE090932701809314
:10DC100026019383828315821482108211821682D8
:10DC20000E94446D8091D9010E94236D80917B0CEC
:10DC30000E94236D80E00E94236D10927B0CC1E452
:10DC4000D7E028813981C901880F991F820F931F5E
:10DC500097FD03967C01F594E794F594E79486E3A9
:10DC6000E81A87EFF80A2A813B81C901880F991FBA
:10DC7000820F931F97FD03968C01159507951595B7
:10DC800007950653174F8E2D0E94236D9F2D9F7071
:10DC9000802F8295807F892B0E94236DC80154E0DC
:10DCA000969587955A95E1F70E94236D249687E013
:10DCB000C135D80731F6C091760C8091770C0E945F
:10DCC000236D8C2F0E94236D0E94446D8091730CF4
:10DCD000882321F080E00E94FA6CF8CFE091740C68
:10DCE000F091750C10828091780090917900805CA1
:10DCF00093469093790080937800C09A13C07894EB
:10DD000086E0DF91CF911F910F91FF90EF900C94DF
:10DD10009A6B80E0DF91CF911F910F91FF90EF9070
:10DD20000C94FE6ADF91CF911F910F91FF90EF90BD
:10DD300008951F920F920FB60F9211242F933F93C5
:10DD40004F935F936F937F938F939F93AF93BF9303
:10DD5000CF93DF93EF93FF938CB59DB520910F0D7B
:10DD6000222321F0C09A10920F0D04C0C09821E028
:10DD700020930F0DC0912201D09123019E012E5FAF
:10DD80003F4F3093230120932201288139813BBDED
:10DD90002ABDE0E1F1E0282F3181381708F48183B2
:10DDA0003081231708F480838A819B81892BD9F4E1
:10DDB0008EE79CE090932301809322018091DF0104
:10DDC0008095817080930F0D87B78F7E87BF0E94EB
:10DDD000526D8091D801882311F0833021F487B7E8
:10DDE000806187BF789480917D0C816080937D0CE9
:10DDF000FF91EF91DF91CF91BF91AF919F918F9163
:10DE00007F916F915F914F913F912F910F900FBE36
:10DE10000F901F9018951F920F920FB60F9211241A
:10DE20002F933F934F935F936F937F938F939F9322
:10DE3000AF93BF93EF93FF938091D8018230C1F4E9
:10DE400080E492EA97BD86BD809178009091790038
:10DE50008F3F910538F488E598E990937900809395
:10DE6000780008C088EC90E0909379008093780067
:10DE70000E94526DFF91EF91BF91AF919F918F9151
:10DE80007F916F915F914F913F912F910F900FBEB6
:10DE90000F901F9018951F920F920FB60F9211249A
:10DEA0002F933F934F935F936F937F938F939F93A2
:10DEB000AF93BF93EF93FF938091D80178949091A3
:10DEC0007C0C981771F0943061F48091C50188231F
:10DED00021F08091020585FD03C00E94526D03C0B0
:10DEE00084E00E94FE6AFF91EF91BF91AF919F91F4
:10DEF0008F917F916F915F914F913F912F910F90F3
:10DF00000FBE0F901F9018959091F904987390315F
:10DF100029F49BEA899F812D112402C0983111F4C4
:10DF200086950895983211F4880F0895903319F466
:10DF3000982F990F890F0895FC01A5E6B0E08C9108
:10DF40008B7F8C93148215821082118216A617A6DD
:10DF500008950C949C6F21E0FC018481811101C023
:10DF600020E0822F0895FC0121818081281B2770E9
:10DF700098E0921B81E0933008F480E00895CF93FD
:10DF8000DF93FC0184818823F1F0815084838281B6
:10DF90009381890F828386A58823F1F187A59FEF5E
:10DFA000980F97A7882331F0809165008460809353
:10DFB000650032C0809165008B7F80936500809101
:10DFC000040587A729C01B98809165008B7F8093EB
:10DFD00065008581882319F0815085831DC080816B
:10DFE00091818917C9F090E0EF01C80FD91F2E81E8
:10DFF00022832E8924832E8523832E8D258328A991
:10E0000026A717A62EA13FEF320F3EA3211104C071
:10E010000196877099278083DF91CF9108958F9221
:10E020009F92AF92BF92CF92DF92EF92FF920F93A7
:10E030001F93CF93DF935C01162FD42EF22E0E94F4
:10E04000B36F882339F19091F904987319F1F501B0
:10E05000C181D0E04E01FFEF8F1A9F0A87E088222E
:10E060009924F50180818815A9F0112329F0909158
:10E070000305965F910F01C090E0CA0DDB1D9E83E2
:10E080008D2D0E94846F8E8BFE8EE8AA0EA3CE8605
:10E09000F5018182DF91CF911F910F91FF90EF9059
:10E0A000DF90CF90BF90AF909F908F900895CF92C8
:10E0B000DF92EF92FF920F931F93CF93DF93EC01C8
:10E0C000162FF42ED22E0E94B36F882301F1909167
:10E0D000F9049873E1F0112329F090910305965FFC
:10E0E000910F01C090E09A838F2D0E94846F8C83E2
:10E0F000DD82EEA61FA6CB8288818983002339F0BA
:10E1000001502D2D4F2D612FCE010E940F70DF91F8
:10E11000CF911F910F91FF90EF90DF90CF900895D6
:10E12000CF92EF920F931F93CF93DF93EC01062FC3
:10E13000642F8091F904869586958695877038813D
:10E140002981321364C110E00132110508F05FC16A
:10E15000F801ED58FF4F0C949E79C12CEE24E39406
:10E1600000E021E03AC1C12CEE24E39400E021E07C
:10E170002EC1C12CEE24E39400E021E04EE12EC13B
:10E1800092E0C92EEE24E39402E022E04AE064E645
:10E190003BC1C12CEE24E3940AE022E045E06FE5A8
:10E1A000CE010E940F7001E02AE045E06FE5CE014C
:10E1B0000E940F700AE022E045E06FE525C1CC2403
:10E1C000CA94E12C02E023E04AE060E5CE010E941F
:10E1D0000F70CC24C39423E04AE06CE3CE010E948C
:10E1E0000F70C12C82E0E82E00E021E04AE06FC011
:10E1F000C12CEE24E39401E021E045E066E4CE0189
:10E200000E940F7022E04FE062E3CE010E940F7087
:10E2100022E04FE0F8C0C12CEE24E39402E021E0BC
:10E2200045E06EE6CE010E940F7003E021E045E07C
:10E230006CE7EAC0C12CE12C00E025E045E062E398
:10E24000CE010E940F7025E045E06AE5CE010E94F4
:10E250000F7002E024E043E06EE6D6C0C12CEE244D
:10E26000E39403E02AE045E060E5CE010E940F70F0
:10E2700001E024E145E060E5CE010E940F7003E07B
:10E280002AE045E0C0C0CC24C394EE24E39402E02D
:10E2900025E044E16AE0B8C0C12CEE24E39402E03A
:10E2A0002AE044E062E3CE010E940F7001E024E125
:10E2B00048E066E4CE010E940F7002E02AE048E0E8
:10E2C00062E3CE010E940F7001E024E144E066E4C5
:10E2D0009BC0C12CEE24E3940AE02AE005C0C12CC7
:10E2E000EE24E39402E022E345E068E78DC0C12C10
:10E2F000EE24E39401E009C0C12CEE24E39402E093
:10E3000004C0C12CEE24E39403E02AE044E160E081
:10E310007BC0C12CEE24E39400E021E048E25EC023
:10E32000813009F474C0C12CE12C00E021E04AE006
:10E330006BE455C0813009F46AC0C12CE12C00E0C7
:10E3400021E04AE061E44BC0C12CE12C00E021E077
:10E3500046E045C0C12CEE24E39405C0813009F4A9
:10E3600056C0C12CE12C00E037C0C12CE12C00E0EC
:10E3700004C0C12CEE24E39401E021E04AE020C077
:10E38000C12CEE24E39402E021E04AE06AE727C0D2
:10E39000C12CEE24E39403E021E04AE06CE71FC0C7
:10E3A000C12CEE24E39403E009C0C12CEE24E394D5
:10E3B00002E004C0C12CEE24E39401E023E04FE02E
:10E3C00068E70DC0C12CEE24E39401E029E144E1AB
:10E3D00005C0C12CE12C02E022E04AE066E4CE0157
:10E3E0000E94577014C0CC24C394E12C02E023E0B7
:10E3F00044E16CE3CE010E940F70CC24CA94EE2459
:10E40000E39423E044E160E5CE010E940F70DF91C8
:10E41000CF911F910F91EF90CF90089546E4682F10
:10E4200083E791E00C9490709091050591FF03C0F3
:10E43000862F0C94A4140C940E72FF920F931F93CA
:10E44000CF93DF93EC01162FF42E47FF03C0842FE8
:10E450000E94A414D7FF06C0D195C195D1098AE1C5
:10E460000E94A414112371F0123019F464E670E0D4
:10E4700002C06AE070E0CE010E944979262FC22FC7
:10E48000D72F082F64E670E0CE010E9449799B01E6
:10E49000562F482FC82FD92F2115310551F12A3079
:10E4A0003105DCF06AE070E0C9010E9449799B0106
:10E4B0008C01EC01653171051CF48EE6820F05C0FC
:10E4C0008CE8820F0E949F148EE60E94A41401150E
:10E4D000110559F1502F11E001C010E084E6850FBD
:10E4E0000E94A414111121C02097F9F08C2F845799
:10E4F00015C08CE8840F0E949F141123B1F01230D4
:10E5000081F46AE070E0802F90E00E944979C82F82
:10E5100086E0860F0E94A4148CE88C0F0E949F1442
:10E5200004C086E0800F0E94A4141F1444F48F2DB1
:10E53000DF91CF911F910F91FF900C94A414DF9164
:10E54000CF911F910F91FF9008950895CF93C82FF9
:10E55000843089F48AE09B01829FB001839F700D13
:10E5600011248091160E882391F17093150E6093FB
:10E57000140EC8E22CC0853039F58091160E6A3031
:10E58000710510F4816001C083608093160E809144
:10E59000160E81FF05C0CB016AE070E00E9435795C
:10E5A0002091140E3091150E121613062CF04427EC
:10E5B0005527461B570B01C0AB01240F351F309365
:10E5C000690D2093680D03C0893208F09EC08091C8
:10E5D000D501EC2FF0E084FD07C0EE0FFF1FE05ADD
:10E5E000F24F718360831AC0C430D1F0EE0FFF1F69
:10E5F000E05AF24F71836083C63081F420916C0D34
:10E6000030916D0D4AE0429FC001439F900D11244F
:10E610009093690D8093680DC4E002C0C930A8F4DE
:10E620002C2F30E0220F331FF901E05AF24F4081C6
:10E630005181F901E25BF24F2081318124173507C6
:10E640000CF047C05183408344C0C03139F5462F98
:10E6500042954F70842F90E02091410D30E0821759
:10E66000930754F08530910524F026E02093410D66
:10E6700003C04F5F4093410DFC01EE5BF24FCB01B5
:10E680008F709927982F8827672F7727860F971FD6
:10E690006AE070E00E943579608337C0CC30C9F4FD
:10E6A000A091780DB091790D2CE330E00E940B79A8
:10E6B00020917104211103C021E02093710430E006
:10E6C00040E050E00E945D793093790D2093780D01
:10E6D0001CC0C232D1F48091A20D9091A30D4AE0EA
:10E6E000489F9001499F300D1124260F371F45E1A7
:10E6F000429FC001439F900D11246BE070E00E9487
:10E7000035797093AD0D6093AC0DCF9108959091D4
:10E71000D50193FD42C09091B50D911105C08E3584
:10E7200009F04DC081E026C08E35E1F38D3521F42E
:10E7300081E08093B40D08952091B40D222321F03F
:10E740001092B40D20E68227913079F48A3308F0D4
:10E750008151803309F487E2E82FF0E0EF58F04E62
:10E76000E491E093B30D82E005C0923031F48093E0
:10E77000B20D83E08093B50D0895682F70E0762F79
:10E7800066278091B20D680F711D8091B30D8F7750
:10E790000E94A6721092B50D08959091EA0D9035E1
:10E7A00018F48093B20D0895682F70E0762F6627D5
:10E7B0008091B20D680F711D84E00C94A6720895CB
:10E7C0001F920F920FB60F9211248F939F93EF9386
:10E7D000FF93ECEEFDE08389882359F08150838B11
:10E7E000848991E0980F948BE80FF11D80818CB99A
:10E7F00001C05598FF91EF919F918F910F900FBE9F
:10E800000F901F901895282F30E0F901EE0FFF1F91
:10E81000EE0FFF1FEA59FB4F8381582F5F70482F7F
:10E820004295437097E0929FD001939FB00D1124C1
:10E83000A253B24F2C91837041F0918140FF03C0ED
:10E84000921718F40895291790F0852F90E0959568
:10E85000879595958795009711F480E0089532810A
:10E8600041FF03C0321718F0F8CF2317B0F708950F
:10E87000E82FF0E0E451F24F93E8960F923018F051
:10E8800060838F5F089560529DE790838F5F31961C
:10E89000F7CFCF93DF93D42FC22F9EE79093EC0D49
:10E8A0008093ED0D82E00E943874E82FF0E0E4518F
:10E8B000F24FD083C1831282138214821582168292
:10E8C0009EE79783885F8093FF0DDF91CF91089536
:10E8D000FC018181848310820895FC0185819681E9
:10E8E000860F911D9683858320913E0D203110F176
:10E8F00074E0959587957A95E1F7818324812817AF
:10E9000010F4821B01C080E08083A42FB0E0AA0F26
:10E91000BB1FA05AB24F90E08D939C9383818617C2
:10E9200008F463838281882311F0681708F46283F6
:10E93000168215820895FF920F931F93CF93DF9352
:10E94000EC0188818D3F78F4893F98F4863F09F483
:10E9500048C0873F09F05BC089818093C50D8B81DA
:10E960008093C30D54C08D3F09F442C08E3FA1F087
:10E970004EC090E0895F9109FC01EE0FFF1FE80F88
:10E98000F91FEA54F24F898182838A8181708183E1
:10E990008B81837080833BC080913E0D8F5F80931D
:10E9A0003E0D40E069818EEC9DE00E946D7441E077
:10E9B0006A8185ED9DE00E946D7442E06B818CED73
:10E9C0009DE00E946D746C81669543E083EE9DE04E
:10E9D0000E946D7480913E0D8031C8F010923E0D02
:10E9E00016C089818093C40D8B818093C20D0FC0A6
:10E9F00019811D5F239603E0EAE5FE2E011738F426
:10EA000089910E948773F092EA0D0F5FF7CF83E23E
:10EA10008093EB0DDF91CF911F910F91FF9008959F
:10EA20001F920F920FB60F9211242F933F934F9383
:10EA30005F936F937F938F939F93AF93BF93EF9366
:10EA4000FF93579878949BB18CB19C7119F01092F8
:10EA5000180E80C09091170E9230D9F030F499239F
:10EA600009F440C0913049F075C0943009F446C0B3
:10EA700030F1953009F44AC06DC08E3709F46AC090
:10EA800092E09093170EE091180EE33108F062C007
:10EA90000DC08D3711F483E02AC08E3729F481E050
:10EAA0009EE00E949B7454C0E091180E91E09E0F6E
:10EAB0009093180EF0E0EF5FF14F80834BC092E02F
:10EAC0009093170EE091180EE33108F043C091E0E7
:10EAD0009E0F9093180EF0E0EF5FF14F90E29827B1
:10EAE000908338C08E3731F41092180E81E08093F5
:10EAF000170E30C08B3171F584E0F9CF95E090931B
:10EB0000170E80933D0D10923C0D24C090913C0D4A
:10EB100091110CC0982F9F7349F494B3906C94BBDF
:10EB200025B3982F907C2F73922B95BB90913C0D21
:10EB3000913019F48093AE0104C0923011F48093A7
:10EB4000B3019F5F90933C0D80913D0D981302C0DF
:10EB50001092170EF894579AFF91EF91BF91AF91D1
:10EB60009F918F917F916F915F914F913F912F91E5
:10EB70000F900FBE0F901F901895EEECFDE01282E3
:10EB8000138211861286108A118A178A108E1092AB
:10EB90007D0D10927C0D10927F0D10927E0D1092C3
:10EBA000A70D1092A60D1092400D10923F0D1092DD
:10EBB000A90D1092A80D08958CE0E6EBFDE0DF01B1
:10EBC0001D928A95E9F70E94BD75109818981092C9
:10EBD000900087E689B959981AB886E08093950025
:10EBE0005F9B02C08CB1FCCF1092FF0D8AB188628E
:10EBF0008AB9549A579A0895E6ECFDE09091CE0DAB
:10EC0000882319F034969091D50D22813381290FF4
:10EC1000311D33832283408151814217530778F499
:10EC2000241B350B3383228390E0880F991F84586F
:10EC3000924FFC0180819181019691838083089598
:10EC40008091EB0D882349F081508093EB0D811169
:10EC500004C01092670D1092660D8091EA0D882312
:10EC600019F081508093EA0D20913B0D222309F485
:10EC70007AC080913A0D882321F0815080933A0D1B
:10EC800072C08091FF0D81116EC091E0392F322347
:10EC900021F48F5F990F8730C9F790959223909355
:10ECA0003B0D843008F041C0982F969521E0622FEB
:10ECB000691B982F917092272091FC0470E027FD2A
:10ECC00013C0FB01EE0FFF1FEE0FFF1FE759FB4FB5
:10ECD00020812F7030E0492F440F02C035952795D1
:10ECE0004A95E2F7237001C020E0FB01EE0FFF1F01
:10ECF000EE0FFF1FE759FB4F40814295437050E0F4
:10ED0000092E02C0559547950A94E2F74170660FA7
:10ED1000771F660F771F67537E4F690F711DFB01C9
:10ED2000E256FD4F6081875016C0863070F48170C6
:10ED3000282F30E0D901AE53B24FF901EC53F24F16
:10ED40002C9140E060818A5006C0863061F420E05A
:10ED500040E060E081EF0E94497485E080933A0DC5
:10ED60001092000E559A8091EB0D882381F08091CE
:10ED70006904807C803C19F480E00E94FC758091DD
:10ED80006D04807C803C19F481E00E94FC758091C8
:10ED9000EA0D8823E1F08091A00D9091A10D2091C2
:10EDA0003F0D3091400D820F931F81312EE092076D
:10EDB00050F080519E40E8EAFDE0208131812F5FD4
:10EDC0003F4F318320839093400D80933F0D0895F2
:10EDD000CF92DF92EF92FF921092410D80913B0D06
:10EDE0008F6080933B0D2091660430E040E050E05E
:10EDF000B0E4CB2EBEE7DB2EB5E0EB2EF12CC70145
:10EE0000B6010E947F793093C70D2093C60D2091E3
:10EE10006A0430E040E050E0C701B6010E947F790B
:10EE20003093CB0D2093CA0DFF90EF90DF90CF90E1
:10EE3000089586B380958E7708958FEF8ABB1BBAAD
:10EE400091E897BB9EE798BB9EE394BB91EC95BB82
:10EE500011BA82BB88E082B987EF83B91092610052
:10EE60001092620084E1809364008BEF80936500D0
:10EE70000E943B680E94DC7580E487B985E886B90A
:10EE800087E083BF8CE981BF82E085BD87B783645B
:10EE900087BF1FBC8AE08EBD10928B0082E88093F2
:10EEA0008A0080917D00806280937D0078948BE35E
:10EEB00096E490934B0180934A0189E10E947B681C
:10EEC0000E949E5FD090E3040E941977C0E081FD0C
:10EED00005C08695CF5FC730D1F71FC0C630E9F0B7
:10EEE0008C2F0E94085F8823C1F0C093E3048C2F0D
:10EEF0000E940B5F81E00E9410600E94786424E011
:10EF000049EA51E060E086E10E94B36588E10E9431
:10EF1000D1120E948E680E9498120E948A6881E035
:10EF200080933A010E948F1810923A010E94A71410
:10EF30008091FC0484FF05C08091F90482FD4FC0DC
:10EF400044C080910505882321F06CE187E00E9490
:10EF500014720E946E180E94786420E048E753E023
:10EF600060E080E00E9483648091020584FD08C017
:10EF700000E12AE047E055E068E380E00E947D651B
:10EF80000E948E680E948A680E9498120E94FA0F5E
:10EF90000E949A158C01F894C091420CD091430CB8
:10EFA0007894C057DE4F0E948E680E946E180E94AF
:10EFB000FA0F0E949A157C010E9419778111BCCF2B
:10EFC000E016F10609F4FEC0B7CF0E942361883C29
:10EFD000910528F460E08AE991E00E94A61B0E9456
:10EFE000FA0F8091F90480FD39C08091FA04817094
:10EFF00012E0181B0E94FA0FE12FF0E0EE0FFF1F46
:10F00000EA54FB4F218132818091FC0480FF06C0CD
:10F01000319521953109458D568D02C0478550891E
:10F02000241B350BE9016096812F0E94B415C81787
:10F03000D907A4F46BE871E089E791E00E949F1280
:10F040000E94FA0F0E946E18812F0E94B415C817F3
:10F05000D90724F40E941977882391F3D0911105E0
:10F060008091F90481FD56C08D2F8873883041F05E
:10F07000803131F0803221F0D77CD860D0931105F7
:10F0800016E1C0E0812F0E946C69CC0FC82B115093
:10F090001E30C1F71C2F1D2763E671E08DE993E157
:10F0A0000E949F1210FF04C060E082E00E94C5121F
:10F0B00011FF04C063E087E10E94C51212FF04C083
:10F0C00066E08CE20E94C512812F887371F0C3FF45
:10F0D00002C069E007C0C4FF02C06CE003C0C5FF06
:10F0E00004C06FE081E40E94C51216FF04C062E113
:10F0F00086E50E94C51217FF04C065E18BE60E94F9
:10F10000C5120E948E68CD1729F00E9419778823B6
:10F1100009F463C08091F904887B29F460E083E5F9
:10F1200091E00E94A61B80917201882351F060E05B
:10F1300088E291E00E94A61B809172018E7F8093ED
:10F1400072010E94981280EF90E0909301018093E9
:10F1500000018091D3010E949F140E94526D2DE006
:10F1600088E190E00FB6F894A89581BD0FBE21BD4F
:10F1700060E081E497E00E946C3D80E297E3909329
:10F180004D0180934C010E948A688091E304D81657
:10F1900029F081E00E9410600E94AF6080913B0DD9
:10F1A000806480933B0D80ED97E09BBD8ABD80E13C
:10F1B00086BF81E08093C60187B7806187BF0E94C8
:10F1C000491CFDCFF8948091420C9091430C7894A7
:10F1D000C817D90709F0E7CEAFCE0E946E1850CFFE
:10F1E00083E791E00C94A96F0E94FC78332312F41A
:10F1F0008A1B9B0B0C940D79A29FB001B39FC00199
:10F20000A39F700D811D1124911DB29F700D811D52
:10F210001124911D08950E94FC78B7FF0895821B68
:10F22000930B08950E94FC78A59F900DB49F900DBC
:10F23000A49F800D911D11240895B7FF0C9412799D
:10F240000E941279821B930B0895DB018F939F9389
:10F250000E941279BF91AF91A29F800D911DA39F33
:10F26000900DB29F900D11240895AA1BBB1B51E174
:10F2700007C0AA1FBB1FA617B70710F0A61BB70B26
:10F28000881F991F5A95A9F780959095BC01CD01CB
:10F29000089597FB072E16F4009407D077FD09D048
:10F2A0000E94357907FC05D03EF4909581959F4FDB
:10F2B0000895709561957F4F0895A1E21A2EAA1BBB
:10F2C000BB1BFD010DC0AA1FBB1FEE1FFF1FA21716
:10F2D000B307E407F50720F0A21BB30BE40BF50B13
:10F2E000661F771F881F991F1A9469F7609570959C
:10F2F000809590959B01AC01BD01CF010895052E2D
:10F3000097FB1EF400940E94967957FD07D00E9447
:10F310005D7907FC03D04EF40C9496795095409596
:10F32000309521953F4F4F4F5F4F089590958095B1
:10F33000709561957F4F8F4F9F4F0895EE0FFF1F80
:10F340000590F491E02D0994FB01DC0141505040FF
:10F3500048F005900D920020C9F701C01D92415060
:10F360005040E0F708956817790768F4FB01DC0165
:10F37000E40FF51FA40FB51F02C002900E9241507A
:10F380005040D8F708950C94DC79DC0101C06D93EE
:10F3900041505040E0F70895DC01CB01FC01E199B8
:10F3A000FECF06C0FFBBEEBBE09A31960DB20D92C8
:10F3B00041505040B8F70895FB01DC0102C00190B4
:0EF3C0000D9241505040D8F70895F894FFCFB9
:10F3CE00F0004AAB03AC03AD03AE036400000A02C7
:10F3DE00FF00C60CFF0000AA05FF09FF0DFF135426
:08F3EE0014AA7E0C7E0C7E0CBB
:00000001FF
